:1000000000000420B1C90400D9C90400DBC9040000
:10001000DDC90400DFC90400E1C9040000000000DC
:10002000000000000000000000000000E3C9040020
:10003000E5C9040000000000E7C90400E9C90400A4
:10004000D9C80400B9B20400956E0000EBC90400E1
:10005000EBC90400EBC90400EBC90400EBC90400C0
:10006000EBC90400EBC90400EBC90400EBC90400B0
:10007000EBC90400E96A0000EBC90400EBC9040005
:10008000EBC90400EBC90400EBC90400EBC9040090
:10009000EBC90400EBC90400EBC90400EBC9040080
:1000A000EBC90400EBC90400EBC90400EBC9040070
:1000B000EBC90400EBC904000000000000000000D0
:1000C000EBC90400EBC90400EBC90400EBC9040050
:1000D000995E0000EBC90400EBC90400EBC9040001
:1000E000EBC90400EBC90400EBC9040000000000E8
:1000F00000000000EBC9040000000000EBC9040090
:1001000000000000000000000000000000000000EF
:1001100000000000000000000000000000000000DF
:1001200000000000000000000000000000000000CF
:1001300000000000000000000000000000000000BF
:1001400000000000000000000000000000000000AF
:10015000000000000000000000000000000000009F
:10016000000000000000000000000000000000008F
:10017000000000000000000000000000000000007F
:10018000000000000000000000000000000000006F
:10019000000000000000000000000000000000005F
:1001A000000000000000000000000000000000004F
:1001B000000000000000000000000000000000003F
:1001C000000000000000000000000000000000002F
:1001D000000000000000000000000000000000001F
:1001E000000000000000000000000000000000000F
:1001F00000000000000000000000000000000000FF
:100200000348044B834202D0034B03B118477047A5
:10021000E0030020E003002000000000054806493C
:100220000B1AD90F01EBA301491002D0034B03B104
:1002300018477047E0030020E003002000000000A2
:1002400010B5064C237843B9FFF7DAFF044B13B11E
:100250000448AFF300800123237010BDE0030020A9
:10026000000000007C00080008B5044B1BB10449E5
:100270000448AFF30080BDE80840CFE7000000006D
:10028000E40300207C000800A3F5803A704700BF1B
:10029000154B002B08BF114B9D46FFF7F5FF0021C2
:1002A0008B460F461148124A121A68F089FB0C4B14
:1002B000002B00D098470B4B002B00D09847002014
:1002C000002104000D000B4867F014FA67F0AEFF40
:1002D0002000290000F038FC67F076FA00000800E2
:1002E000000000000000000000000420E0030020E7
:1002F000DC430120117C0600C36823F04A0343F06D
:100300000803C360704770B5856804464DB1284640
:1003100050F8046B5EF016FE28464CF084FC35461F
:10032000F4E7626820689200294668F049FB23469A
:10033000C4E9025553F8180B984201D04CF073FCF5
:10034000204670BD8268002322B1117F12680B44E1
:10035000DBB2F9E7C068B3FBF0F070472DE9F04776
:10036000B4B03D4FDFF80491054612A8884658F016
:10037000B1FA3A4B12930024BB68ADF8BC4053F875
:100380000C2CF9682E94D0326A44CDE93044CDE982
:100390003244009342F8D01C019453F80C0C2146CF
:1003A000684458F036FA3B69029353F80C0C7B69A9
:1003B00002AE21463350304458F02BFA7B68BA69BC
:1003C00053F80C3CD0336B440AA843F8D02C244B90
:1003D000009303F1280214330293224B1292CDE9C9
:1003E0000334CDE90544CDE9074409944DF06EFB93
:1003F0001D4B039318230B9303A90EAB12A8CDE951
:100400000C348DF8384058F004FA444608F1100ACC
:100410004FF030074FF00208544512D0494630469D
:100420005EF019F8026852F80C2C03461344394662
:10043000C3F808805EF068F814F8011B5EF0D6F887
:10044000EAE703A928465EF0AEF968465EF0CEFB07
:10045000284634B0BDE8F0879CDB07000CD20700CB
:10046000D0DB070094DC0700D8DA0700F9020000AF
:100470002DE9F84398460368064653F821000D46D7
:10048000174658B104688146236A984510D17A68A6
:10049000A3689A420CD12AB9D9F80000BDE8F883C4
:1004A0000446F1E76168386868F042F90028F3D043
:1004B00020680028F2D07368A146046AB4FBF3F206
:1004C00003FB1244A542EBD00020E7E72DE9F043FF
:1004D000594A044687B00E46D1E900014CF0A6FB0C
:1004E0006368B0FBF3F703FB170780460346324609
:1004F00039462046FFF7BCFF814618B11C3007B0D3
:10050000BDE8F08324204CF0C5FB3246034652F888
:10051000081B43F80C9B91420546436042D11146AB
:1005200006F1180051F804CB43F804CB8142F9D10D
:100530007368AB604FF00009C6F8049086F8089025
:100540000123326004F1100100936268E36885F8CA
:100550001C9004A858F07CF89DF81030002B49D06E
:10056000059F012F22D1264646F8189FA446002059
:10057000A2684CF8080F82B3136AB3FBF7F107FBCC
:100580001133D2F800E056F82310F9B9A1681160D0
:10059000A26046F823C0116809B146F82020184629
:1005A0007246E8E7B3684160C360C1E7B7F1005F36
:1005B00001D357F0DDFFBA00104603924CF06AFBFE
:1005C000039A4946064668F0FBF9CFE709681160CF
:1005D00056F823301A600346E1E7234653F8180B18
:1005E000984201D04CF01FFBB8FBF7F3C4E9006759
:1005F00007FB13872368C5F8208053F82720B8002D
:1006000052B112682A6053F827301D60E368013345
:10061000E36005F11C0072E7A2682A60A5603AB1A8
:10062000126A6168B2FBF1F601FB162243F8225010
:1006300004F108021A50E9E707690FC7F0B595B051
:100640006D469DF8687085E80F002F48072100F07F
:100650003BF9092F3C4620D9642F34BF02260326DC
:100660000AAB2D22314608A808935EF0C2FC089B15
:10067000264A1E444FF0640C632C10D9B4FBFCF0E6
:100680000CFB1041044602EB410012F811104078B7
:1006900006F8010C06F8021DEEE70126E0E7092C3A
:1006A00085BF1A4A02EB4401303412F8142083BF8C
:1006B000497859701A701C70089C20466AF040FAFC
:1006C00081B2204600F000F90221114800F0FCF848
:1006D00095E80F0004AC84E80F0021460EA8FFF750
:1006E0003DFE0EA90B48FFF7F1FE07700EA85EF065
:1006F00029FC0848FFF726FE044608A85EF022FC05
:10070000204615B0F0BD00BFE4350700EC3507000A
:1007100058530700FC03002010B50E4C20464CF047
:1007200005FB0D4A0D4920464CF078FA0C4800F1C3
:10073000180301224FF07E5103600023C0E901231A
:100740000161BDE81040C0E90533034A0549C360B3
:100750004CF064BA180400200000002095CF04007B
:10076000FC03002007030000094A138873B9094BF2
:100770001988094B1B88C3F500608142C8BF81B24C
:10078000118019B10548184406F002BC704700BF3B
:100790001C060020200E00201E0E00201E06002039
:1007A0000749084A0B8810880344C3F30A030B80E7
:1007B00005490B881B1A0B8000231380FFF7D4BF59
:1007C0001E0E00201C060020200E00202DE9F743FD
:1007D000364FB7F800900E461346B9F1000F1BD103
:1007E0000A4633484FF400616CF0A0F8B0F5006F92
:1007F000044607D32F48314606F025FE204603B0B5
:10080000BDE8F0832C4B3880A3F800902B4BA3F865
:100810000090FFF7A9FFF1E7DFF89C802448B8F8C3
:1008200000500192A944C9F30A094D458CBFA5EBBC
:100830000905C9F50065ADB20A46484429466CF081
:1008400075F8041E04DA1B48314606F0FCFDE0E7AB
:10085000A54203DD3B8823443B80DAE7B4F5006F13
:1008600020DA3B886BB1FFF77FFF06F081FB10B900
:10087000FFF796FFF5E706F095FC0146104806F0F5
:10088000E2FD019B0A4832464FF400616CF04EF8DD
:10089000041E00DCFEE7094A3C800023A8F8003073
:1008A0001380B6E707483146CFE700BF200E00208F
:1008B0001E060020B53607001E0E00201C06002074
:1008C000D6360700EF3607002DE9F843184E194FCA
:1008D0000D464FF0000845B33488B7F800E01649DC
:1008E000C4F50064A4B2AC4228BF2C4600EB040956
:1008F00048450BD0338810F801CB0EEB0302C2F34E
:100900000A02013301F802C03380F1E72D1BADB2BA
:100910004444FFF729FF1FFA84F825B106F028FBAD
:1009200018B9FFF73DFF4846D5E74046BDE8F883D4
:10093000200E00201E0E00201E060020F8B52A4FB3
:100940002A4C05464618AE424CD92B780D2B26D0A2
:1009500011D8082B11D00A2B1DD02388B3F5FF7FA7
:1009600030D801212846FFF7AFFF23885A1C228088
:1009700029781F4A0DE07F2BEFD1238813B3032181
:100980001C48FFF7A1FF2388194A013B9BB2238033
:100990000021D15416E0184B1B780D2B12D00221E8
:1009A0003846FFF791FF238811490022581ECA5488
:1009B000944601445BB902B123800D4801F0BAFCB2
:1009C000002323800C4B15F8012B1A70BBE7087825
:1009D0000A2801D00D28EED1013B01F801C99BB2D4
:1009E0000122E7E7F8BD00BF0C3707001A06002018
:1009F0001A0400200937070019040020FFF7D0BEB1
:100A000007B50A49019000230B8009490B80094969
:100A10000B8009490B8006F0ABF9019A0749104693
:100A200003B05DF804EB01F083BC00BF1A060020A0
:100A30001E0E0020200E00201C060020CD07000006
:100A4000F0B5E5B004A9054606F09CFB24A904A86E
:100A500006F06BFB8022002104A867F0B1FF0123A0
:100A6000114A8DF88C308DF88B30104B1A926A46F3
:100A7000164603F1100718685968344603C4083352
:100A8000BB422646F7D10FCA0CAC84E80F00012305
:100A900024A904A88DF8863006F05BFB24A928461B
:100AA00006F0FFFA65B0F0BDCDAB1A000E370700B7
:100AB000F0B5054697B0084614460E4606F0CEFC43
:100AC0001323014607AA304606F0CCFC9DF81C30E3
:100AD0000093E3696169A2692069174FFFF7AEFDD2
:100AE00003AC2622387000210CA867F069FF21466C
:100AF000124806F0D0FB94E80F0010AE86E80F0015
:100B000040F2BC4300212846ADF8523007F040F8CF
:100B1000044670B10122394606F0A2FC30B90849FA
:100B20000CAB2246284607F065F810B1204606F0C7
:100B30008FFC17B0F0BD00BF220E00201E3707004B
:100B4000240E002070470000F0B5204F87B0054606
:100B50000E463146284605F0BDFE06F025FB04464C
:100B6000FFF74EFF2046FFF76BFF0121204606F0FE
:100B700037FB34220021384667F022FF1022002183
:100B800001A867F01DFF40F2BC43114AADF81430D4
:100B900039462346204607F009F83946012301AAC1
:100BA000204607F01DF80121204606F06CFE05F0F6
:100BB000BBFE18B1204606F003FBCAE7204606F04C
:100BC000CFFC204605F0B6FEF1E700BF240E002062
:100BD000B10A000008B5034A0349083004F02DFDAE
:100BE000002008BD263707001B3A070010B50C6827
:100BF00024B9806806F0E6FA204610BD2320FCE701
:100C0000803002F08BBA00002DE9FF410D680446E8
:100C10000E4685B908306549039004F00EFD64491D
:100C2000039804F00AFD6349039804F006FD284682
:100C300004B0BDE8F0815E49304623F064F9002835
:100C400043D07368002B32D154F8080F5A4EDFF8A6
:100C50008C8106F0D4FB594902680546204604F011
:100C6000ECFC10273368EB5800937368424604216C
:100C7000204604F0FFFC013F06F10806F2D16A6C41
:100C80004F49504EDFF85481204604F0D6FC10271F
:100C90003368EB580093736842460421204604F001
:100CA000E9FC013F06F10806F2D10025BFE74649FD
:100CB000301D23F028F908B90725B8E7B568002DDD
:100CC000FAD1A06806F09FFBB1E73A49304623F01D
:100CD0001AF900283FD0736883BB54F8080F3B4DC6
:100CE000DFF8FC8006F005FE092706462B686A68D7
:100CF000F35A4146204604F0A0FC013F05F10805E7
:100D0000F4D1334FDFF8DC8005257A684146204670
:100D100004F0D4FB57F8083B3344D3E900232046C2
:100D200004F018FC013DF0D120462A4904F0C6FB2E
:100D3000D6E90E23204604F00DFC78E72249301D49
:100D400023F0E1F80028B7D0B568002DB4D1A06831
:100D500006F0DDFD6BE71549304623F0D4F8002896
:100D6000AAD07368A3B954F8080F1B4DDFF86C8044
:100D700006F0B4FD042607462B686A68FB58414616
:100D8000204604F05AFC013E05F10805F4D18CE739
:100D90000D49301D23F0B7F800288DD0B568002D1F
:100DA0008AD1A06806F09EFD41E700BFA23C070083
:100DB0002F3707003337070084490700373707000C
:100DC0004C37070004490700775D07009C4807007F
:100DD000044A070070370700E4480700443707005B
:100DE000593707006037070008B5806806F0F2F948
:100DF000002008BD70B50E6804460D468EB954F843
:100E0000080F06F0F9F9054628B120460F4904F00D
:100E100014FC304670BD20460D4904F00EFC2846F7
:100E2000F8E70A49284623F06EF8064628B1012162
:100E3000A068BDE8704006F0D3B90549284623F004
:100E400062F808B13146F3E70720E3E7853707008A
:100E50008837070030B585B0044602A9806806F0DF
:100E6000E8FC0546F0B904F10800029A0F49019028
:100E700004F0E3FB9DF80C200D49019804F0DDFB24
:100E80009DF80D200B49019804F0D7FB9DF80E202A
:100E90000949019804F0D1FB9DF80F2007490198FA
:100EA00004F0CBFB284605B030BD00BF8D370700EE
:100EB0009F370700B4370700AD370700C537070075
:100EC000383003F0ABB800F5EA50103003F01EB92B
:100ED0000B6837B50546084683B9A86805F10804CC
:100EE00006F068FA10B1A86805F076F901462046C8
:100EF00004F0B4FB0024204603B030BD0DF107011F
:100F000004F032FC04460028F5D19DF807201AB9F8
:100F1000A868114606F047FA9DF80710A86806F081
:100F200050FA04460028E6D19DF80730002BE2D0A5
:100F30000249A8682A4606F036FADCE74920000094
:100F400070B5044680680E4610F096FD054606F022
:100F500043F985420CD00849304622F0D4FF48B10D
:100F600004F1080005492A4604F067FB002070BD23
:100F70000C20FCE70720FAE7593807001B3A070066
:100F800010B5044654F8080F06F06EFC03490246FB
:100F9000204604F052FB002010BD00BFCE3A0700EF
:100FA000024B034A083004F02FBC00BF69790000EF
:100FB0005F79000010B500F10804806806F075FC48
:100FC000044A0549002818BF1146204604F035FBA5
:100FD000002010BDDA370700DF37070070B50E6854
:100FE00004460D4666B954F8080F06F01BFC06F0DF
:100FF0001EFC18490246204604F01FFB304670BD17
:101000001549284622F07FFF20B1A068BDE8704056
:1010100006F0F9BB1149284622F075FF20B1A068FF
:10102000BDE8704006F0F4BB0D49284622F06BFF86
:1010300020B1A068BDE8704006F0E6BC094928462A
:1010400022F061FF20B1A068BDE8704006F0EEBC60
:101050000720D4E71B3A0700E5370700EE37070003
:10106000F4370700FB370700303002F0FDBC883052
:1010700003F0C8BB403004F053B9000038B50C6829
:10108000054608464CB906F0A7F80949024605F19D
:10109000080004F0D2FA002038BD064922F033FFE0
:1010A00018B105494FF4C972F1E72320F4E700BFF6
:1010B0001B3A070002380700364A070038B50C46CD
:1010C00005460949204622F01EFF58B164684CB914
:1010D00006F0B7F90549024605F1080004F0ADFA3B
:1010E000204638BD0720FCE706380700AC6907003A
:1010F00013B50C687CB908300849019004F0DEF99A
:101100000749019804F0DAF90198064904F095FAC4
:10111000204602B010BD2320FBE700BF0C380700BB
:101120000E380700956207002DE9F0410B68044670
:1011300094B008467BBB54F8080F1C4EDFF8808043
:1011400002AF394606F096F9BDF808201849204646
:1011500004F073FABDF80A201649204604F06DFA2F
:10116000BDF80C201449204604F067FA08253368BE
:10117000FA1820465168019152880092FB5A726811
:10118000414604F05AFA013D06F10806EFD100206D
:1011900014B0BDE8F081094922F0B5FE18B1A0688D
:1011A00006F06AF9F3E70720F2E700BFF44607000C
:1011B000133807001D38070026380700775D070041
:1011C0003338070010B5044608460A4922F09BFE52
:1011D00030B10022A0681146BDE8104006F09CBB6B
:1011E0000549A068224606F097FB002808BF242086
:1011F00010BD00BF41380700FD20000038B50D6864
:101200005DB9044654F8080F05F0D0FF04490246C2
:10121000204604F012FA284638BD0720FCE700BF3C
:101220009B37070038B50D685DB9044654F8080FC0
:1012300006F012FB04490246204604F0FEF9284657
:1012400038BD2320FCE700BF9B3707000B6837B58C
:1012500005460C469BB980680DF1060106F0E9F8D9
:10126000044648B9BDF806209DF806300D49120A1B
:1012700005F1080004F0E1F9204603B030BD08464E
:1012800022F03AFE02280BD12368A8681A78597810
:1012900001EB022189B203B0BDE8304006F0C4B8CA
:1012A0000724E9E747380700F8B50E460546124916
:1012B000304622F028FE074628B10121A868BDE883
:1012C000F84006F0E0BA0D49304622F01CFE044614
:1012D00008B13946F2E70A49304622F014FE48B117
:1012E00006F0E1FA0749024605F1080004F0A5F905
:1012F0002046F8BD2320FCE7596707004C3807005B
:1013000059380700364A070030B50D68044687B0E3
:1013100008466DB954F8080F1822694605F057FFC2
:101320000B496A46204604F088F9002007B030BD1A
:10133000084922F0E8FD48B154F8080F05F044FFD1
:1013400002460B46204604F005F9EEE70720EDE7DC
:101350001B3A07009D4E070037B50D686DB904466E
:10136000694654F8080F05F0DBFF2046082269465D
:1013700004F0D4F8284603B030BD0720FBE7096825
:10138000006868F031B9000038B505460C4641B92F
:101390000068904704490246284604F04EF920466A
:1013A00038BD0720FCE700BF1B3A070038B50C46E4
:1013B00005461249204622F0A6FD38B1104A616860
:1013C00005F10800BDE83840FFF7DEBF0D492046B3
:1013D00022F099FD08B10C4AF1E70C49204622F0B1
:1013E00092FD08B10A4AEAE70A49204622F08BFD3D
:1013F00008B1094AE3E7072038BD00BF2DA7070061
:101400002975000051380700317500005738070072
:1014100039750000613807004175000038B5054690
:101420000C4641B90068904704490246284604F03A
:1014300004F9204638BD0720FCE700BF364A070004
:101440002DE9F0430D6895B004460E468DBB8068CB
:10145000DFF8908006F074FAA9460646AFB2BE42A5
:1014600035D9A068ADF80E9008AA394606F0FCFA06
:10147000E8B99DF84930C3F3C0021B0717D4ADF893
:101480000E20A06804AB0DF10E02394606F0F1FA09
:1014900068B904F1080341461846BDF838200193A5
:1014A00004F00CF8019804A904F070F8E9E701359C
:1014B000D4E70A49304622F026FD60B1084A716837
:1014C00004F1080015B0BDE8F043FFF7A7BF002006
:1014D00015B0BDE8F0832320FAE700BFAA3C07005F
:1014E000557900006838070070B50C6886B005466D
:1014F0000E4664B955F8080F02A906F003FB28460A
:10150000102202A904F00AF8204606B070BD4B680C
:101510005BB9102202A9204622F0D4FC0028F4D1A5
:10152000A86802A906F0F3FAEFE70B49304622F06B
:10153000EAFC70B1A868746806F01CF90190A8680C
:1015400006F0A6F80199024602AB204605F0CCFD54
:10155000E4E70720D9E700BF6F38070073B50C68D0
:1015600005460E463CB10DF10701204622F091FCE4
:1015700060B102B070BD55F8080F06F0E2FA0849F4
:101580000246284604F059F82046F2E773682BB962
:101590009DF90710A86806F0D9FAEAE70720E8E7FE
:1015A000AC690700F0B5044600F10805134B144A76
:1015B000144F154E8DB00221284604F095F8A0680E
:1015C00006F029FB0446B4B120463022694605F0F6
:1015D00069FE6A463946284603F070FF04F112009E
:1015E0003022694605F05EFE6A463146284604F020
:1015F00024F8246BE7E720460DB0F0BD70470700E4
:1016000068470700723807007B38070030B50C6860
:1016100085B0054664B955F8080F694606F077F8B5
:1016200028461022694603F079FF204605B030BDF8
:1016300010226946204622F045FC0028F6D1A86811
:10164000694606F069F8F1E730B50C4687B0054603
:101650002149204622F057FCA0B1201D0DF11701B1
:1016600004F082F8044638B99DF817303BB11B49A5
:101670002A46A86806F06FFA204607B030BD024639
:101680000146F6E7206820B30DF1170122F0BAFBFE
:1016900004460028F0D19DF817001F2817D8012113
:1016A00081400F4B01930023A868029500934FF6E9
:1016B000FF7206F0FFF804460028DDD1094B0A4A04
:1016C000072105F1080004F00FF82424D4E70724CB
:1016D000D2E70146E5E700BF85380700892300000F
:1016E0002D240000284807000C4807002DE9F74387
:1016F0000D680446002D37D100F10806284B294A11
:10170000294FDFF8AC80DFF8B0900321304603F0BA
:10171000EBFFA068E9B206F025FA00B3A90289B28E
:101720000DF10303A068ADF804100DF1060206F0F8
:1017300020FA39462A46304603F0C0FEBDF806209E
:101740004FF6FE739A421BBF9DF803301749184AA3
:10175000920A04BF43464946304603F06EFF013506
:101760003F2DD6D1002517E0284601A922F05BFBCA
:10177000054688B954F8080FBDF804100DF10303AD
:101780000DF1060206F0F5F99DF80330BDF80620CC
:101790000849204603F051FF284603B0BDE8F08316
:1017A0006447070058470700913807009A38070038
:1017B0001FA80700B2380700A63807007FB50C46FF
:1017C00000232349ADF80E300546204622F09BFB4E
:1017D000064610B1606800BB0434206838B30DF1D0
:1017E0000D0122F00FFB00BB9DF80D001F281BD838
:1017F0000124844005F10800DEB1164B164A02218F
:1018000003F072FF154BBDF80E20A8680095214625
:1018100005F005FE48B9242007E00DF10E0122F085
:1018200002FB10B90834D8E7072004B070BD0446A5
:10183000E0E70B4B0B4A052103F056FF0A4BBDF8BE
:101840000E20A8680095214605F0E4FDE2E700BF00
:10185000C138070055470700484707002521000009
:1018600050470700344707002D24000037B50C68A7
:10187000054674B955F8080F05F08AFC0E494FF477
:101880007A72B0FBF2F2284603F0D7FE204603B08E
:1018900030BD4B686BB901A9204622F063FB0028DC
:1018A000F5D1019BA8684FF47A71594305F075FC96
:1018B000EDE70720EBE700BF9B37070037B505468C
:1018C00008680DF1070170B9A86804F0F1FC04463E
:1018D00030B99DF907200A4905F1080003F0ADFE73
:1018E000204603B030BD22F0D4FA04460028F7D1D8
:1018F0009DF90710A86804F0EFFC0446F0E700BF6C
:10190000D13807000B6837B505460C4683B98068A7
:101910000DF1070104F0F8FC044630B99DF90720E9
:10192000144905F1080003F088FE204603B030BDDD
:101930001149204622F0E7FAC8B160680DF10701AD
:1019400048B9A86804F0E0FC04460028EDD19DF9F0
:1019500007200A49E5E722F09CFA04460028E4D172
:101960009DF90710A86804F0D9FC0446DDE70724B8
:10197000DBE700BFC8380700D8380700AC690700AC
:1019800037B5054608680DF1070170B9A86804F07D
:1019900085FC044630B99DF907200A4905F1080085
:1019A00003F04BFE204603B030BD22F072FA04462D
:1019B0000028F7D19DF90710A86804F045FF0446F8
:1019C000F0E700BFD1380700F0B50B6885B00546D9
:1019D0000E4663B955F8080F05F027FC0446002CA5
:1019E00052D02146284603F0D1FD2469F7E7284963
:1019F000304622F088FA50B17068694622F058FAF1
:101A000018B9A868694605F015FC05B0F0BD214974
:101A1000304622F078FA50B17068694622F048FAF0
:101A20000028F2D1A868694605F009FCEDE71A49DB
:101A3000304622F068FA074648B1184B184A311D63
:101A400005F1080005B0BDE8F04003F0CBBE154934
:101A5000304622F058FA044648B155F8080F05F010
:101A600081FE0146284603F091FD3846CDE70E4938
:101A7000304622F048FA48B155F8080F05F076FED6
:101A80000146284603F082FD2046BEE72320BCE73E
:101A9000E038070053380700E438070053720000AD
:101AA00049720000F0380700F638070073B50C687B
:101AB00005460E4634B101A9204622F053FA60B122
:101AC00002B070BD55F8080F05F04FFC07490246FB
:101AD000284603F0B2FD2046F2E7736823B9019966
:101AE000A86805F047FCEBE70720E9E79B3707000C
:101AF00037B50C6805465CB955F8080F05F0C8FD08
:101B000008220146284603F009FD204603B030BDF7
:101B100008226946204622F0D5F90028F6D1A868A7
:101B2000694605F0B9FDF1E737B50C6805465CB9C3
:101B300055F8080F05F0DBFB08220146284603F0A4
:101B4000EDFC204603B030BD08226946204622F055
:101B5000B9F90028F6D1A868694605F0CCFBF1E791
:101B600030B50B68044687B0084683BBA06801A95E
:101B700005F07FFE054638BB08341B49204603F0BC
:101B80009DFC082201A9204603F0C8FCBDF80C20EA
:101B90001649204603F051FD9DF8112014492046B6
:101BA00003F04BFD9DF812201249204603F045FD3D
:101BB0009DF813201049204603F03FFD9DF81520A5
:101BC0000E49204603F039FD284607B030BD0C49C8
:101BD00022F099F928B1A06807B0BDE8304005F0BF
:101BE0004DBE0725F0E700BFFC38070007390700A6
:101BF000103907002439070039390700B9370700C1
:101C000042390700024B186800B9FEE7704700BF71
:101C1000580E0020037813F0010F0B461CBF7222F0
:101C200003F8012B0278920744BF642203F8012BCA
:101C30000278520744BF6E2203F8012B8B4204BF87
:101C40002D2203F8012B00221A700846704700006D
:101C50007FB50C68002305460E468DF804308CB91C
:101C600055F8080F05F032FD03A98DF8080002A809
:101C7000FFF7D0FF1E490246284603F0DEFC20464F
:101C800004B070BD1B49304622F03DF938BB3368C3
:101C90000146013B044613F8012F5AB16E2A05D0C4
:101CA000722A05D0642A20D10124F4E70121F2E749
:101CB0000120F0E728B19DF8043043F001038DF8CE
:101CC00004302CB19DF8043043F002038DF8043049
:101CD00029B19DF8043043F004038DF804309DF8D9
:101CE0000410A86805F002FDCAE70720C8E700BF96
:101CF0001B3A07001FA80700F0B50446A1B00D4627
:101D00000026227DF3B29A421BD92269284652F856
:101D10003310DF0022F0F7F801360028F1D06946D1
:101D2000284622F0F9F82369A4693B4428465E68F6
:101D300022F0FDF80138C1B201AA2046B04721B017
:101D4000F0BD2320FBE770B5064600680C4608B9D5
:101D5000072070BD2F2167F0D3FB054688B104F141
:101D60000801013022F04EF80028F2D1227A013A1F
:101D70003F2AEDD8287030682146BDE8704021F038
:101D8000EFBF1720E5E70000013002289ABF024BA1
:101D900053F82000014870471C430700F9A10700D1
:101DA0002DE9F341804608680F4616461D46C0B12E
:101DB000114622F07DF800232B70044668B1386884
:101DC00001A922F07AF840B9324601A9404605F04F
:101DD0005BFB044608B901232B70204602B0BDE826
:101DE000F0810724F9E7000038B50C4600F108053A
:101DF000284603F0B9FB228A1D49284603F05EFB02
:101E0000A37C1C49032B96BF1B4A1C4A52F8232073
:101E1000284603F053FBE27C194902F001022846F0
:101E200003F04CFBA37CE3B9E37C5B0714D51549B5
:101E30006269284603F042FB04F11801284603F0CA
:101E400093FBA37C032B07D1E37C628D0E49C3F384
:101E50004003284603F032FB2846BDE8384003F033
:101E60003BBB228D0949284603F028FBE9E700BF68
:101E7000CD3A07001A3A0700A44607006A5F070038
:101E8000523907005F3907007F39070073390700AF
:101E900010B500238EB0CDE901330446A06801AA35
:101EA00003A905F02AFE20B903A92046FFF79CFFED
:101EB000F4E700200EB010BD03289ABF024B53F880
:101EC00020000248704700BFB44607006A5F070061
:101ED000F0B50E4689B041490546304622F013F868
:101EE000074600B10436336813BB55F8080F3C4E63
:101EF00005F087F90446002C51D02146284603F00E
:101F000033FB87B1607CFFF7D7FFA17C237CC1F353
:101F100040010191A17C01F0010102460091284697
:101F2000314603F0CBFA284603F0D6FA6469E2E7BB
:101F30002C49304621F0E7FF90B1706802A921F0EA
:101F4000B7FF58B9069BA8689B0C9B0443F4403329
:101F500043F4507302A9069305F05DF909B0F0BD92
:101F60002149304621F0CFFF044650B1706802A9E4
:101F700021F09EFF0028F1D1A86802A905F050F9D0
:101F8000ECE71A49304621F0BEFF074648B155F844
:101F9000080F05F0E3FB0146284603F0F7FA204658
:101FA000DCE71349304621F0AEFF044648B155F84E
:101FB000080F05F0CBFB0146284603F0E7FA384648
:101FC000CCE70C49304621F09EFF20B155F8080FB0
:101FD00005F0C0FBDFE72320C0E700BF9A39070008
:101FE0009D390700E038070053380700C63907005D
:101FF000D0390700D539070030B597B00B6800938A
:102000008B88ADF804300D490D4B0E4D002A08BFEA
:102010000B4600F10804029320460023ADF8563029
:1020200003F05AFA684605F011FA28B903AA2946BE
:10203000204603F002FBF5E717B030BDDE3907009C
:10204000DB3907001B3A070013460A4601461846CB
:10205000FFF7D2BF024A0349083003F02FBA00BF8E
:10206000284307001B3A0700437F37B5044673B186
:1020700081B30846019105F095F8019A1649034687
:1020800004F1080003B0BDE8304003F0D6BA037F86
:1020900003B9FEE724291DD000F1080579B90F49DD
:1020A000284603F0CAFA002304F12000237706F043
:1020B00027FF204603B0BDE83040FFF7CBBF0846FE
:1020C000019105F06FF8019A03490346284603F091
:1020D000B4FAE8E703B030BDE1390700EE39070094
:1020E00010B505490446083003F0A7FA2046002140
:1020F000BDE81040FFF7B8BFF3390700FFF7F0BFA6
:1021000010B419B95DF8044BFFF7AEBF91F9013077
:102110000A785DF8044B0249083003F08EBA00BF1C
:10212000063A07000B4601461846FFF7E9BF0000D4
:1021300070B504460D4611461A4603F06FF9234662
:102140000026164AA683C4E9025443F8202F2946E4
:10215000C4E90A342246C4E90C5404F1380001F001
:1021600039FD2246294604F1400003F005F82246D5
:102170002946C4E9205404F1880002F028FB04F544
:10218000EA5022462946103001F08EFF2046266193
:102190006661A661FFF75EFF204670BDC7210000A3
:1021A00010B5054C13460A4601462046FFF7C0FF0E
:1021B000024B1C6010BD00BF600E0020580E0020B6
:1021C0000021FFF751BFC068FFF7FABF2DE9FF41BB
:1021D0000B680393234B00930C2305460E464A22BB
:1021E00021490DEB030005F0E4FD044668B1826867
:1021F0006368511005EB6200D20744BF6A58D35898
:10220000311D04B0BDE8F04118471849304621F0AF
:102210007AFEE0B1DFF85080154F05F1080658F856
:10222000242039463046033403F007FADE2CF6D179
:102230000F4F00242A7DE3B29A420FD92A6939460A
:1022400052F83320304603F0F8F90134F2E7314612
:10225000284604B0BDE8F041FFF74EBD002004B0B1
:10226000BDE8F0817F1300002C430700143A0700FB
:102270001B3A070030B50446A3B00D4601B9FEE78E
:10228000437F5BB1202201A9284621F015FDA0B1B2
:1022900001462046FFF7E8FE23B030BD037F002B48
:1022A000FAD1012303774FF4C071284606F0A1FC50
:1022B000B0F5C07FE6D30620EAE7019B23B9237778
:1022C0002046FFF7C7FEE7E701A92046FFF77EFF9C
:1022D0000028DDD1019B002BDAD1237F002BEFD02A
:1022E000DAE70000F0B501230F4E104F437789B0B5
:1022F0000446142556F8041B1D22684668F08EFC1F
:1023000000236A46394604F108008DF81D3003F0B9
:1023100094F969462046FFF7ADFF013DEAD1284612
:10232000657709B0F0BD00BFBC470700193A070048
:10233000FFF736BF07B50190FFF764FC019903B0C2
:102340005DF804EBFFF796BF082203F0D5B8000054
:1023500013B50C4608300A49019003F0AFF8019814
:102360002146FFF7F1FF227A06490198C2F30013D4
:1023700002F00F0202B0BDE8104003F05EB900BFEA
:102380001E3A0700383A07000B4601461846FFF789
:10239000DFBF000038B504460D4619B9BDE8384026
:1023A000FFF762BE91F839309B0604F1080412D59C
:1023B00001F108022046164903F080F8154920462D
:1023C00003F07CF805F119012046FFF7BDFF124923
:1023D000204603F073F86A8E1049204603F06EF829
:1023E00029462046FFF7B0FF95F836200C492046D5
:1023F00003F064F895F937200A49204603F05EF8A7
:1024000095F8382008492046BDE8384003F015B952
:102410004F3A07009738070074A50700583A07009D
:10242000623A07006A3A0700713A07000B46014614
:102430001846FFF7AFBF00002DE9F04F0C468FB0F4
:1024400085490546204621F05EFD064600287ED1DE
:102450008249204621F057FD00287FD120680DF1E8
:10246000020121F0E0FC064600286CD1BDF8021004
:10247000A86802AA05F0F3FA0646002863D10835D9
:10248000BDF822207649284603F0D7F8BDF8202071
:102490007449284603F0D1F82846734903F00EF832
:1024A00008220DEB0201284603F038F89DF8312090
:1024B0009DF80030C2F3000161F30003C2F3400253
:1024C00062F3410362F3820301A968468DF800308C
:1024D000FFF7A0FB65490246284603F0AEF89DF8D9
:1024E000312063492846C2F3001203F0A6F89DF894
:1024F00024206049284603F0A0F8049A5E49284643
:1025000003F09BF8059A5D49284603F096F89DF87C
:1025100025205B49284603F090F89DF9262059496B
:10252000284603F08AF8BDF82E205749284603F0C4
:1025300084F808E04946204602F0C0FF8AE02046C1
:1025400002F0CAFF002630460FB0BDE8F08F4F4BB7
:102550004F4A0E2105F1080003F0C6F8A868DFF81D
:102560005491DFF854A1DFF854B105F0E9F90027E0
:102570008046B9B2414505F10804E0D2A86802AA34
:1025800005F072FA002865D19DF831301B0761D43F
:10259000BDF82220002ECDD05146204602F08EFFFD
:1025A000BDF820205946204602F088FF049A394998
:1025B000204602F083FF059A3649204602F07EFF4E
:1025C0009DF825203449204602F078FF9DF824200C
:1025D0003249204602F072FF9DF83120304902F066
:1025E0000102204602F06AFF9DF831202C49C2F317
:1025F0004002204602F062FF9DF831202849C2F3D4
:102600008002204602F05AFF9DF8302025492046DE
:1026100002F054FF9DF831202349C2F300122046F6
:1026200002F04CFFBDF82C201B49204602F046FF6B
:10263000BDF82E201849204602F040FF1B492046D5
:1026400002F03CFF02A92046FFF77EFE1849204613
:1026500002F0F3FF01378CE7453F0700793A0700A6
:10266000BB3A0700C83A0700FC380700D33A070016
:10267000DC3A0700F23A0700FF3A07003939070051
:10268000103907000C3B0700153B0700AC4707005B
:10269000744707008F3A0700983A07009F3A0700EF
:1026A000A63A0700AB3A0700B03A07009738070090
:1026B000113A0700B73A07007E3A0700853A07004B
:1026C0002DE9F0430C4693B000239249ADF8063053
:1026D0000546204621F017FC0646002840F00D81F3
:1026E0008D49204621F00FFC002840F00D818B49D8
:1026F000204621F008FC0646002840F0A9808849C1
:10270000204621F000FC0746002800F0F4808249B2
:10271000201D21F0F8FB38B9824B834A042105F1D2
:10272000080002F0E1FF3E46DFF848827F4FDFF805
:102730004892A86808AA0DF1060105F06EF8002875
:1027400040F08280BDF8302005F10804002E00F032
:10275000C3804946204602F0B1FE08A92046FFF793
:10276000F3FD0A9802A9152205F0DBF802AA20461B
:102770006F4902F0A3FE0B9802A9152205F0D1F8CB
:102780006C4902AA204602F058FFD2E7BDF830207B
:102790004946204602F092FE2C4608AA54F8080F3B
:1027A0000DF1060105F039F800284AD1002EEDD0D0
:1027B0009DF8463013F0080F14BF432252224146C1
:1027C000204602F07BFEBDF830203946204602F05C
:1027D00075FE0A9A5849204602F070FE9DF93D2088
:1027E0005649204602F06AFE9DF93E205449204693
:1027F00002F064FE9DF846205249204602F0010294
:1028000002F05CFE9DF846204E492046C2F340028D
:1028100002F054FE9DF846204A49C2F38002204649
:1028200002F04CFE2046484902F048FE08A9204626
:10283000FFF78AFDBDF844204449204602F0FDFE22
:10284000AAE7204602F048FE002013B0BDE8F0835E
:1028500005F108043E4B3F4ADFF81C813E4F3F4ED6
:102860000721204602F040FFA86808AA0DF10601E2
:1028700004F0D3FF0028E7D1BDF8302041462046C0
:1028800002F01CFE08A92046FFF75EFD02A9BDF874
:10289000400002F0F1FD39460246204602F00EFEED
:1028A00002A9BDF8420002F0E7FD3146024620468B
:1028B00002F004FE9DF93D202949204602F0FEFD6C
:1028C0009DF93E201D49204602F0F8FD0A9A25494F
:1028D000204602F0B2FEC7E74146204602F0EEFD78
:1028E00008A92046FFF730FDDDE90A2339462046D6
:1028F00002F0A3FE1DE70720A7E71B4B1B4A0A2196
:1029000005F1080002F0F0FEDFF86890DFF86C8057
:10291000174F41E7453F0700793A07002E3B070074
:10292000923B07008448070030480700AD3B070092
:102930009B3B0700A33B0700423B07004A3B0700C5
:10294000513B0700A63A070097380700583B07009D
:1029500092480700684807006D3B0700783B070076
:10296000823B0700893B0700884807004048070072
:10297000853A0700873A0700613B07003A3B0700AA
:102980002DE9F04F0C4689B06E490546204621F0EE
:10299000BAFA074600286ED16B49204621F0B3FAF7
:1029A00000286FD120680DF10A0121F03CFA06469B
:1029B000002840F0C280BDF80A10A86803AA05F0FC
:1029C00097F80646002840F0B8809DF81C205F4923
:1029D000083502F00102284602F02FFE9DF81C3057
:1029E000DA0740F1AA809DF816205949284602F0DE
:1029F00024FEBDF814205749284602F01EFE9DF81B
:102A0000172055499202284602F017FE9DF81C2017
:102A10005249C2F34002284602F00FFE9DF81C30D6
:102A20009B0740F18A8028464D4902F047FD03A9E3
:102A30002846082202F072FD9DF8182049492846D0
:102A400002F0FBFD9DF819204749284602F0F5FDEC
:102A50009DF81A204549284602F0EFFD9DF81B20FD
:102A60004349284602F0E9FD67E01A4649462046F8
:102A700002F024FD59E03F4B3F4A092105F10800CF
:102A800002F032FEA868DFF81091DFF810A1DFF83D
:102A900010B105F02BF8002680462C46F3B254F80E
:102AA000080F019303AA194605F022F800283CD12B
:102AB000019B002FD9D09DF816205146204602F0E8
:102AC000FDFCBDF814205946204602F0F7FC9DF8A5
:102AD00017202A49204602F0F1FC9DF818202849C9
:102AE000204602F0EBFC9DF819202649204602F012
:102AF000E5FC9DF81A202449204602F0DFFC9DF8F1
:102B00001B202249204602F0D9FC2149204602F030
:102B1000D5FC03A92046FFF717FC9DF81C201D4992
:102B2000C2F34002204602F088FD0136F3B243456D
:102B3000B3D9204602F0D0FC0026304609B0BDE8EB
:102B4000F08F00BF453F0700793A0700D93B0700E7
:102B5000CC370700C83A0700E33B0700F23B070009
:102B6000FC380700FB3B0700103907002439070039
:102B7000043C0700E8460700C4460700C43B0700C2
:102B8000CB3B0700983A0700D23B07007E3A07008C
:102B9000973807000B3A0700B73A0700633A070077
:102BA000853A070070B50C46096806461D46FEF7D3
:102BB000EBFB48B1216831B1636823B930682B461B
:102BC000BDE870401847072070BD000008B5034AF3
:102BD000034B0830FFF7E6FF08BD00BFBD770000DC
:102BE000C577000008B5034A034B0830FFF7DAFF4A
:102BF00008BD00BF757700007D770000F7B50C6851
:102C000005460E461F464CB120460DF1060121F047
:102C10000AF9044650B1204603B0F0BD0068904761
:102C200007490246284602F008FDF4E7736823B915
:102C3000BDF806102868B847EDE70724EBE700BFAA
:102C4000364A0700F8B50E4605461A49304621F0C7
:102C50005AF938B1184B194A311D05F10800FFF730
:102C6000CDFFF8BD1649304621F04DF9044610B1AC
:102C7000144B154AF0E71549304621F044F908B9DC
:102C80000720EEE7776857B955F8080F04F0FBF90D
:102C90000F490246284602F0D0FC3846E1E70D49CC
:102CA000301D21F030F90028EAD0A86804F0EFF9CF
:102CB0002046D6E70C3C07007F70000077700000CC
:102CC000193C07006F70000067700000223C07008D
:102CD000364A0700775D0700F7B50C6805460E46D3
:102CE0001F4644B1204601A921F03CF9044650B1E9
:102CF000204603B0F0BD00689047074902462846C9
:102D000002F09BFCF4E773681BB901992868B84787
:102D1000EEE70724ECE700BF9B37070008B5034A3E
:102D2000034B0830FFF7D8FF08BD00BF7D760000D9
:102D30008776000008B5034A034B0830FFF7CCFF45
:102D400008BD00BFA7790000B179000038B50C4676
:102D500005460E49204621F0D6F838B10C4B0D4AF5
:102D6000211D05F10800FFF7B7FF38BD0A492046CD
:102D700021F0C9F838B1094B094A211D05F10800B5
:102D8000FFF73CFFF1E70720EFE700BF263C070015
:102D9000E7770000DD7700002E3C0700FD7700009C
:102DA000F3770000F7B50D46096807461E46FEF7A3
:102DB00035FB044660B128680DF1070121F022F8C7
:102DC000044628B96B6833B99DF807103868B047D6
:102DD000204603B0F0BD0724FAE7000008B5034A17
:102DE000034B0830FFF7DEFF08BD00BF7D79000010
:102DF0008779000008B5034A034B0830FFF7D2FF7C
:102E000008BD00BFBB790000C579000008B5034AC2
:102E1000034B0830FFF7C6FF08BD00BF377A00003C
:102E2000417A000008B5034A034B0830FFF7BAFFA8
:102E300008BD00BF4B7A0000557A000008B5034A70
:102E4000034B0830FFF7AEFF08BD00BFCF7900008D
:102E5000D979000070B50C4605461049204621F08E
:102E600052F8B0B1261D0E49304621F04CF840B161
:102E70000C4B0D4A04F1080105F10800FFF792FF21
:102E800070BD0A49304621F03EF820B1084B094A8E
:102E9000F0E72320F4E70720F2E700BF383C070003
:102EA000423C0700897300007F730000403C07002C
:102EB0009D7300009373000073B50C4606460DF138
:102EC00006012068154620F0AEFF28B963682BB9CB
:102ED000BDF806103068A84702B070BD0720FBE7B8
:102EE00038B50C6800F108054CB9806804F01EFA8A
:102EF00005490246284602F0A0FB204638BD034A99
:102F00002846FFF7D9FFF9E7493C0700377300006F
:102F1000F7B50E4605462149304620F0F4FF38B19A
:102F20001F4A311D05F10800FFF7C6FF03B0F0BDD1
:102F30001C49304620F0E7FF074668B104361A49BD
:102F4000304620F0E0FF20B1A86804F095F9002099
:102F5000ECE7164A3146E5E71549304620F0D3FF45
:102F6000D0B155F8080F0DF1070104F08BF90646B2
:102F700070B13C460F4F9DF80720E3B29A4207D943
:102F800036F813203946284602F098FA0134F2E761
:102F9000284602F0A1FADAE72320C7E7E038070065
:102FA0005D720000503C0700573C07006B72000048
:102FB0005B3C0700B73A070070B50C68164605463B
:102FC0001A4614B1FFF778FF70BD0068B047034997
:102FD0000246284602F031FB2046F5E7364A070054
:102FE00008B5034A034B0830FFF7E6FF08BD00BFF2
:102FF000417900004B79000008B5034A034B0830C3
:10300000FFF7DAFF08BD00BF917900009979000051
:1030100073B50C4606460DF107012068154620F0F1
:10302000F1FE28B963682BB99DF807103068A847EE
:1030300002B070BD0720FBE7F8B50D460646134900
:10304000284620F060FF06F1080748B1B0680EF08E
:103050000BFD02460E49384602F0EFFA0020F8BD9B
:103060000C49284620F04FFF18B1B0680EF000FD63
:10307000EFE7094A29683846FEF7D0F90028EED074
:10308000064A29463846FFF7C3FFE8E75F3C0700DA
:10309000693C07006F3C0700AD720000B77200008A
:1030A00008B5024A0830FFF7B3FF08BD7379000086
:1030B00008B5024A0830FFF7ABFF08BDF7790000FA
:1030C00038B500F108040D46054A09682046FEF7A8
:1030D000A5F920B1034A29462046FFF799FF38BDDC
:1030E000E3790000ED79000038B50C4605460A7A10
:1030F000074902F0A2FA62880649284602F09DFAC2
:10310000626805492846BDE8384002F096BA00BF1B
:103110002C4A0700394A07004B4A07001FB50B68C5
:103120000446E3B90F4902F0C9F9206801A903F088
:1031300095FF78B9204602F0CFF90B49BDF804207D
:10314000204602F07AFA01A92046FFF7CDFF0020C1
:1031500004B010BD0549204602F06FFAF7E72320BE
:10316000F6E700BF5E4A07006B4A07007C4A07008B
:10317000D1E9002302F0EEB9D1E9042302F0EAB963
:10318000B1F85A20014902F058BA00BF364A070088
:1031900001F13002014902F050BA00BF1B3A0700AA
:1031A000B1F85820014902F048BA00BF493C070075
:1031B0000A6F014902F041BA824A07004A6D01498B
:1031C00002F03BBA9B3707000822413102F0A6B952
:1031D0001022203102F0A2B9493102F009BA0B687D
:1031E000186830B104330B60014602F1300003F07F
:1031F0007DBF07207047000008B5FF22002102486C
:1032000065F0DEFB002008BDC02B002010B50C6867
:1032100034B9044991F8FE2002F080F9204610BD2F
:103220000720FCE7C02B002038B50D4604460C49AA
:10323000284620F068FE28B120680A49BDE83840D9
:1032400003F02FBF0849284620F05DFE28B1206812
:103250000449BDE8384003F02EBF072038BD00BF49
:103260008A4A0700C02B00204469070009680068EB
:1032700066F0BAB90968006866F0B6B90B6810461E
:103280001A1D0A6000F141010822186820F01ABED8
:103290000B6810B514461A1D0A60186804F1100175
:1032A00020F05EFD08B92083A07610BD0B68181DC4
:1032B0000860186802F1540120F054BE10225C31FD
:1032C00002F02CB92DE9F0410D4607461B4928684C
:1032D000144620F018FE2B681A1D2A6020B3D3F87C
:1032E0000480B8F1000F27D094F8773093B104F13F
:1032F000300694F8783093B104F1410204F15C0394
:103300003146404603F0F0FE10B92B6804332B60C1
:10331000BDE8F081386804F02DFA0646E9E7386820
:1033200004F0B6F90246E9E704F15C011868BDE86B
:10333000F041102220F0C6BD0720E9E76F380700F2
:103340000B68181D0860186802F1700120F00ABEB1
:103350000B6810B514461A1D0A601868214620F043
:10336000FFFC08B92081A07210BD30B50B6885B094
:1033700015461A1D0A601868694620F099FD044632
:1033800028B96B4603CBC5F84900C5F84D10204657
:1033900005B030BD0B6810461A1D0A6000F120010F
:1033A0001022186820F08EBD0B68181D0860186880
:1033B00002F15A0120F037BD0B68181D086018682B
:1033C00002F1580120F02FBD30B50C46A1B00546E2
:1033D0001F49204620F097FD30B11E49286821B0D2
:1033E000BDE8304003F058BE1B49204620F08BFD5D
:1033F00030B11849286821B0BDE8304003F056BE0E
:103400001649204620F07FFD50B12868694603F038
:10341000B9FE18B90F49684603F087FE21B030BDE8
:103420000F49204620F06FFD78B10A4D6068FE23F9
:103430002A466946ADF8003020F052FD0028EDD153
:10344000BDF8003085F8FE30E8E70720E6E700BF6A
:103450008A4A0700C02B002044690700914A0700F0
:10346000954A070070B50C46E2B00546174920465C
:1034700020F049FD18BB1649204620F044FD18B342
:103480000126FE236068ADF8063022AA0DF1060180
:1034900020F026FD78B9BDF806308DF8863102A9F6
:1034A00022A803F02AFE044628B9286822A946B9B2
:1034B00003F0F7FD00B10446204662B070BD00265F
:1034C000DFE703F0F8FDF5E70724F5E78A4A070090
:1034D0004469070070B51368A2B006460D46019214
:1034E000D3B91E4802A903F008FE044688B96B68E8
:1034F00088336B4413F80C3C5BB1EA68AB6851103D
:10350000D50706EB620048BF725802A948BFD358DE
:103510009847204622B070BD8022002102A865F0A5
:103520004FFA6A692B69511006EB6200D20748BF57
:10353000725801A948BFD35802AA984704460028E8
:10354000E7D16B68054988336B44012203F80C2CE2
:1035500002A803F0FEFD0446DBE700BFC02B0020FD
:1035600038B50C460A882249054601F0A7FFA37822
:10357000D80703D51F49284601F0A0FFA378990773
:1035800003D51D49284601F099FFA3785A0703D5B2
:103590001A49284601F092FFA3781B0703D5184962
:1035A000284601F08BFFA378D80603D51549284695
:1035B00001F084FFA378990603D51349284601F04A
:1035C0007DFFA3785A0603D51049284601F076FFFF
:1035D000E378DB0703D50E49284601F06FFFE27858
:1035E0000C492846C2F34202BDE8384002F025B833
:1035F000B73A0700863C0700983F07006864070059
:10360000EA4D0700B03F0700FF4D07007038070084
:103610007AAF0700354A07006C31FFF7A1BF000001
:1036200073B50023019313680E46186801A9154667
:1036300020F0F9FB044600287FD129684A680B1D59
:103640002B60002A77D0013A12F8013F002B5BD0A3
:10365000722B05D8622B05D8432B3FD0522B4CD070
:1036600007246AE0633B0F2BFAD801A050F823F03F
:10367000D336000061360000E736000061360000F6
:1036800061360000613600006136000061360000DE
:10369000613600006136000061360000BF36000070
:1036A000B1360000F136000061360000C936000076
:1036B0009DF8063043F001038DF80630C4E79DF80D
:1036C000063043F00203F7E79DF8063043F00403A9
:1036D000F2E79DF8063043F00803EDE79DF8063069
:1036E00043F01003E8E79DF8063043F02003E3E7DA
:1036F0009DF8063043F04003DEE79DF8073043F0C5
:1037000001038DF807309FE7886801F108032B60FB
:1037100088B10DF1030120F075FB88B92B689DF885
:1037200003200433072A2B609AD89DF8073062F3F0
:1037300043038DF8073001983060204602B070BD19
:103740000446FAE713460A4603F16C01FFF768BF27
:1037500007B5044B00930E22182304F02AFB03B094
:103760005DF804FB753200002DE9F047A2B0044675
:10377000084602A903F0C1FC064658BBDFF85CA06E
:10378000DFF85C80DFF85C900C27DAF804300193F6
:10379000414601A8FFF7DCFF436888336B440546C8
:1037A00013F80C3C93B1DAF800204946204601F0AA
:1037B00085FEEB685A1013F0010F18BFA25804EBF6
:1037C0006300AB6802A918BFD3589847013F0AF1BC
:1037D000080ADAD1304622B0BDE8F0878C4B0700EA
:1037E000584C07008462070070B5C0B005460E460D
:1037F0000068694603F050FC044630B933683BB9B1
:1038000069462846FFF7B0FF0446204640B070BD29
:103810000649304620F077FB30B19DF8FE2069461E
:10382000284601F07BFEF0E70724EEE73C3F070067
:1038300070B5C0B005460E460068694603F036FC18
:10384000044630B933683BB969462846FFF78CFF18
:103850000446204640B070BD0649304620F053FB78
:1038600030B19DF8FE206946284601F057FEF0E78A
:103870000724EEE73C3F07002DE9F047C4B00E46B1
:1038800004468022002104A865F09AF8334FDFF83F
:10389000D880331D02934FF00009029BD3F800A09B
:1038A000BAF1000F39D0394603A8CDF80CA0FFF7C4
:1038B0004FFF0546C8B14269029B511004EB6200FC
:1038C0000433D20748BF625802932B6902A948BF4C
:1038D000D35804AA984700283BD16B6803F5887336
:1038E0006B44012203F88C2CD7E70298414620F064
:1038F0000AFB002830D0029B1A1D02928022ADF8EC
:103900000C20586824AA03A920F0EAFA08BB029BFD
:103910009DF80C9004330293BFE71149304620F024
:10392000F2FA054668B90F49304620F0ECFA98B132
:10393000CDE9005520684B4624AA04A903F0CFFB2B
:1039400007E0CDE900AA20684B4624AA04A903F0A9
:10395000BCFB44B0BDE8F0870720FAE7584C0700ED
:103960008A4A0700446907003C3F07002DE9F04FF1
:10397000002493B0CDE90344DFF8E490DFF8E4A03D
:10398000059406460D4601F104082746D8F800B014
:10399000BBF1000F3AD02F49CDF808B002A8FFF7CD
:1039A000D7FE58B1426802F148030DEB0302012132
:1039B00002F83C1CC3460BF10408E7E749464046C1
:1039C00020F0A1FA70B12022ADF80820D8F8040048
:1039D0000AAA02A908F1040B20F082FA48B99DF85E
:1039E0000870E8E75146404620F08DFA044618B9C1
:1039F000072013B0BDE8F08FD8F8040006A908F13D
:103A0000040B20F055FA0028D5D0F2E712492846D9
:103A100020F079FA58B130680CB10DF1180BCDF8DF
:103A200000B03B460AAA03A903F04AFBE1E70B49B1
:103A3000284620F068FA0028DAD030680CB10DF181
:103A4000180BCDF800B03B460AAA03A903F042FBCD
:103A5000CFE700BF584C07008A4A070044690700B7
:103A60003C3F0700CDA60700F0B50B6885B00546C2
:103A70000C462BB9224905B0BDE8F040FFF774BEF3
:103A80002049204620F03FFA70B11F4F1F4E0024FE
:103A900057F8242031462846033401F0CEFD1B2C74
:103AA000F6D1002005B0F0BD23681949039303A89F
:103AB000FFF74EFE014630B1221D284605B0BDE895
:103AC000F040FFF707BD23680393124B00930C23CC
:103AD0000DEB03000C49092204F06BF9034668B1B1
:103AE00082685B68511005EB6200D20744BF6A58D8
:103AF000D358211D05B0BDE8F04018472320D1E779
:103B0000C02B0020143A0700EC4B07001B3A0700BB
:103B1000584C07006D32000038B50C6805464CB9AA
:103B2000006803F0CCFC04490246284601F085FDFC
:103B3000204638BD0720FCE7364A070038B50C6838
:103B4000054608464CB9286803F0BEFC0849024601
:103B5000284601F072FD002038BD064920F0D3F957
:103B600018B1286803F0B5FCF5E70720F4E700BFBB
:103B7000364A0700775D07000968006865F034BDC4
:103B800030B50C4687B005461149204620F0BBF9F8
:103B9000D8B102A9201DFEF7D6F8172807D10023B7
:103BA00060688DF810300822694620F08BF930B932
:103BB0009DF81030286823B102A903F0AFFC07B0CC
:103BC00030BD694603F0A5FCF9E70720F7E700BF21
:103BD000A84D0700C0E900127047437C5A0744BF54
:103BE000702301F8013B437C1B0744BF612301F8AC
:103BF000013B437CDA0644BF642301F8013B437C6C
:103C00009B0644BF632301F8013B437C5A0644BF33
:103C1000722301F8013B437CDB091CBF6F2301F8D1
:103C2000013B837CDB0744BF732301F8013B837CAA
:103C30009A0744BF6E2301F8013B837C5B0744BFB6
:103C4000442301F8013B00230B70704730B50C464C
:103C500087B0054601F0A4FC01A92046FFF7BDFF8F
:103C60009DF8043023B1094901AA284601F026FC39
:103C7000607C40F3010040B2FEF786F8A38A044955
:103C80000246284601F0D9FC07B030BD1A3A0700B9
:103C9000AE4D0700037D1B0744BF732301F8013BB2
:103CA000037D5A0744BF6E2301F8013B037D9B0649
:103CB00044BF612301F8013B00230B7070470000F3
:103CC00030B50C4687B0054601F06AFC01A92046D4
:103CD000FFF7E0FF9DF8043023B1094901AA284607
:103CE00001F0ECFB207D40F3010040B2FEF74CF800
:103CF000638A04490246284601F09FFC07B030BDA4
:103D00001A3A0700AE4D070038B50C4605464A681A
:103D1000114901F0D3FB227A04F10901284601F090
:103D2000EBFB0E49284601F0C9FB94F8072104F586
:103D30008471284601F0E0FB94F80631DB0703D5D7
:103D40000749284601F0BAFBB4F800220549284685
:103D5000BDE8384001F071BCB74D070074A50700FD
:103D6000BC4D0700CD3A070013B9006803F0B8BB9B
:103D70001720704713B9006803F0B7BB17207047CE
:103D800013B9006803F0B6BB17207047F0B5ADF566
:103D90001B7D00230E46624900930446154601F040
:103DA0004CFC4FF6FF77334606AA69462046FFF7DC
:103DB000DBFF50B9BD4203D0BDF82C30AB42F2D18D
:103DC00006A92046FFF742FFEDE75649204601F0DD
:103DD00034FC002300934FF6FF7733460CAA694664
:103DE0002046FFF7C7FF50B9BD4203D0BDF84230AF
:103DF000AB42F2D10CA92046FFF762FFEDE74A493A
:103E0000204601F01AFC002300934FF6FF7733465B
:103E100019AA69462046FFF7B3FF50B9BD4203D047
:103E2000BDF86432AB42F2D119A92046FFF76CFF0E
:103E3000EDE7002E5DD14FF6FF739D4259D13B490E
:103E40003B4D204601F0F9FB0096206801AA694627
:103E500003F055FB88B90DF10601204601F0A0FBE7
:103E60009DF805309DF80420002B14BF63232D23FB
:103E70002946204601F0E1FBE7E7206812A903F09C
:103E800043FB2C49204601F0D8FB9DF860309D078C
:103E900032D5BDF84A202849204601F00FFB9DF895
:103EA0006030D8072DD5BDF848202449204601F0C0
:103EB00005FB9DF86030190728D5BDF85E201E4926
:103EC000204601F0FBFA9DF860305A0723D59DF893
:103ED0004C200DF14D01204601F00EFB9DF86030A5
:103EE000DB0603D51649204601F0E8FA204601F02A
:103EF000F3FA0DF51B7DF0BD1249204601F0DEFA04
:103F0000CDE71049204601F0D9FAD2E70D49204605
:103F100001F0D4FAD7E70C49204601F0CFFADDE7EB
:103F2000BF4D0700C94D0700D14D0700DB4D07000D
:103F3000E54D0700EC4D0700B73A0700893A070046
:103F4000FE4D0700FB4D07001FA8070030B5C3B0AA
:103F5000FF2305468DF8073081B900680DF107038E
:103F600002AA03F0A7FA044628B99DF8072002A97F
:103F7000284601F0D3FA204643B030BD0C24FAE7BE
:103F80002DE9F04F85B000244FF6FF73DFF88480F1
:103F9000DFF88490ADF80E3006460D462746A2465F
:103FA0005FFA84FB05EB8B0355F82B20D2B1184642
:103FB000414601931FF0A7FF019B70B9494618467F
:103FC0001FF0A1FF60B955F82B000DF10E011FF095
:103FD0002AFF18B105B0BDE8F08F82460134DFE753
:103FE0000746FBE7BDF80E20BAF1000F00D14FB134
:103FF0004FF6FF739A420BD127B151463046FFF777
:10400000A5FFE7E730465146FFF7C0FE0020E1E795
:104010000720DFE7CA3907003C3F07002DE9FF41D1
:104020000B6805460C4693B9DFF878801A4F0026D6
:1040300058F8262039462846033601F0FEFA0C2EA1
:10404000F6D123682BBB232004B0BDE8F0811349CF
:1040500020461FF058FF0028E6D123680393104B39
:1040600000930C230DEB03000E49042203F0A1FE84
:1040700003460028E7D082685B68511005EB6200B8
:10408000D20744BF6A58D358211D04B0BDE8F0419F
:1040900018470020D8E700BF1B3A0700143A070072
:1040A000793B0000184E0700C0E90012027A6FF356
:1040B0000002027270470968002330B513600139AD
:1040C0004FF47A730A2511F8010FF0B1A0F1300412
:1040D000092C12D8B3F57A7F02BF106868431060CC
:1040E0000878A0F130041068B3F57A7F03FB040070
:1040F0001060E8D0B3FBF5F3E5E72E2804D1B3F563
:104100007A7F01D16423DEE7072030BD70B50E460B
:1041100092B004464E4930461FF0F5FE28B12068A3
:1041200003F017FA002012B070BD4A4930461FF064
:10413000EAFE054600B1043600213C2203A864F0E3
:104140003FFC454930461FF0DEFE68B1706803A9A8
:104150001FF0AEFE0028E6D1206803A903F056F850
:1041600008B90720DFE708363C4930461FF0CBFE90
:1041700018B101238DF84430043620680DF107038F
:1041800007AA3146FDF70CFE0028CCD19DF8073078
:104190003BB13349204601F091F907A9204601F0CF
:1041A000F5F9706800282ED1B068002831D1F36885
:1041B000002B35D1306900283BD173696BB102AA5D
:1041C00006F114012046FFF776FF0028ABD1029BD1
:1041D000B3F5803FC5D2ADF84030B369002BC0D1F4
:1041E000204B0B93204B206803A9CDE90C3403F03E
:1041F000ABF9002897D1237A002D65F300032372D1
:1042000008BF24208FE70EA91FF00DFE0028CBD099
:1042100089E70DF13A011FF006FE0028C7D082E7BA
:104220000FAA06F10C012046FFF745FF0028C1D078
:1042300079E70DF142011FF0E5FD00287FF473AF2F
:104240009DF84230B3FA83F35B098DF84330B4E74D
:104250004C38070041380700484E07004B4E070016
:104260004E4E0700A54200005143000037B54A8A70
:1042700008320C46054692B2084901F01FF9214662
:10428000284601F071F9238A0093A28AA37D04498C
:10429000284601F0D2F903B030BD00BF714E0700CF
:1042A000804E07000B4601461846FFF7DFBF0000AF
:1042B000024B186800B9FEE7FDF7D6BE580E002085
:1042C00037B50C464B880A881E49054601F0F6F8BA
:1042D000218899B1237B8BB9628891420ED38B1AC6
:1042E0004FF47A72534393FBF1F30A212846B3FB50
:1042F000F1F201FB1233144901F0E0F8628892B147
:104300006368608901904FF47A714B43B3FBF2F21A
:10431000B2FBF1F301FB132200920C4922899BB2FC
:10432000284601F0CBF8284601F0D6F8297A11F09A
:10433000010105D1284603B0BDE83040FFF7B8BF02
:1043400003B030BDA04E0700CD4E0700E64E07007B
:104350000B4601461846FFF7B3BF90F8A43223B1CD
:104360000B6823B9083003F018B90D2070470720F7
:1043700070470B68F7B50446CBBB90F8A432C3B3C3
:1043800090F8A932ABB104F0D9FF04F5C25008305F
:1043900028F0E2FC04F5BA50183028F01BFC04F5B4
:1043A000D1500C303CF0B0F904F5C65018302DF067
:1043B000F6F904F1080003F0F4F80027064684F843
:1043C000A77204F52B70019003F008F9019803F02F
:1043D00007F9054604F51E7003F0F0F884F8A4729E
:1043E0004EB9BD4208BF0546284603B0F0BD0725BB
:1043F000FAE70D25F8E73546F6E70B6810B50446F1
:104400005BB990F8A43253B1083003F0C8F818B97A
:1044100084F8A50284F8A60210BD0720FCE70D2051
:10442000FAE70B6833B990F8A4322BB100F51E708F
:1044300003F0C2B8072070470D2070472DE9FF41F7
:1044400090F8A43205460E46002B5ED000F580534E
:10445000D3F83C37002B5ED10F68002F57D04C6843
:10446000002C54D190F8A83243B390F8A9820846A2
:10447000B8F1000F13D01FF03FFD024605F5BA500A
:104480003946183029F0B8FF002842DA20F08000C1
:1044900010F5D24018BF012004B0BDE8F0811FF034
:1044A0002BFD03AA03460092CDF804803A4605F599
:1044B0002B7105F1080003F085F8EDE790F8A732BD
:1044C0004BBB00F53974C0F8D832C0F8DC4208465E
:1044D0001FF012FD40F62622904203D830461FF00E
:1044E0000BFD02463168C5F8E022204664F052F91F
:1044F000002205F5367105F1080003F048F80028A0
:10450000CAD1012385F8A732C6E70D20C4E70720EA
:10451000C2E72046C0E70520BEE70968006865F0ED
:1045200063B800002DE9F04790F8A4528AB0044621
:104530000E46002D40F0E2800B68002B42D1012393
:10454000A0F8A83240F6262540F6262204F5397157
:1045500004F52B7003F034F82022002102A864F047
:104560002FFA674B039394F8A832002B00F0BF801A
:10457000644B0593644B069304F10806634B079361
:104580002068029404F60A5302AA3146CDE90835A0
:1045900002F0F1FF054688B95D4B039320685D4B3F
:1045A000049302AA04F51E71029402F0FCFF054672
:1045B000002800F09F80304602F0F3FF28460AB042
:1045C000BDE8F087544930461FF09DFCA8B1A4F81F
:1045D000A85270680028B5D002A91FF0C3FC054698
:1045E0000028EBD1029DEB1D05EBD3056A1E40F6BA
:1045F00025239A42A8D90725E0E7484930461FF00D
:1046000082FC074618B10123A4F8A832E1E7444927
:1046100030461FF078FC0028EDD040F2011304F57D
:10462000C658A4F8A83208F1180804F5D15A04F0C5
:104630006BFE0AF10C0A404604F5BA592DF0AAF8AF
:1046400009F11809504604F5C25508353CF058F8F0
:10465000484627F0D5FF284628F014FB3A46314952
:10466000284627F0D8FF3946284627F0CDFF2E49A7
:10467000284627F0D9FF03221146284628F051F892
:1046800003221146284628F047F8E92227490097D7
:104690003B4650463CF03CFD024618B124492046BA
:1046A00000F0CBFF40F22D32224940462DF0FCFCB9
:1046B000024618B12049204600F0BFFF40F299227F
:1046C0001E4940462DF0F0FC024618B11C49204618
:1046D00000F0B3FF2946484628F0E0F902460028DA
:1046E0003FF477AF1749204600F0A7FF71E7164B5C
:1046F00004933FE7012384F8A4325FE718255DE7C0
:104700009D4E0000FD4E000045500000E5480000B1
:1047100091490000D1490000104F0700174F0700D2
:10472000204F070099960000EC5D0700244F07001A
:104730000D5007002E5007005B53070082530700FF
:104740001B56070042560700C14C000030B590F8D8
:10475000A43287B005460C46A3B1206801A91FF01A
:10476000A7FB58B9606805A91FF05DFB30B9A368C5
:1047700033B901A905F1080002F005FF07B030BD0B
:104780000720FBE70D20F9E730B590F8A43287B099
:1047900004460D46CBB1286801A91FF089FB80B9FA
:1047A000686805A91FF03FFB58B9AB685BB904F511
:1047B0001E74204602F000FF18B901A9204602F03D
:1047C000F9FE07B030BD0720FBE70D20F9E7C0E98F
:1047D00000120122A0F8A82200F580520021C0F8A2
:1047E000A41280F8AA1200F52B73C2F83C17C2F885
:1047F0004017C2F8481700F10801C2F85017C2F874
:10480000543770472DE9FF410B6805460C4693B9B4
:10481000DFF878801A4F002658F8262039462846B7
:10482000033600F00AFF1E2EF6D123682BBB23208F
:1048300004B0BDE8F081134920461FF064FB002856
:10484000E6D123680393104B00930C230DEB030078
:104850000E490A2203F0ADFA03460028E7D0826829
:104860005B68511005EB6200D20744BF6A58D35809
:10487000211D04B0BDE8F04118470020D8E700BF73
:104880001B3A0700143A07001B4500000C5E0700A6
:10489000042A96BF104B114A53F82220104910B534
:1048A000044600F0CAFE94F8A93223B104F5BA50C8
:1048B000183028F08CF904F58052002384F8A532D2
:1048C000A4F8A63204F52B70C2F83C37BDE81040BE
:1048D000C2F8403702F082BEF85D07006A5F070049
:1048E0006056070013B50446019102F049FE019A93
:1048F000214602B0BDE81040FFF7CABF38B51546E3
:1049000090F8A522044662B11D4900F0D7FD294662
:10491000204600F077FE20461A4900F08EFE012066
:1049200038BD00F10801196090F8A9320BB90020D8
:10493000F6E700F5C255083513460121284628F050
:10494000A5F9024618B11049204600F076FE04F59C
:1049500080530022D3F8281A284627F089FE04F550
:10496000D15204F5C6510C321831284627F062FEA8
:1049700002460028DBD00549204600F05EFED6E75F
:104980006856070098560700B1560700D956070029
:1049900037B50D460446019202F00AFE019B2A46F5
:1049A000214603B0BDE83040FFF7A8BF38B51D462B
:1049B0000123044680F8A532044900F07FFD294612
:1049C0002046BDE8384000F02FBE00BFFF5607006C
:1049D00037B50D460446019202F0EAFD019B2A46D6
:1049E000214603B0BDE83040FFF7E0BFF0B52E4FE1
:1049F00087B0044600F58055D5F840371BB900262E
:104A0000304607B0F0BD04F52B710846039102F063
:104A1000E3FD0028F3D0D5F840670399B6F5826F1F
:104A2000334628BF4FF4826398424FF0000216D9F4
:104A30009E4294BF00260126059294F8A92202B353
:104A400004F5BA501A463946183029F0D5FC00282A
:104A500007DDD5F84037059098421DD9FEE7164688
:104A6000EAE720F0800010F5D24F15D001260F495B
:104A7000204600F0E2FD0023C5F83C37C5F840377A
:104A8000BEE705AA0196009204F108003A4602F03A
:104A900099FD06460028EAD1D5F84037059A9B1AB9
:104AA000C5F84037A8E700BF195707002A5B070081
:104AB00000F5805370B5D3F84C27D3F848374FF43E
:104AC000FA515C0801FB02440849B4FBF3F40546C3
:104AD00000F0B3FD4FF47A732846B4FBF3F20449B7
:104AE00003FB1243BDE8704000F0A7BD3F5B070029
:104AF000815B0700F8B50E460546404930461FF079
:104B000002FAD8B13E49284600F0D8FC05F580539A
:104B1000D3F83C672EB13B49284600F08EFD0020BB
:104B2000F8BDD3F848473CB12846374900F085FD29
:104B30002846FFF7BDFFF2E73449EDE73449304638
:104B40001FF0E1F960B395F8A732002B54D105F5B9
:104B50008054D4F83C37002B4ED17068A8B94FF47C
:104B60009033C4F83C37B368D3B901F0BCF895F87A
:104B7000A872D4F83C67C4F84407C4F840678FB102
:104B80002846BDE8F840FFF731BF05F5B9511C31A3
:104B90001FF0E8F90028C3D1D4F83C37002BE2D14C
:104BA0000720BDE705F5397340F626226121184636
:104BB00063F006FF06F6252140F625229142AED984
:104BC00040F62623B6FBF3F203FB1266002E18BF55
:104BD000334605F5B951C4F83407C4F83077C4F842
:104BE00038373A46103105F1080002F0D0FC0028B1
:104BF00095D0C4F83C7793E7052091E79C5B0700CC
:104C0000A35B0700BA5B0700C25B0700CC5B070031
:104C1000D55B070038B5054605F5805401F063F80B
:104C2000D4F84437C01AD4F83C37C4F84807C4F85D
:104C30004C372846FFF73CFF0023C4F83C3738BD0B
:104C400070B590F8A8620446114606B1FEE700F57B
:104C5000805500F53673D5F83C2742B9994205D105
:104C600090F8A73203B9FEE780F8A72270BD9942F9
:104C700000D1FEE7D5F840378A68934200D2FEE7BC
:104C80009B1A40F625229342C5F840370FD940F6CB
:104C900026238B603246083002F079FC0028E5D0EC
:104CA0000649204600F0C9FCC5F83C67DEE7002B4A
:104CB000DCD1BDE87040FFF7ADBF00BF2A5B070045
:104CC00013B50446019102F05BFC019A214602B043
:104CD000BDE81040FFF7B4BF73B500F5BA551835FD
:104CE00011490446284627F0DFFC024618B10F4957
:104CF000204600F0A2FC0E220D49284627F0BCFCFD
:104D0000024618B10B49204600F097FC002604F536
:104D1000BA51094B094A00961031284627F07EFC0B
:104D200084F8AA6202B070BDD95B0700E35B07009C
:104D3000085C0700175C070019760000E5750000A5
:104D400038B590F8AA320546CBB900F5BA501830FC
:104D500027F072FD0124024638B90A49284600F0BE
:104D60006CFC85F8AA42204638BD20F0800313F57C
:104D7000D24FF8D00449284600F05FFCF3E7002446
:104D8000F1E700BF475C07005E5C0700F0B590F8F4
:104D9000A43287B004460F46002B5FD000680DF1A7
:104DA000030301AAFCF7FCFF054608BB9DF803308E
:104DB0003BB12B49204600F081FB01A9204600F0C1
:104DC000E5FB786805A91FF02EF8054680B9BB6899
:104DD000002B41D007F10805224928461FF093F81F
:104DE000064640B9204928461FF08DF820B907250E
:104DF000284607B0F0BD0126FB68002BF7D194F8D8
:104E0000A9326BB1002304F5C2501A461946083086
:104E100027F03CFF024618B11449204600F00DFC73
:104E2000324601A904F1080002F0AFFB0546002854
:104E3000DED1012384F8A532734084F8A63294F8B9
:104E4000A932002BD4D0002ED2D12046FFF744FF48
:104E50002046FFF775FFCBE70126D0E70D25C7E712
:104E6000775C0700A05C0700A55C0700B15607004F
:104E700010B50446084900F0E0FB94F8A93253B19C
:104E800094F8A6323BB92046FFF726FF2046BDE83E
:104E90001040FFF755BF10BDAA5C070007B5019091
:104EA00002F06EFB019903B05DF804EBFFF7E0BF81
:104EB00038B590F8A8320446154603B9FEE7114606
:104EC00000F52B7002F086FB94F8A93213B120464E
:104ED000FFF736FF04F58053D3F83C276AB1D3F8C7
:104EE000403723B12046BDE83840FFF77FBD25B9E4
:104EF0002046BDE83840FFF78DBE38BD37B50D46BA
:104F00000446019202F03CFB019B2A46214603B075
:104F1000BDE83040FFF7CCBF2DE9F0471F4690F8C1
:104F2000A532ADF5007D04460E461546CBB990F886
:104F3000A922012380F8A53280F8A6327AB994F824
:104F4000AA32DBB994F8A932002B4BD097B1334980
:104F500020460DF5007DBDE8F04700F06EBBFFF781
:104F6000BBFE94F8A932002BE9D02046FFF7E8FEFB
:104F70000028E4D00DF5007DBDE8F087002DE5D0D8
:104F800094F8A93283B304F5BA56DFF89880DFF8B5
:104F9000989018360DF10C0A4FF4FA7251463046CB
:104FA00029F016FE021E07DA12F5D24F0CD0494640
:104FB000204600F042FBEDE7CDF800A01346414645
:104FC000204600F03AFBE5E715492A46204600F066
:104FD00034FBBBE7454500D0FEE72946304602F0EA
:104FE000DAFAB3E7002DB1D003A9304602F0D1FAC6
:104FF000DFF838904FF00008039A002AEAD0D2E98F
:1050000001234946009220461A4600F016FB039BF6
:105010009A681B6803939044EEE700BF315D070078
:10502000FB5C0700DE5C0700C65C0700145D070040
:1050300010B400F108048C4200D0FEE75DF8044B88
:10504000FFF76ABFF7B50D4616461F46044602F045
:1050500097FA009733462A462146FFF7E9FF03B047
:10506000F0BD00F10C01006802F0B5BD13B500F110
:105070000C0104460068019102F09DFD40B9064A0A
:1050800001992068234602B0BDE8104002F08EBDB1
:10509000182002B010BD00BF1954000010B50C68F4
:1050A0000B4634B100F10801BDE81040184600F08D
:1050B0005BBB017A00F0D2FA204610BD0968006897
:1050C00064F092BA70B50C4686B005461349204686
:1050D0001EF019FFB0B104340026206801A91EF0AB
:1050E000E7FE68B9606805A91EF09DFE40B9A36897
:1050F00093B92868334601AA05F10C0102F070FD4E
:1051000006B070BD064920461EF0FDFE10B1043405
:105110000226E2E70126E0E70720F1E7845E0700C8
:10512000875E070030B587B004460DF103030068C1
:1051300001AA0D46FCF734FEB8B99DF803303BB127
:105140000C49204600F0BAF901A9204600F01EFAE9
:10515000686805A91EF067FE38B9AB683BB92068DE
:1051600001AA04F10C0102F040FD07B030BD072098
:10517000FBE700BF775C070010B50123C0E9001210
:1051800004460372342200210C3063F019FC2046DF
:1051900010BD73B5302305460C468DF807306126E7
:1051A000DCB101220DF10701284602F059F9A8B936
:1051B0009DF807305A2B07D07A2B0AD0392B0AD109
:1051C00041238DF8073001E08DF80760013CA4B25F
:1051D000E6E73023F5E70133F3E7204602B070BD80
:1051E00070B590B005460191322603AA0DF10A016F
:1051F00001A8ADF80A601EF07CFE044608B1242820
:105200000AD1BDF80A2003A9284602F029F908B1FD
:10521000044601E0002CE8D1204610B070BD00002B
:10522000F0B58DB00F4601238DF805300546037AA1
:105230008DF804302622002102A863F0C1FBBB6870
:10524000EBB128680DF1060306AA3946FCF7A8FD64
:105250000446002857D19DF806303BB12C4928461A
:1052600000F02CF906A9284600F090F978680DF1B5
:105270002A011EF0D8FD0446002844D108372868CA
:1052800001A902F085FC064600283BD0214938469A
:105290001EF039FED0B178680DF106011EF0C3FD95
:1052A000044678B9BDF806103046FFF772FF044691
:1052B00040B9286802AB324605F10C0102F09AFCB5
:1052C000044600B3304602F0C3F81CE012493846E9
:1052D0001EF019FE28B17968C1B13046FFF780FF92
:1052E000E5E70E4938461EF00EFE00B104373C6873
:1052F00064B138461EF000FE21460246304602F0F8
:10530000AFF8D4E7032420460DB0F0BD0724D9E759
:105310008A5E0700B05E07003C3F0700B35E0700EF
:105320002DE9FF410B6805460C4693B9DFF87880FC
:105330001A4F002658F8262039462846033600F032
:105340007CF9122EF6D123682BBB232004B0BDE8D4
:10535000F081134920461EF0D6FD0028E6D12368CF
:105360000393104B00930C230DEB03000E49062210
:1053700002F01FFD03460028E7D082685B685110E9
:1053800005EB6200D20744BF6A58D358211D04B010
:10539000BDE8F04118470020D8E700BF1B3A0700DE
:1053A000143A0700BD500000E05E0700F0B5044667
:1053B000ADF2E45D08460D46164602F04BF807468E
:1053C000284602F04BF811493A1A204600F076F8C8
:1053D00006F11001204600F0C7F8728C0C492046F7
:1053E00000F06CF8284602F039F801AA014640F2B4
:1053F000DB53284602F036F801AA0023135405496E
:10540000204600F01AF90DF2E45DF0BDB65E07002B
:10541000ED3A07001B3A0700FFF7C8BFC0E90012CA
:10542000704700232DE9F041137550EA010305464A
:105430000C4606D1302302F11306D3743046BDE882
:10544000F08102F11406284621460A22002361F069
:10545000C7FF303206F8012D0023284621460A22D4
:1054600061F0BEFFA8462746B8F10A0F77F10003A6
:1054700005460C46E7D2E1E737B504460722684601
:105480000D4603F021FC642142F2107363434FF692
:10549000FF70B3FBF0F36846B3FBF1F201FB12338C
:1054A000024903F039FC284603B030BD285F0700ED
:1054B000D0E9003018474068FFF7FABF0EB403B5D3
:1054C00003AA52F8041B0192FFF7F5FF02B05DF842
:1054D00004EB03B0704700000149FFF7EFBF00BFC6
:1054E000585307000A46024B0249FFF7E7BF00BFC7
:1054F000F9A10700505F0700F8B5074E07460C46B4
:105500008D18AC4206D014F8012B31463846FFF70F
:10551000D5FFF6E7F8BD00BF305F070010B50446C1
:10552000FFF7EAFF2046BDE81040FFF7D5BF0000B7
:1055300010B586B01946044610466A46FFF771FF5B
:10554000034902462046FFF7B9FF06B010BD00BF71
:105550001B3A070010B50446FFF7EAFF2046BDE8F6
:105560001040FFF7B9BF000010B58AB004462822EA
:105570000846694601F094FE03496A462046FFF753
:105580009DFF0AB010BD00BF1B3A070010B50446CE
:10559000FFF7EAFF2046BDE81040FFF79DBF00007F
:1055A00010B58CB004462D220846694601F07CFEF9
:1055B00003496A462046FFF781FF0CB010BD00BFCB
:1055C0001B3A070013B5CC884B880A8864BAA4B28A
:1055D0000194898849BA89B25BBA52BA00919BB2E8
:1055E000024992B2FFF76AFF02B010BD355F0700B3
:1055F00010B50446FFF7E6FF2046BDE81040FFF770
:105600006BBF000010B58CB00446302208466946D6
:1056100001F048FE03496A462046FFF74FFF0CB0F1
:1056200010BD00BF1B3A070010B50446FFF7EAFFA4
:105630002046BDE81040FFF74FBF0EB417B505AACE
:10564000044652F8041B0192FFF735FF2046FFF78E
:1056500043FF03B0BDE8104003B07047034A044B5A
:10566000002914BF11461946FFF7E7BF465F070040
:10567000AB4007000CB473B506AD044655F8046B97
:10568000FFF730FF2A46314620460195FFF713FF0A
:105690002046FFF721FF02B0BDE8704002B070471E
:1056A0002DE9F341DFF83C800D4F14468E18B442CB
:1056B0000FD041460190FFF701FF14F8015B0198FC
:1056C000002DF4D03946013D0190EDB2FFF7F6FE12
:1056D000F5E7044902B0BDE8F041FFF7AEBF00BFF7
:1056E0001FA8070037A707002DE9F04FDFF87090DB
:1056F000DFF870B085B004460E461F46154603F12C
:10570000FF3802EB810A55451CD055F8043B18F8C8
:10571000012F03921846029365F012FA039A029B36
:105720000230904206D8C2F1010259462046FFF7E6
:10573000C5FEE8E700934946134620465242FFF76C
:10574000BDFEE0E720460549FFF777FF3A463146C0
:10575000204605B0BDE8F04FFFF7A2BF123A0700A0
:10576000545F07004E5F070070B50D4609490646B5
:105770001EF0C9FB044618B101232B70002070BD38
:10578000054930461EF0BFFB08B12C70F6E7232018
:10579000F5E700BF5B5F0700625F070073B5064671
:1057A00008460DF107011546FFF7DEFF044630B944
:1057B0009DF807103068A847204602B070BD23242A
:1057C000FAE737B5054608460DF107011446FFF71D
:1057D000CBFF28B99DF807102868A04703B030BD5B
:1057E0002320FBE770B50E68154604461A461EB125
:1057F000BDE87040FFF7D2BF0068A84701462046C9
:10580000FFF72CFF304670BD70B50E681546044694
:105810001A461EB1BDE87040FFF7D3BF0068A84725
:1058200001462046FFF71AFF304670BD00F14020C8
:1058300000F50030002382B0036003680193019BF0
:1058400002B0704708B5094B020103EB0010084B8A
:105850004168C3F84813C168C3F808130089FFF70B
:10586000E5FF044B0021995408BD00BF745F070099
:1058700000400240D02C002037B521490122D1E858
:105880004F3FDBB28DF807309DF807306BB1BFF3A7
:105890002F8F1C4BD3F804211B4B12B91A68D20767
:1058A0002CD518680230400826E0C1E8432F002BB1
:1058B000E5D1144B0222C3F80823BFF35F8FD3F85E
:1058C0000431114A4BB1136801331360BFF35F8F8A
:1058D0004FF48270FFF7AAFF01231068094C0225DC
:1058E00001304008C4F80453BFF35F8F00240C70EC
:1058F00013B113680133136003B030BD1868D2E7E9
:10590000C02C002000400240C42C00202DE9F041B2
:1059100006460C46FFF7B0FF0546BFF35F8FDFF882
:105920002080D8F80475BFF35F8FFFF7A5FF3060C4
:10593000854218BFD8F804752760BDE8F08100BF24
:105940000040024013B5044601A96846FFF7DEFF98
:10595000019843F6095240F2FF130021E0FB0231A7
:10596000580A009A064B40EAC150490AE2FB03017B
:1059700024B94FF47A72002361F032FD02B010BDF9
:105980000080841EF8B5194D05EB0013044606018E
:105990001889FFF74BFF0F462046FFF7D3FF3FB9AB
:1059A000134B3344D3E90223904271EB03031CD31E
:1059B0003544104B6A68C3F84823022CEA68C3F8E0
:1059C00008230AD0032C0CD0094A012393550A4A14
:1059D0001370BDE8F84000F0BABFBDE8F84043F0EE
:1059E000FDBDBDE8F84043F019B9F8BD745F07008C
:1059F000D02C002000400240BF2C00202DE9F041B7
:105A00003D4D3E4E05EB021C1401DCF80C70C6F84F
:105A10000873DCF80470C6F84473D3E90067B04239
:105A20005DD9831B002B5ADA013F0026431846EB51
:105A300006003844F31832B94FF47A7101FB00F6CE
:105A4000A3FB013030442E495E0B46EAC046470BAB
:105A5000A6FB016E01FB07EE360F46EA0E164FEA73
:105A60001E7E43F609514FEA4E2747EAD6574FEAC2
:105A7000462CA6FB01689E1B01FB0E8E60EB0E0EF2
:105A8000204B40F23140704303FB0E00A6FB036342
:105A9000013E184447F6FF7340EB0300C00B10EBC8
:105AA0000C0047F1000720F07F46A0FB010301FB3B
:105AB000073140F2FF13C01841F10001B2B1400AB2
:105AC00040EAC150490A104B0C4A2344C3E9020181
:105AD0002B5903F5A87342F82360BDE8F081B0426A
:105AE000A3D2361A002EB8BF01379EE74FF4FA2230
:105AF000002361F075FCE6E7745F07000040024098
:105B0000D07B63087B2DE8BDD02C0020F0B585B09C
:105B100005460E46684601A91446FFF7F7FE019AAE
:105B20002B4F43F6095040F2FF130021E2FB0031F6
:105B30005B0A009A43EAC153490AE2FB073118465F
:105B400024B94FF47A72002361F04AFCCDE90201D6
:105B500002AB224631462846FFF750FF1D4B019A03
:105B6000D3F804359A4203D001A96846FFF7CEFE68
:105B7000019B43F60952023340F2FF100021E3FB80
:105B80000201400A009A124B40EAC150490AE2FB66
:105B9000030124B94FF47A72002361F021FC0E4B0B
:105BA00003EB0413D3E90253A84271EB03034FEA5A
:105BB000041206D301212046FFF7E4FE40BF05B0E2
:105BC000F0BD064B1344DA68024BC3F80423F6E732
:105BD0000080841E00400240D02C0020745F07002B
:105BE00038B52A484022002162F0EAFE284B002006
:105BF0001860284B1870284B00240025C3E9004585
:105C000046F06CFC46F0A8FC0028FBD0234BC022D9
:105C100083F824231022C3F884215A60204A0023E9
:105C2000C2F808354FF48270FFF700FE0223C2F875
:105C300044334FF4A070C2F80433FFF7F7FD4FF47C
:105C40008033C2F848334FF4A270C2F80833FFF72C
:105C5000EDFD4FF40033C2F848334FF4A470C2F89E
:105C60000833FFF7E3FD4FF48023C2F848334FF4C5
:105C7000A670C2F80833FFF7D9FD4FF40023C2F82D
:105C80004833C2F808330123136038BDD02C0020FC
:105C9000C42C0020C02C0020C82C002000E100E013
:105CA000004002402DE9F04100260B4F0446B0466B
:105CB0000A4D87F800802B7C1BB120462E7403F020
:105CC000D3F92B781BB120462E7003F095F93B7861
:105CD000002BEDD1BDE8F081BF2C0020D02C00209E
:105CE0000120FFF72FBE08B5FFF7FAFF4FF47A72D5
:105CF000002361F075FB08BD084611460022FFF73E
:105D000005BF0020FFF79EBD08B5FFF7E9FF08BDFE
:105D1000084611460122FFF7F9BE0120FFF792BDA8
:105D200070477047044B4FF48022C3F80823BFF339
:105D30004F8FBFF36F8F704700400240024B4FF40C
:105D40008022C3F80423704700400240FFF7DCBF05
:105D50001F2070470222FFF7D9BE0220FFF772BD55
:105D600030B5144D144C85B0694601A8FFF7CEFD3F
:105D7000009943F6095240F2FF100023E1FB0203B1
:105D8000400A019A40EAC3505B0AE2FB0503CDE9F1
:105D90000203032202AB3E21FFF730FE4FF4002343
:105DA000C4F80433D4F80435009A9A42DCD105B023
:105DB00030BD00BF0080841E0040024037B504465D
:105DC00003200D46FFF7BEFD6B46CDE9000103221F
:105DD00029462046FFF712FE034B4FF40022C3F87A
:105DE000042303B030BD00BF004002400320FFF792
:105DF00029BD0000214A08B5012353604FF4A0706B
:105E0000FFF714FD4FF48033C2F848334FF4A2700B
:105E1000C2F80833FFF70AFD4FF40033C2F84833E5
:105E20004FF4A470C2F80833FFF700FD4FF480234D
:105E3000C2F848334FF4A670C2F80833FFF7F6FCF7
:105E40004FF40023C2F84833C2F808330223C2F8E3
:105E500008334FF48270C2F84833FFF7E7FCFFF7CE
:105E6000C5FF074B1022C3F88420C3F88421002209
:105E700083F82423BDE8084046F05ABB00400240A6
:105E800000E100E0004870474C410240014B986B34
:105E9000704700BFD02C0020114BD3F8042170B5FF
:105EA00022B10222C3F80823FFF7E6FC0D4D0C4E89
:105EB0000024D6F80423EB681A420AD02B8903F198
:105EC000402303F500331B681BB10021E0B2FFF74C
:105ED00059FD0134042C05F11005EAD170BD00BF55
:105EE00000400240745F0700FFF7FABE012303FA87
:105EF00000F0084A82B0C04352E8003F0193019B82
:105F000003400193019B42E800310029F4D102B023
:105F1000704700BF802D0020074A82B052E8003F42
:105F20000193019B23F001030193019B42E800319F
:105F30000029F3D102B07047802D00200123094AC7
:105F400082B003FA00F052E8003F0193019B034343
:105F50000193019B42E800310029F4D102B000F026
:105F6000F6BC00BF802D0020F4230B70CE234B70B5
:105F700036238B704FF0805382B01A6E5B6EC1F87F
:105F80000330CA7102B0704707B58DF8041001A83C
:105F9000090A8DF8051042F0CBFE03B05DF804FB52
:105FA00010B40748CB1D1C7800F8014B8B4203F15D
:105FB000FF33F8D15DF8044B084642F0BBBE00BF8A
:105FC000502D002007B58DF8041001A8090A8DF89E
:105FD000051042F0B1FE03B05DF804FB08B5114BAB
:105FE00001221A70104B7F221A70104B104A1A604F
:105FF000104ADA60104A00231370104A194642F81A
:1060000023100833802BFAD110227F210C4862F034
:10601000D7FC0C482022002162F0D2FCBDE80840E9
:1060200042F097BE492D0020482D0020A02F0020CF
:10603000D12F0020C02F0020942D0020982D00206B
:10604000602D0020102D002008B542F0C7FE42F060
:10605000A5FE024B00221A6008BD00BF802D002063
:1060600008B50C4B1B7883B942F0ACFE04280ED067
:1060700004D8022814BF0220012008BD0638C0B28F
:10608000022834BF03200220F7E70020F5E70320B1
:10609000F3E700BF492D0020034B1A7812B100200E
:1060A000187070470D207047492D002010B5084C1E
:1060B00023784BB9FFF7D4FF012803D0054B1B68A9
:1060C000DB0703D501232370002010BD0D20FCE762
:1060D000492D0020802D002008B542F082FE28B90D
:1060E00000F093FDFFF718FF002008BD0020FFF728
:1060F00013FFFFF723FFF7E70B68F7B58A8803F86C
:10610000012C07460C4642F05DFE022801D100F04A
:106110007BFD204600F082FC90B1204600F083FC1D
:1061200070B1E37E9B070BD41E4B2046197800F01C
:1061300098FC1D4B196820464A1C1A6000F093FC1D
:106140006669A079D6B1256800903346681E226939
:10615000012142F060FE0028064612BF00250D25F1
:106160000126FFF7D9FE384621460BF05CFC16B934
:106170000220FFF7E3FE284603B0F0BD42F0BEFD6B
:10618000E57E206815F0040505D00138354642F05B
:1061900081FE0126E5E72946013842F030FE064639
:1061A000DFE700BF582D00205C2D0020004870471D
:1061B000A02F002008B5064B4FF4206043F00103E8
:1061C000984742F036FEBDE8084042F034BE00BFBA
:1061D000C05F0700FB20704742F03EBE084642F019
:1061E0003DBE084642F03CBE07B58DF80410090AD2
:1061F0008DF8051001A8002142F034FE00280CBFE4
:106200000320002003B05DF804FB08B50846012117
:1062100042F028FE00280CBF0320002008BD07B56F
:106220008DF80410090A8DF8051001A8002142F02C
:1062300022FE00280CBF0A20002003B05DF804FBFA
:1062400008B50846012142F016FE00280CBF0A20BE
:10625000002008BD002042F011BE012042F00EBE19
:106260004FF47A7310B55A430A4C0B4B2260084620
:106270001970FFF751FE42F041FD206842F0D3FD56
:1062800020B10520FFF732FE002010BD0520FFF7EA
:1062900055FEF9E74C2D00204B2D002010B50C4683
:1062A00021B142F03EFD2070002010BD0720FCE728
:1062B00013B50C4661B101A842F0EAFD054A9DF80C
:1062C000053012785E3B9B1A2370002002B010BD8F
:1062D0000720FBE7592D002013B50A4B1B78194402
:1062E00048B210F15E0F0BDB0024019442F02AFD4E
:1062F0008DF8050001A842F0C4FD204602B010BD93
:106300000720FBE7592D002021B1034B1B780B70B0
:106310000020704707207047592D0020F7B50B4C1F
:10632000054601A80E4694F9007042F0B1FD9DF8B3
:106330000530217826705E3B591A49B22846FFF78E
:10634000CBFF00B1277003B0F0BD00BF592D002076
:10635000F8B5404D0446102600272B684BB1204667
:10636000002229460BF056FB28682F60013842F0C6
:106370005EFD013E05F12005EFD1374D2B689F07EB
:1063800012D5364F0120FFF7B1FD3A683449002A93
:106390002046334618BF3A460BF04EFB386818B11A
:1063A000013842F044FD3E602B685E0708D50220AC
:1063B000FFF79CFD2A490F23002220460BF03CFBEF
:1063C0002B68180708D50320FFF790FD24490E23FA
:1063D000002220460BF030FB2B68D90608D504209C
:1063E000FFF784FD1F4B00211A7820460BF012FBAB
:1063F0002B685A0608D50620FFF778FD1A4B204671
:1064000093F900100BF026FB2C6814F0010408D05F
:1064100042F0E7FC0446A0B900F0F7FB2046FFF786
:1064200065FD2B689B0611D5104B187842F066FC71
:106430000F4B186842F0F7FC28B9BDE8F84000F0AF
:1064400086BA0124EDE70520FFF750FD002CF4D1BA
:10645000F8BD00BF982D0020802D0020102D0020B9
:10646000A02F0020942D00204A2D00204B2D00202D
:106470004C2D00202DE9F047DFF8D4901F4605464B
:106480008846924600235C0154F8091000294FD138
:1064900009EB04062022304662F092FA6B1C49F8A0
:1064A00004302B78B38086F8158086F816A042F069
:1064B00034FCB0716A78DFF89C8012F020023ED183
:1064C0004C4404F11009E37D62F3000389F80730BE
:1064D000FFF71AFC29788246384642F036FC074618
:1064E000FFF7FEFBAAEB0703C01A61F10001C4E944
:1064F0000201002388F800306B78124D13F0200F52
:1065000010D0304600F080FA60B199F807302A7850
:1065100062F3410389F807300B4B1B6823610B4B77
:106520001B78237500232B70BDE8F04700F00FBAED
:106530000133102BA7D1002301351D60FFDE98F831
:106540000020BDE7362D0020302D0020342D002006
:10655000982D0020352D0020431E092B09D8DFE897
:1065600003F00516191C1C1C1C051C1C0D4B1222CB
:106570001A700D4A002313700C4A0828137001D0BA
:1065800005280DD1074A00201370FFF7D7BC054B33
:106590001122EDE7034B1622EAE7024B0122E7E75F
:1065A0000420F2E7942D0020352D0020362D002008
:1065B00070B54378224A234EC3F3001111701B07B4
:1065C0004FF0000188B00446317033D51C2201A879
:1065D00062F0F6F9631C009368462378ADF8043046
:1065E00000F032FA0446684600F01DFA10B30CB30E
:1065F000154B1B789C421FD05A1E94421ED001336B
:106600009C4217D1114B124D124A29681160124A4F
:1066100002931470214601226846327000F021FA7C
:10662000296868464B1C2B6000F01DFA0B49684630
:1066300000F0E8F908B070BD094BE4E7094BE2E768
:10664000352D0020362D0020582D0020702D0020E3
:106650005C2D0020302D0020342D0020502D0020F6
:10666000382D0020842D00202DE9F047089E144C81
:10667000914698460D4629B92160BDE8F0470120B2
:10668000FFF75CBCFFF740FBAA4607461AF8011B60
:10669000304642F05AFB0646FFF722FBBE1B801B2A
:1066A00061F10001C4E90201C4F800A02B78A380C5
:1066B00084F8159084F8168042F02FFBA071DCE777
:1066C000102D0020013906290AD8DFE801F004075F
:1066D0000704070404000220FFF730BC0320FBE797
:1066E0007047000008B542F029FB034B1870BDE865
:1066F00008400620FFF722BC4A2D00206FF06300FF
:106700007047000010B50A4C204600F087F970B1C0
:10671000204600F088F950B1E37EDB0607D4054B34
:10672000A36020460449BDE8104000F06BB910BDDD
:10673000A02F0020382D0020502D002070477047DA
:1067400000F00CBFFFF7D0BBF8B50020DDE906650F
:1067500017461C4645F086FE0A4B1F7094E80F0052
:10676000094F0A4C87E80F0096E80F0084E80F00F5
:1067700095E80F00064C84E80F00BDE8F8400020C3
:1067800045F072BE582D0020842D0020382D0020A9
:10679000702D002010B500200C4645F063FE034B21
:1067A00000201C60BDE8104045F05EBE5C2D00205E
:1067B00010B500200C4645F055FE054B1A68A24264
:1067C00038BF1C600020BDE8104045F04DBE00BF42
:1067D0005C2D0020A0F10B030F2B9DBF024BC018B6
:1067E00010F90B0C7F207047602D002008B5FFF7D3
:1067F000F1FF074B93F900307F2B04D09842A8BFDC
:10680000184640B208BD7F2808BF0020FAE700BF45
:10681000482D002010B508460C4642F06FFA42F0B1
:10682000D1FA022801D100F0EFF92046FFF7DEFF90
:1068300042F075FA42F0DDFAFFF76EFB00280CBF5C
:106840000D20002010BD000010B50C4642F065FA86
:106850007F2C07D0044B1C70FFF7C8FF42F05FFA93
:10686000002010BD0720FCE7482D002021B1034B7C
:106870001B880B800020704707207047982F00204E
:106880007047000008B5034B08461980FFF7F8FF72
:10689000002008BD982F0020FEE7000010B50C4C2A
:1068A00000F0B1F900F05EF8FFF7CEFB00F0CEF992
:1068B00023780BB900F0BBF9207800F04EFA00F015
:1068C0008DF9FFF797FABDE8104000F0A1B900BFBD
:1068D000E430002010B5124C23780BB1FFF7DEFF37
:1068E000104B0122C3F8402545F0E0FD00F08EF981
:1068F000FFF776F900F02CF923780BB900F0B5F822
:10690000207800F025FA00F093F9FFF767FB00F01C
:106910001FF800F077F900F0A8F80023237010BDED
:10692000E430002000E00140014B1878704700BFC0
:10693000E430002010B50446FFF70AFD00F011FA1C
:1069400000F016F82046BDE81040FFF7ABB97047DD
:10695000034B0022C3F8042501221A60704700BFD0
:1069600000C00040014B01225A60704700C0004047
:106970001A4BF7B51A4CD3F8002125688AB10022CA
:10698000C3F80021D3F800210192019AD3F8082519
:10699000D3F80835920544BF6FEA83536FEA9353E7
:1069A0002360FFF79DF90F4B0F4FD3E90026821AA2
:1069B00061EB060697424FF00002B2413FBF074A23
:1069C00001261660C3E900012368AB4204D003B07E
:1069D000BDE8F04042F0AAB903B0F0BD00C00040ED
:1069E000583000205030002080C3C90170477047E4
:1069F000034B18680028B8BF033040F38700704786
:106A00005830002005F027B808B504F035FC00F434
:106A10004050A0F500535842584108BD036818780B
:106A2000C0F3C000704707B50DF1070104F072FE16
:106A300040B99DF80700A0F108035842584103B03F
:106A40005DF804FB0020FAE707B500230DF107010C
:106A50008DF8073004F0AEFE9DF8070003B05DF836
:106A600004FB04F0BDBE04F075BE704708B545F0E8
:106A70003BFF002008BD08B5086845F08BFF0020EB
:106A800008BD08B5104645F049FF80F00100C0B2CE
:106A900008BD002070470000074A084B19681368BA
:106AA00099421FBF1368591C116003F07F031ABF7E
:106AB000034AD05C00207047DC300020E03000202A
:106AC0005C300020074B0022C3F8002182B0D3F8CD
:106AD00000210192019A0122C3F804231A6002B036
:106AE000704700BF00D00040154BD3F8002113B50C
:106AF00022B3D3F80823D20720D50022C3F80021FF
:106B0000D3F800210192019A0E49D3F808450E4BA3
:106B10001A680868121A7F2A06D81A68501C18606A
:106B200002F07F02094884541B680A689B1A7F2B75
:106B300081BF034B0122C3F808235A6002B010BD85
:106B400000D00040DC300020E03000205C3000202D
:106B500038B5802200211C4861F032FF1B491C48D7
:106B600000230B6003601B4BC02283F80D234FF4FE
:106B70000052C3F880211A60174BD3F8042542F065
:106B80000102C3F80425D3F8002222F00102C3F861
:106B90000022FFF797FF03680A689B1A032BFAD9B4
:106BA00003680A689B1A032B0CD9042500200402F1
:106BB000FFF772FF013D40EA0400F8D1BDE838401C
:106BC00062F09AB80020F9E75C300020DC30002049
:106BD000E030002000E100E000D00040074B01223F
:106BE000C3F808235A60064B4FF40052C3F88020C4
:106BF000C3F88021002283F80D23704700D00040A5
:106C000000E100E0704770477047704700F040B8FF
:106C100000F04CB80CB407B504AB53F8042B019347
:106C200000F04AF803B05DF804EB02B0704770471B
:106C30004FF08043044AD3F8001411604FF0FF3244
:106C4000C3F80024704700BFE83000207047000000
:106C500008B500F088F80A4B187018B1094B0422E7
:106C60001A6008BDBFF34F8F0749084BCA6802F48A
:106C7000E0621343CB60BFF34F8F00BFFDE700BF5F
:106C8000E4300020E830002000ED00E00400FA05C8
:106C900008B50121002045F0B7FB0028A2BF024B38
:106CA00001221A7008BD00BFEC300020014B002209
:106CB0001A707047EC30002070B51E461E4B1B78D2
:106CC000A4B004461546002B33D0FFF70CF81B4B3D
:106CD0001B4A0090802103A862F02EFB601E03284F
:106CE00096BF184B184B53F82030184A6D210DF100
:106CF0001F0062F021FB133084B22A4603AD3346F5
:106D0000C4F1800115FA80F065F010FE002810DB58
:106D10000444A4B2802C28BF802404F190036B4467
:106D20000A2203F8842C621C92B22946002045F006
:106D30003BFB24B070BD00BFEC300020CB5F0700F0
:106D4000D35F0700FC5F0700C65F0700DE5F070038
:106D500008B900F00AB800F009B808B900F092B814
:106D6000704700F03DB90020704770477047000041
:106D700030B52E4D287885B0002855D14FF0A0436E
:106D80002B4C4022C3F8082506210322C3F81827FC
:106D9000C3F82007C4F80C150821C4F814152021E5
:106DA000C3F81C07C3F80815C3F814270523C4F853
:106DB00008350723C4F810350123C4F86C354FF0AB
:106DC000EB73C4F82435C4F82001D4F820310393C0
:106DD000039BC4F82401D4F824310293029BC4F825
:106DE0000801D4F808310193019B4FF48073C4F873
:106DF00004334FF40173C4F804330E4BC02283F8FC
:106E000002230422C3F880211A6045F0ADFB45F04F
:106E1000E9FB0028FBD00823C4F8003501232360D8
:106E200000202B7005B030BD1820FBE7F9320020A0
:106E30000020004000E100E038B50F4D2B78C3B1D1
:106E40000E4B00240422C3F88020C3F8802183F86D
:106E500002430B4B4FF48072C3F808234FF40172C6
:106E6000C3F80823C3F8004545F0A8FB2C70204662
:106E700038BD1820FCE700BFF932002000E100E037
:106E800000200040024B1B780BB1FFF7D5BF7047C5
:106E9000F93200201FB5284BD3F8042391051ED5E5
:106EA000D3F82421DAB10022C3F82421D3F8243105
:106EB0000193019B204BD3F82021002A3AD00022D5
:106EC000C3F82021D3F8202103921C49039A012200
:106ED0000A70DA6004B0BDE81040FFF738BDD3F89F
:106EE00004235207E6D5D3F80821002AE2D0002275
:106EF000C3F80821D3F8082111490292029AD3F865
:106F000018450A880F4892B284540A880132C2F3A5
:106F100008020A800A880C4909880132C2F3080273
:106F200089B2914204BF4FF40172C3F80823FFF7FE
:106F30000EFDBFE704B010BD00200040F832002075
:106F4000EE320020ED300020F0320020064908B576
:106F50000B683BB1054B1A7822B100220A601A7007
:106F6000F9F74CFD08BD00BFF4320020F8320020D4
:106F700008B5054B054A196811B11378002BFBD0F1
:106F8000FFF7E4FF002008BDF4320020F8320020B3
:106F900073B5104D2B6804460E4683B90E4A2C601B
:106FA0000020C2F82001D2F8201101910199C2F805
:106FB00044450121C2F84865916002B070BD074B9D
:106FC0001B780BB10520F8E7FFF7D2FF2B68002BE9
:106FD000E4D0F7E7F432002000200040F83200202F
:106FE00038B51A4B1A4C1D881A88238892B29BB266
:106FF0009A42ADB226D023889BB29D420BD2208804
:107000002188144BC1F5007113FA80F089B2F9F7A9
:1070100095FC0023238023889BB29D4209D92088B8
:1070200021880C4B691A89B213FA80F0F9F786FCB3
:107030002580094BD3F8042352075CBF4FF401723B
:10704000C3F80423BDE83840FFF780BFEE320020CC
:10705000F0320020ED3000200020004000F5FF401D
:10706000243000F0E9BD00F500404088704700F58D
:1070700000400BF0F5BF00F500400088704700F5B8
:1070800000400CF01FB800F500408088704700F504
:10709000004000238380704700F5A640383005F09B
:1070A000D0BD00F5A640343005F0B6BF00F5A640CF
:1070B0006C3005F0C6BD00F5A640683006F095BA04
:1070C00000F5A640343006F0FDB800F5A640343097
:1070D00006F0A6B800F5A640683006F0F3B800F553
:1070E000A640683006F09CB806F0E0BD08B507F091
:1070F00035F9182808BF002008BD30B5C3B00546D3
:1071000068460C4605F024FA6846294605F009FB56
:10711000684605F029FA30B16846214605F04AFA7A
:10712000002043B030BD0720FBE730B5C3B00446B4
:1071300068460D4605F00CFA2146684605F0D2FB7C
:10714000044618B92946684605F0DDFA204643B0E2
:1071500030BD30B5C3B004460D46684605F0F8F9B9
:107160002946684605F0DDFA2146684605F0BAFB77
:10717000044618B92946684605F0C5FA204643B0CA
:1071800030BD00000846014905F080B9D83600201E
:1071900000F5E040D0F85C0F704700F5FE404C3041
:1071A00006F05EBE00F028BE02F080BB00F5004095
:1071B000D0F83401704700F5004090F83001704776
:1071C00002F088BB02F05EBB143001F073BF1430D4
:1071D00001F0E0BF02F0A3BB004870470C6007005D
:1071E00000F5A24008B57C3019B11CF0ABF90020C5
:1071F00008BD1CF0D1F9FAE700F5A04090F8200294
:10720000704700F5A040D0F87C01704700F5A2401F
:107210007C3009F027B900F5A2407C3009F09CB819
:1072200000F5A2407C3009F0DFB800F5A040D0F8AE
:107230008001704700F5A2407C3008F069BF00F57E
:10724000A2407C3008F0A0BF00F5A04090F8840177
:10725000704700F5A04080F88411704700F5A74002
:107260000A465230002108F0D3BB00F5A7400A4679
:107270005230012108F0CCBB00F5A040002380F87B
:10728000D633704700F5A04300F5A74093F8D633F6
:107290000B70523070470B460146184608F0EABAA8
:1072A00008F060BB09F044BA08F040BB00F5A0400C
:1072B00090F86A04704738B500F5A043044693F887
:1072C000A93693B900F5A840603002F087FF054663
:1072D00048B904F5A640343005F0C4FD04F5A640D5
:1072E000683006F021F9284638BD0D25FBE700F58A
:1072F000A9401430704738B500F5A043044693F810
:10730000A9565DB900F5A9400C3004F04DFD04F517
:10731000AD40283011F04EF9284638BD0D25FBE769
:107320000148FEF721BE00BFD836002000F5A0407E
:10733000B0F86804704738B500F5A043044693F8E8
:10734000A95685B900F5A840603002F041FE04F569
:10735000A640343005F086FD04F5A640683006F0FE
:10736000E3F8284638BD0D25FBE700F5AD400830B1
:1073700002F0B9BB00F5AD40083002F0C0BC00F52A
:10738000A04090F87804704700F5A04080F8781489
:10739000704700F5A04090F87904704700F5A040D0
:1073A00080F87914704700F5A040C0F8AC14C0F81C
:1073B000B024704700F5A04090F86004C0F3C0000E
:1073C000704700F5A04310B593F8204234B900F59A
:1073D000A840603003F0B4FA204610BD0D20FCE751
:1073E00000F5A04310B593F8204234B900F5A84049
:1073F000603002F075FD204610BD0D20FCE700F561
:10740000AA401030704700F5AA40882200211030B1
:1074100061F0D6BA00F5A840603002F02CBF00F54C
:10742000A840603002F04CBF00F5A840603003F087
:10743000A3BA21B100F5A840603003F0B9BA072023
:107440007047012070470FB404B0704700F022BDB0
:1074500000F05DBEC08B704700F05DBE008C7047D1
:1074600000F065BF00F0F1BE10B51C4600F03CFF17
:10747000204610BD02F05DBA02F0A6BA0B4600220B
:107480000146184607F029B870B500F5FB4086B0F4
:107490000E4604306946154618F02BFB044638B9F1
:1074A00032466946284608F040F9204606B070BDCD
:1074B0000D24FAE700F5FB40043018F0C5BA00F5DA
:1074C000E04090F8880D704700F5E04090F88A0E93
:1074D000704700F5E04090F8883D80F88A3E70479C
:1074E00000F5FB40043018F063B800F5FB400430B1
:1074F00018F06EB800F5FB40043018F079B800F5CC
:10750000FB40043018F079B800F5FB40043018F067
:1075100048BD00F5FB40043018F0C0BD00F5FB404D
:10752000043018F0CBBD00000048704752640700DB
:1075300000487047536407000048704755640700CF
:10754000004870475464070000F5004084301CF088
:10755000D3BD00F5004084301CF04CBD01F0FEBAF4
:1075600010B50446FFF727FE20B1201DBDE81040EE
:1075700001F066BC10BD0B460146184609F0F0BC90
:10758000D0F81C02704709F09CBB09F0F1B809F073
:1075900052BA09F02AB909F035B909F04DB909F024
:1075A00052B909F055B90B460146184609F0E2BA3E
:1075B000006A704709F0A9BB09F0FCBA09F005BBE5
:1075C00009F024BF10B40446084621465DF8044B78
:1075D00009F057BF09F022BF09F039BF09F03BBFDE
:1075E00009F03FBF1FB50023019303AB009314467E
:1075F00013460A46D0E9001009F043FF20B903986A
:1076000004B118B104B010BD0148FBE70148F9E727
:107610000094FFFF8097FFFF2DE9F743D0F800901B
:107620008846484601A91546FFF7B3FFF0B904465E
:10763000AC4210D0019E76B1B26871682F1B9742A0
:1076400028BF174608EB04003A4661F0A3F83368F8
:1076500001933C44ECE705B154B100222146484671
:10766000FFF799FF204603B0BDE8F0830148FAE731
:107670000148F8E70094FFFF0097FFFF00F5A040E6
:10768000D0F8C406704700F5AD40283013F094BB25
:1076900000F5A7402830704738B500F5A0430446F0
:1076A00093F8A95685B900F5A740283005F0DCFF0E
:1076B00004F5A640343005F0D5FB04F5A64068304B
:1076C00005F032FF284638BD0D25FBE707B500F56C
:1076D000A040694690F8AA368DF8043001A817F04A
:1076E00024F89DF8000003B05DF804FB13B50446D0
:1076F0008DF80410684601A917F027F804F5AD408D
:107700009DF80010283013F06FFB02B010BD00F59B
:10771000A74058300DF057BC38B500F5A0430446DB
:1077200093F8A95685B900F5A74058300DF03AFDF9
:1077300004F5A640343005F095FB04F5A64068300A
:1077400005F0F2FE284638BD0D25FBE700F5B040F8
:107750006030704700F5B0404830704700F5B040E9
:107760003030704700F5B0407830704700F5B140D8
:107770000C30704700F5A7403030704700F5A0424C
:1077800038B592F8A9260546A2B9A9B10B789BB1E4
:1077900000F5A740303006F009FE044605F5A64086
:1077A000343005F05FFB05F5A640683005F0BCFEFF
:1077B000204638BD0D24FBE70724F9E700F5A74074
:1077C0004130704700F5A04393F8A93623B900F57E
:1077D000A740303006F0FEBD0D20704700F5A040F8
:1077E000D0F8E803704700F5A740012258300DF0AB
:1077F0004FBC00F5A040B0F81E04704700F5A04053
:10780000A0F81E14704700F5AD40283012F0D2BA2F
:1078100000F5AD40283012F0B3BA00F5AE40143098
:1078200017F02CBD00F5A04090F8A906704716F09F
:10783000D3BF38B500F5AD44283420460D4610F0CE
:10784000EBFD38B1204610F08DFF03C885E803003A
:10785000002038BD1020FCE708B500F5AD40283009
:1078600010F080FF006808BD00F5A040B0F8B80631
:10787000704700F5AD40283011F078B900F5AD4003
:10788000283012F08BBA00F5AD4010B528300C4608
:1078900021B1BDE81040002113F082B9012110F0A0
:1078A00009FE204610BD0420704700F5AD40283089
:1078B00014F047BA7FB505910A990391099902918D
:1078C0000021019100F5F1409DF8201000917030E9
:1078D00005A90BF0F3FF07B05DF804FB00F5AB4022
:1078E0007C30704700F5AB40102200217C3061F005
:1078F00067B810B500F5A04300F5AD442834204624
:1079000093F8A91610F0BEFC04F5807010BD00F5C8
:10791000AD40283010F0A6BC00F5AD40283013F083
:107920005BBB13B50446684601F0CEF94FF47A709C
:1079300000236A46A4FB000101F0DEFB02B010BD8B
:1079400000F5A040B0F8C808704700F5B1404830D5
:107950000BF0E6BC00F5AD40283014F06CBB00F530
:10796000AD40283013F0C2BE00F5AD40283013F012
:10797000E5BE00F5AD40283015F0D8BB00F5E0407D
:1079800090F8B708704700F5E04080F8B7187047E6
:1079900000F5FE4005F0A8BE08B500F5FE4005F074
:1079A000FCFE002008BD00F5E040D0F8C80E70478E
:1079B00000F5E040C0F8C81E704700F5E04090F8C0
:1079C000B408704700F5E04080F8B418704700F53F
:1079D000E04090F8B508704700F5E04080F8B51831
:1079E000704700F5E04090F8C808704700F5AD40DA
:1079F000283015F0E3BC3E2904D800F5E3405030B0
:107A00001BF072B80720704700F5A04393F8A93621
:107A1000022B05D100F5AD400321283015F04EBCF6
:107A2000033B012B94BF00200D20704700F5AD40B3
:107A3000283015F095B900F5E04090F8B608704789
:107A400000F5E04080F8B618704700F5E04090F887
:107A5000C708704700F5E04080F8C718704700F588
:107A6000B14048300BF06CBC00F5B14048300BF031
:107A700081BC30B500F5B14087B0483015461C4692
:107A80000BF0C8FB80B3837F03F00F03012B02D000
:107A9000063B012B28D82B88009000226846ADF8C1
:107AA00006308DF804200BF0BBF8BDF80630052B2E
:107AB00002D9172007B030BD68460BF058F800F126
:107AC000100350F8042B44F8042B9842F9D1BDF868
:107AD000063068460133ADF806300BF0A1F8BDF86A
:107AE00006302B800020E5E70720E3E73E207047C3
:107AF00000F5E34050301BF046B800F5F24060302E
:107B000009F0C4BF00F5A74058300DF06BBA38B586
:107B100000F5A043044693F8A95685B900F5A7409F
:107B200058300DF061F904F5A640343005F09AF9AB
:107B300004F5A640683005F0F7FC284638BD0D2551
:107B4000FBE700F5E04090F9C908704700F5AD404B
:107B5000283016F0FDB900F5E040C0F8E418C0F890
:107B6000E828704700F5E040084490F86008C00934
:107B7000704707B500F5E34050300AB90DF1060231
:107B80000BB90DF105031BF0ABF803B05DF804FB76
:107B900010B50446084600F093FA024604F5A140E9
:107BA0000021BDE810402C3009F0BABD00F5A1401D
:107BB0002C3009F0DABE00F5A040D0F8B4301BB18B
:107BC000994206D01B6BFAE71720B0FA80F0400903
:107BD00070470020F9E700F5A1402C3009F0EEBE17
:107BE00000F5A1402C3009F03FBD00F5A1402C303C
:107BF00009F07EBD10B492F8324014F00C0F06D09C
:107C000000F5A1405DF8044B2C3009F0BFBD072002
:107C10005DF8044B704700F5A040D0F8B400704701
:107C20004FF6FE7202800022027770474FF6FE7315
:107C300003800023037770470B4601884FF6FE72DE
:107C400091421DBF07C883E8070000201720704736
:107C500007B502884FF6FE739A4209D001230091BE
:107C6000044805491A4619F0E7FB03B05DF804FB28
:107C70001720FAE7D0B50020516407007FB505460C
:107C800001AE2348314619F031FCBDF804202C88A0
:107C9000A2424FF6FE7320D09A4235D09C420CBFD0
:107CA00001240324029B1B4AB3F5967F38BF4FF48F
:107CB0009673934294BF0293029296E8070085E878
:107CC00007002A462146144816F028FF13482A4682
:107CD00021460CF0A1F804B070BD9A4216D09DF870
:107CE0000C202B7A9A420BD1BDF806206B889A4261
:107CF00008D16C68029B9C4214BF04240524D1E780
:107D00000324CFE70424CDE70224D6E70024D4E7F8
:107D1000D0B500209BC420009CB60020A4B6002053
:107D200070B588B00023174C0193054602AA01A93B
:107D3000204617F03DFCB0B99DF81A305B07F5D529
:107D400005F10C04214602A807F0CEFA48B92E7FAF
:107D500002AD0FCD0FC4002E2B68237018BF022672
:107D60000AE0032608E02B7F53B11122002105F120
:107D70000C0060F025FE0126034831460CF000FBA4
:107D800008B070BD5CB40020A4B6002010B5044655
:107D9000FFF774FF2046BDE81040FFF7C1BF034660
:107DA00008461A7F1AB103F10C0107F007BC104610
:107DB00070472DE9F84F0A9D8046894616469A4637
:107DC0004FF0000BB34512D20BEB0604671007FB14
:107DD0000A9739464046A8470028C4F34F0407D005
:107DE00003DD01341FFA84FB34462646EAE7002708
:107DF0003846BDE8F88F000025289ABF024B53F89B
:107E000020000248704700BFE86107004760070094
:107E1000F0B5ABB004460D46164604A9962202A85A
:107E20001F4600F051FF0E21204600F0E2FE0E4BEF
:107E30000E491844009023460E220D4C02A800F073
:107E40006BFF3A46314602A800F045FF2146094A39
:107E500002A800F061FF04AB224610212846FEF77D
:107E6000D9FE2BB0F0BD00BF9D6207008062070005
:107E70001B3A0700F9A107000EB403B503AB0121BB
:107E800053F8042B0193FFF7C3FF02B05DF804EB36
:107E900003B070472DE9F74F044600F10C01492269
:107EA000684600F011FFB4F856504FF6FE739D423D
:107EB0005DD04FF6FF739D4200F097809DB34FF663
:107EC000FD739D425BD0B4F856504A49DFF83491B7
:107ED000DFF834A1DFF828B1684600F01DFF4FF647
:107EE000EF736F1E9D428CBF0123112305F1100813
:107EF0001F441FFA88F8BFB22E46BE4248D0A3885E
:107F0000B34240D9236851469A5D684600F004FFA9
:107F100006F00703072B03D15946684600F0FCFE24
:107F20000136B6B2E9E73E21A06800F062FE00F13A
:107F30000A06B6B2C6F1480606EBD67257103D21C6
:107F4000C2F34F02684600F0F7FEA388A2682A49F0
:107F5000684600F0E1FEF21B92B23D21684600F057
:107F6000EBFE4FF6FD73A4F8563000203EE04822A9
:107F70002D21684600F0E0FE4FF6FF73F3E7002383
:107F8000A4F856309FE74946684600F0C5FEBFE7B3
:107F90001A49DFF87890684600F0BEFEBD4218D05E
:107FA000A388AB4211D923685E5D7E2E0FD8304680
:107FB00060F070F9002808BF2E2632464946684610
:107FC000013500F0A9FEADB2E8E72026F5E72E2640
:107FD000F3E70B49684600F09FFEA388A4F856809B
:107FE0004345C2D84FF6FE73BDE7172003B0BDE886
:107FF000F08F00BF123A07008962070074A50700DE
:10800000113A0700CBDA070097620700E94D070035
:1080100010B5002300F5A1424360083200F10803C7
:1080200019468033934204D0446843F8804C416041
:10803000F6E700F5A04300229A6010BDF8B50E4E99
:1080400004460F46656885B104F5A0402B6863605F
:108050000389428901339BB29342038138BF13469F
:10806000438100232B602846F8BD394630460FF087
:1080700037FC0028E6D0F6E7888C002010B500F524
:10808000A04241B143680C680B6013894160013B19
:1080900013812146F5E710BD4A681AB98B680BB900
:1080A000FFF7ECBFFEE700F5A0400089C0F1A0009B
:1080B00080B27047A0207047017042707047000086
:1080C000024B002808BF1846704700BFAC6207008B
:1080D000F8B504460F4605464C26BE42E0682968BE
:1080E0000FD219B17C362D68B6B2F6E794F831108C
:1080F000C1F34101FFF7A2FF28600028F2D103205D
:1081000004E000242C60FFF7B9FF2046F8BD0146CB
:10811000C068FFF7C1BF38B5838B0D46194489B2DB
:108120009942044608D3FFF7D3FF20B9238CE58397
:10813000AB4200D9258438BD0720FCE70368012045
:108140001BB101301B68C0B2FAE77047038CC28BC9
:108150001944914200DDFEE789B29142018400D9C1
:10816000FEE77047C38B8B4200D2FEE70184704765
:1081700090F83030C3F3C3030A2B09D8012202FA66
:1081800003F340F24E72134214BF012000207047E7
:1081900000207047C38B8B4200D2FEE75B1AC3837B
:1081A000038C828B8B420A4486BF591A89B2002104
:1081B00082830184704730B5C48BA1420BD3002168
:1081C000998011889888884288BF998011889B88F7
:1081D000CB1A138030BD15880D44A542A4BF641A84
:1081E0001480848B9860214489B24B29044605D8B9
:1081F000343008441860C1F14C01E1E74C3924687F
:1082000089B20CB99C60FEE77B2906D89C600434D7
:108210000C441C60C1F17C01D2E77C39EFE70B888C
:108220000BB99380704793681B68936003B9FEE7AE
:10823000043313607C2393800B887B2B98BF93803F
:108240000B8892889B1A0B807047F0B587B0154653
:10825000ADF806300DF1060203AB0646FFF7ABFFA3
:108260002C46BDF8107067B103993A46204660F07D
:1082700091FA03AA0DF1060130463C44FFF7CFFF07
:10828000EFE7601B80B207B0F0BD10B51C46FFF7EA
:10829000DCFFA04214BF0620002010BD70B586B0E0
:1082A0001546ADF806301C460DF1060203AB064636
:1082B000FFF781FFBDF810208AB10A9B0398294679
:1082C0001DF023FB58B1BDF8103003AAE41A0DF1DC
:1082D000060130461D44A4B2FFF7A1FFEAE7B4FA55
:1082E00084F0400906B070BD30B587B01446C28B2B
:1082F000ADF806300B449342054600DDFEE703ABC4
:108300000DF10602FFF757FFBDF810206AB12146B4
:10831000039860F0D9FABDF8103003AA0DF10601F8
:1083200028461C44FFF77BFFEEE707B030BD2DE980
:10833000F041B0F81E800F4608EB020189B20546F5
:108340001646FFF7E8FE044628B933463A4641464A
:108350002846FFF7C9FF2046BDE8F0812DE9F0412E
:108360000D46C98B86B017461A4491420646ADF8B1
:10837000063022DBB0F81E80434499B2FFF7CBFEF3
:108380000446D8B903AB0DF1060239462846FFF77B
:1083900012FFBDF810308BB1039A41463046FFF70B
:1083A000A3FFBDF8103003AA98440DF1060128463A
:1083B0001FFA88F8FFF733FFEBE70624204606B0E4
:1083C000BDE8F081F8B504460D46164600F13407C5
:1083D000A38B9E4218D994F83110E068C1F3410193
:1083E000FFF72CFE30B323680360A38B20604B2B78
:1083F00006D83430C3F14C02F918184460F0CAF9B9
:10840000A38B7C33A383E3E79B1BE28BA383238CA7
:108410003244334492B29BB29A42E28300D2FEE7E6
:1084200023844DB1204633462A460021FFF75CFFE6
:108430000020F8BD0320FCE72846FAE7F0B58242A9
:108440000D4689B006461446194601D1AB4216D3F3
:108450006B460EAA2046FFF7AEFEBDF804307BB394
:10846000009A29463046FFF73FFFBDF804106A46E0
:108470000D4420460EA9ADB2FFF7D1FEEDE7BDF8E1
:1084800038201544D318ADB29CB2BDF83830BBB11A
:10849000202B1F4628BF2027E41BDB1BA4B2ED1BAB
:1084A000ADF838306A463B462146ADB23046FFF75C
:1084B000CCFE3B466A4629463046FFF715FFE4E707
:1084C00009B0F0BD37B51546009102462946002394
:1084D0000446FFF7B3FF2946204603B0BDE830400D
:1084E000FFF758BE1F2900D9FEE700EBD10080231B
:1084F00090F82C2001F0070143FA01F10A4214BF61
:108500000120002070471F2900D9FEE700EBD100B1
:10851000802301F007010B4190F82C1021EA0301A0
:1085200080F82C1070471F2900D9FEE700EBD1001E
:10853000802301F0070143FA01F190F82C30194330
:1085400080F82C10704700F12C033030834205D0A6
:1085500013F8012B002AF9D0012070470020704742
:1085600038B50B8883848B7880F826300D46044616
:1085700091F9031028300CF091FE297904F12A00BA
:108580000CF0C0FE6B7994F83120C3F3000363F361
:10859000000284F831206B7994F83220C3F3400351
:1085A00063F3410284F8322038BD0B6910B503B182
:1085B000FEE74B6873B98C6864B991F83130086193
:1085C00064F3C30381F83130036823B9C1E90111B1
:1085D000016009E0FEE75B684B6004688C609960AD
:1085E0000368012A5960F3D010BD91F831301B07A0
:1085F00054BF0B690023984200D0FEE74B68C3B11B
:108600008B68B3B10268914203D1994208BF00233D
:108610000360D1E9013253608A689A6091F8312091
:10862000002363F3C302C1E901330B6181F83120F8
:108630007047FEE710B5FFF7D8FFBDE810400846C9
:10864000FFF765BD10B5044623682BB1596819B111
:108650002046FFF7EFFFF7E710BD006800B1406864
:10866000704702460B4652F8230030B9032B1ABF5D
:108670000133DBB203469942F5D1704708B50021BA
:10868000FFF7EFFF00B1406808BD08B550F8213092
:108690004BB103291ABF0131C9B20021FFF7E1FF35
:1086A00000B9FEE74368184608BD0021FFF7D9BFAF
:1086B00010B50446006994F831301B0707D528B17E
:1086C000FFF7F3FFA04214BF6068002010BD002830
:1086D000FCD00068F6E710B504464068206008B199
:1086E000FFF7E6FF606010BD10B50C46FFF7B5FF61
:1086F000024678B1238801332380FFF71FFD63888A
:10870000D18B1844636860800B4463601046FFF7A8
:10871000CFFFEDE710BD10B50446086818B920601A
:108720006060204610BD406820600028F8D0FFF748
:10873000BFFFF5E738B50B6905460C4603B1FEE708
:10874000086191F8311041F0080184F83110C1F34B
:108750004101FFF786FF38B14368C4E901309C60EE
:10876000446045F8214038BDC4E90144F9E791F877
:10877000313010B51C07C3F3C00248BF0A699042EC
:1087800000D0FEE7C3F3410350F8232091420BD100
:108790008A68914218D092F83140C4F341049C4257
:1087A00018BF002240F82320D1E9012393604A68D2
:1087B0005A600023C1E901330B6191F8313043F075
:1087C000080381F8313010BD0022EBE7032910B512
:1087D0000C461ED803693BB990F8313064F342036C
:1087E00080F83130002015E090F83120C2F34101CB
:1087F000A142F7D01207EFD501461846FFF7B7FFA1
:1088000091F8313064F3420381F83130FFF792FF81
:10881000E8E7072010BD2DE9F0410D4659780746DD
:1088200090461E46FFF70AFC044648B3802200210A
:1088300060F0C6F83178238EE76005F0070545EA59
:10884000012525F0F805ED0523F4837323F00103DA
:10885000ED0D1D4394F83230A4F81C8023F00D0375
:1088600043F00503258684F8323071782046FFF7FF
:10887000ADFF014638B121463846FFF70DFC002414
:108880002046BDE8F0812046FFF745FC0028F7D0E0
:10889000F1E70000014B0022FFF7BDBFAC6207000B
:1088A000014BFFF7B8BF00BFAC620700F7B590F807
:1088B0003130C78B0E4690F83010C3F30002C3F37B
:1088C00041038DF804208DF80530828B054601ABFD
:1088D000C06801F00701FFF79EFF044600283DD065
:1088E000BE4228BF3E46334600222946FFF736FDEA
:1088F000002836D12A8C1346B242E28B28BF334679
:108900009A4200D2FEE7238495F8303094F8302064
:10891000C3F3C30363F3C60284F8302095F8322012
:1089200094F8323062F3000384F8323095F8323034
:1089300094F83220C3F3810363F3830284F8322076
:10894000AB69A3616B8C6384AB8CA38495F82630F0
:1089500084F826302B8D23856B8D6385204603B0EC
:10896000F0BD2046FFF7D3FB0024F7E710B5FFF773
:10897000FEFEBDE810400846FFF7C9BB10B504462F
:108980002046FFF77BFE014618B12046FFF7EEFFB9
:10899000F6E710BD10B504460846FFF76FFE034624
:1089A000206010B1FFF784FE03466360204610BDCF
:1089B00008B5FFF763FE08BD10B50C46FFF7F8FFDA
:1089C000024678B1238801332380FFF7B7FB638821
:1089D000D18B1844636860800B4463601046FFF7D6
:1089E00067FEEDE710BD000006490022C0E9002245
:1089F000C0E90212C0E90422C0E90622C0E9082247
:108A0000704700BFB98A000003680B4303604368E6
:108A100019434160083000F009BA4368194201D196
:108A2000FFF7F2BF7047000070B50568044685B3D4
:108A3000002303602946174812F0F4FA1648294625
:108A40000BF0E6FD1548294604F0A2FE144829461D
:108A50000AF0FCFA1348294618F0CCFC12482946C3
:108A600009F0FAFF1148294616F04AF8104829463D
:108A70000BF0B8F90F4829461BF00EFE04F118065A
:108A8000A64206D0236913B1616928469847083485
:108A9000F6E770BD808D00202CB70020D8B50020EF
:108AA000D4B60020B0B50020C4B700209CB600208A
:108AB000A4B60020788900200148FFF7B5BF00BFA9
:108AC0000037002007B5074A138803B9FEE7013BCA
:108AD0009BB213801BB9019000F030FC019803B0E9
:108AE0005DF804FBFA32002031B16FF00043994287
:108AF00008BF0121016070470121FBE737B50E4D2A
:108B00002B884FF6FF729342044600D1FEE763B90B
:108B100000F0FAFB04210DEB010000F01DFC00B198
:108B2000FEE701990548FFF7DFFF2B882046013358
:108B30002B8003B030BD00BFFA320020FC32002091
:108B4000026848F24E33A2FB0323014613EB5200A6
:108B500044BF20F00043581C08607047034B1B883B
:108B600003B9FEE70248FFF7EBBF00BFFA3200206F
:108B7000FC320020814238B504460D4600D8FEE79D
:108B8000FFF7ECFF2D1BC0B290FBF5F105FB1100C8
:108B90002044C0B238BD814238B504460D4600D8E5
:108BA000FEE7FFF7DBFF2D1B80B290FBF5F105FB25
:108BB0001100204480B238BD814238B505460C46CC
:108BC00000D8FEE7FFF7CAFF641BB0FBF4F101FB1E
:108BD0001400284438BD814238B50C4688BF84B2A1
:108BE0006100054601310020FFF7E6FF2844001B25
:108BF00038BD10B540B10023441E98B2814203D95C
:108C00000133E25C002AF8D110BD024610F8013BA6
:108C10001BB18B42F9D1104670471A46FBE7F0B5FD
:108C2000066800240625374601363B78303BDBB228
:108C3000092B0AD804EB840403EB44039CB2A24240
:108C40004FF00005EFD2062501E007600C702846C2
:108C5000F0BDFF22FFF7E3BFA0F14103192B9CBF3A
:108C60002030C0B2704738B503463AB1012A11D05E
:108C70001B78002B0CBF0222012209E0013911F8F8
:108C8000014F034610F8015B002CF1D0AC42F6D046
:108C9000104638BD0139044611F8015F234614F827
:108CA000010B002DE4D0FFF7D7FF02462846FFF75F
:108CB000D3FF8242F0D00022EAE708B5FFF7D3FFE6
:108CC000831E5842584108BD10B5002401608480BD
:108CD000C2800C7010BD70B504460E46E5888188D0
:108CE0000068A9420844134634BF691A002132467D
:108CF00063F01CFE002800DAFEE7A388E28818442F
:108D000080B2904228BF2368A08022BF9B18002217
:108D100003F8012C204670BD0EB417B505AA044611
:108D200052F8041B0192FFF7D6FF204603B0BDE8BE
:108D3000104003B070470000F8B5074F05460E46D7
:108D400014463CB1324639462846013CFFF7E4FF61
:108D5000A4B2F6E72846F8BDE94D070070B5054610
:108D60000E460024B44226D2285D030604F1010415
:108D700005D45FF07FFA0028F4D000201CE010F04A
:108D80004003FAD0810612D5C20612D50307F4D4E7
:108D90000323013BDBB2FF2BE4D0B442EDD02A5DCC
:108DA00002F0C002802A04F10104F2D0E5E70123B9
:108DB000EFE70223EDE7012070BD10B5044661F036
:108DC000BFFE01462046BDE81040FFF7C7BF2DE9B2
:108DD000F04105461F4614461AB902700020BDE84E
:108DE000F0811046FFF705FF814206460BD9012F9F
:108DF00003D12046FFF7E1FF38B1721C2146284617
:108E00005FF0C8FCEAE70720E9E70620E7E7000093
:108E1000036823B9016004484960F7F793BE5A68B4
:108E20004A60596001607047D836002043680146A7
:108E300013B90248FFF7ECBF704700BFDC360020D3
:108E400038B500250468056054B1606884421CBFD1
:108E5000436863600368456008BF00249847F3E7F0
:108E600038BD4368496810B59C1A8A1AD20FB2EB14
:108E7000D47F08BF5B1A4FEAD47008BFD80F10BD6B
:108E800070B505680C4625B9BDE870404B680848C8
:108E900018478B6898476A68831A002B0146236835
:108EA000B8BF121ABDE870400148A8BF0022184799
:108EB000D836002038B50C461146A26894420346C5
:108EC00006D00568AC4204D10260FFF7D9FFA46068
:108ED00038BD2A460021002AF9D0944208D0114614
:108EE0009268F8E78B68002BF1D09B688B60EEE707
:108EF0000029F7D1002DEAD0AA681A60E7E7000040
:108F00000146024A0248FFF7D5BF00BFBC62070016
:108F1000E03600202DE9F047936805460C461646DA
:108F200098473246814621462846FFF7C3FFD5F8C9
:108F300000A04FF00008574647B14A463946204640
:108F4000FFF78FFF10B9B846BF68F5E7B8F1000F1B
:108F500008D1C4F808A031462C602846BDE8F04787
:108F6000FFF78EBFD8F80830A360C8F80840BDE806
:108F7000F08700004160024A01460248FFF7CABF7D
:108F8000BC620700E0360020002A00DAFEE7114448
:108F9000FFF7F0BF13B504460191FCF7A4FE019A58
:108FA0000146204602B0BDE81040FFF7EDBF8368E0
:108FB000984203D04368CB1A002B01DAFFF7DABFDF
:108FC000704770B5066804460D467EB18B689847B9
:108FD0007368C01A002809DB20462A463146FFF78D
:108FE00069FF33683046BDE870401847294620467F
:108FF000BDE87040FFF744BF10B50446FEF7DBF84C
:1090000030B104F108000349BDE81040FFF7D9BFB3
:1090100010BD00BFBC6207004160024A0146024821
:10902000FFF778BFB0620700E4360020002A00DABC
:10903000FEE71144FFF7F0BF13B504460191FCF7BA
:1090400063FE019A0146204602B0BDE81040FFF7DA
:10905000EDBF00000146024A0248FFF72BBF00BFE8
:10906000B0620700E436002010B50446FEF7A3F80E
:1090700030B104F10C000349BDE81040FFF7A1BF77
:1090800010BD00BFB062070010B50446FCF72BFE10
:109090000023206063600146054BA36004F10800D3
:1090A000206101F18041FFF765FF204610BD00BF40
:1090B000ED90000010B50446FCF715FED4E9003130
:1090C000E2689A42A0EB030002D10028A8BF013158
:1090D00010BD0368C168994202BF43680133436011
:1090E00001F180410830FFF745BF00000148FFF75C
:1090F000F0BF00BFEC3600202DE9F3411F46204BA6
:1091000083424FF000038B4104460E46154611D2B0
:1091100019A3D3E900235EF063F91A4902462846F1
:10912000FFF7FAFD204614A3D3E9002331465EF091
:1091300057F914461448B4FBF0F200FB12444EF603
:1091400060204FF47A78B4FBF0F3104900FB13442D
:109150002846B4FBF8F60096FFF7DEFD47B10C4950
:1091600008FB1642284602B0BDE8F041FFF7D4BD27
:1091700002B0BDE8F08100BF005C260500000000E1
:10918000FF5B2605C862070080EE3600CE6207004E
:10919000DD62070013B504466846FFF795FD2046DB
:1091A000FFF788FF01236A46FFF7A6FF02B010BD54
:1091B000704710B590B183880B2B11D904682046F5
:1091C00037F034F8062037F025F801220146204612
:1091D00037F05CF8003818BF012010BD0720FCE70D
:1091E0000120FAE708B538B183880B2B06D900684F
:1091F00037F020F8002008BD0720FCE70120FAE73F
:1092000013B50446684600F04EFA6CB1A3880B2BE8
:109210000CD9BDF804200099206837F0FDF800381B
:1092200018BF012002B010BD0720FBE70120F9E7BD
:1092300008B548B183880B2B08D9006837F046F988
:10924000003818BF012008BD0720FCE70120FAE71D
:1092500008B548B183880B2B08D9006837F046F968
:10926000003818BF012008BD0720FCE70120FAE7FD
:1092700008B520B100682EF051FF002008BD07207E
:10928000FCE710B5044648B18388EF2B08D9006885
:109290002EF058FF00202060A08010BD0720FCE7C2
:1092A0000120FAE708B550B18388EF2B09D900688F
:1092B00000212EF063FF003818BF012008BD0720F1
:1092C000FCE70120FAE708B548B18388EF2B08D9FD
:1092D00000682EF06FFF003818BF012008BD07207E
:1092E000FCE70120FAE708B548B18388EF2B08D9DD
:1092F00000682EF067FF003818BF012008BD072066
:10930000FCE70120FAE7000007B5094836F00CFD3C
:10931000084836F04DFB0023054A074905480093ED
:1093200036F073FB00B1FEE703B05DF804FB00BF4D
:10933000483400200033002071FD030008B50448C4
:1093400036F0A4FCBDE80840024836F045BB00BF3B
:10935000483400200033002008B50A46014603487F
:1093600036F0F4FBBDE8084000F0D0B80033002030
:109370002DE9F04F9DB0222B0F46DDF89890BDF8F7
:109380009C4006461146984600D9FEE71A4613A8A7
:109390005FF000FA19F0010500D0FEE74FEA59032B
:1093A000059308F170030DEB03090DF12C0B002C54
:1093B00076D001352B0E09F8243C2B0C09F8233C00
:1093C0000DF13C0A2B0A09F8223C09F8215C08F14E
:1093D0000403CDF800A013AA3946304634F0FCF956
:1093E00020B100F093F81DB0BDE8F08F07AB0093FB
:1093F000524610233946304634F0EEF90028F0D1B9
:1094000007A852464FF0040C136850F8041BBCF137
:10941000010C81EA030142F8041BF5D101230393F7
:10942000039B059A93422AD2CDF800B0102307AAD5
:109430003946304634F0D0F90028D2D107AB00933A
:109440005A4610233946304634F0C6F90028C8D1B0
:10945000042358460DF11C0E514604930A685EF829
:10946000043B50F804CB534083EA0C0341F8043B1F
:10947000049B013B0493F1D1039B0133CFE7102CF4
:10948000A24628BF4FF0100A289852460FA95FF055
:1094900081F9289BA4EB0A0453442893A4B286E7DD
:1094A0002046A0E700F1080310B503601023838075
:1094B0000446FFF77EFE00B1FEE7204610BD10B562
:1094C0000446FFF78FFE00B1FEE7204610BD08B549
:1094D000FFF796FE00B1FEE708BD08B5FFF7A8FE4E
:1094E00000B1FEE708BD08B52022FFF7B1FE00B1CC
:1094F000FEE708BD10B503490446034837F0F8FEFF
:10950000204610BDD35A0200BB5A020010F5405F3E
:1095100000F0BB806DDC10F5D04F00F0B88038DC77
:1095200010F5D24F00F0B3802EDC10F5FE4F2ED098
:1095300006DB10F5F04F5AD010F5E24F00F0A9808D
:10954000C00F704700F140030C2BF9D801A252F86C
:1095500023F000BFEF950000419500008F950000BB
:10956000EF950000EF950000419500004195000047
:1095700041950000939600004195000093960000ED
:1095800041950000EF95000010F5D14FD8D1032090
:10959000704710F5705F7CD015DC10F57C5F78D0DB
:1095A00002DC10F57E5FF1E710F5765F71D005DC27
:1095B00010F57A5F6DD010F5785FBFE720F080037B
:1095C00013F5745FBAE710F5665F10D00CDC10F588
:1095D0006A5F5ED005DC10F56E5F5AD010F56C5FE7
:1095E000ACE710F5685FA9E710F5645FA8D1082023
:1095F000704710F5025FFAD037DC10F51C5FF6D02B
:109600000EDC10F5225FC2D005DC10F5265FBED05F
:1096100010F5245F92E720F0800313F5205F8DE7BB
:1096200010F50E5F35D011DC10F5145F31D007DC7A
:1096300020F0800313F5185F2BD010F51A5F7DE73B
:1096400010F5125F25D010F5105F77E710F5085F71
:109650001FD004DC20F0800313F50C5F6EE710F5DB
:10966000065F16D010F5045F68E710F1330F06DAD5
:1096700010F1400FBFF666AF10F58C5F86E710F172
:109680001E0FB4D010F11C0FB0E701207047052069
:1096900070470720704700BF08B5084691B2FFF732
:1096A0005BFE002008BD0A6802608A8882807047DD
:1096B00070B500250446C0E90155C5601030FFF7BC
:1096C00019FF04F11100FFF719FA214604F1140003
:1096D000FFF7DAFC214604F12800FFF785F921465F
:1096E00004F150001CF0D8FA214604F17400FEF792
:1096F0008FFC214604F5A14004F018FF04F5A240B8
:1097000021467C3019F014FF04F5A4402146243092
:1097100019F0D4FF04F5A540214620301AF0B6FD1B
:1097200004F5A6402146343003F0AEFE04F5A64011
:109730002146683003F0E6FE04F5A74021462830B4
:1097400003F0AEFF04F5A7402146303004F04AFE96
:1097500004F5A04304F5A74083F8D65321465830BA
:109760000BF04EFD04F5A84021465C300BF03FFEA7
:1097700004F5A8402146603000F046FC04F5AB40FB
:10978000214630300CF0C4FE04F5AD4021462830AF
:1097900011F03AFF04F5F140214670300AF072F8FA
:1097A00004F5F2402146603008F0A2FC04F5FB40CD
:1097B0002146043016F0B2FC04F5FD402146583035
:1097C00017F02EFD04F5FD4021467C3018F0BEF860
:1097D000214604F5FE4003F06FFF04F5FE402146EC
:1097E0004C3004F0B7FA04F5FF4021462430FEF770
:1097F00017FA04F5FF402146443015F009F804F546
:10980000FF4021464C300AF0A3FD04F5FF4004F56B
:10981000004621467C3009F079FB2146304609F0AC
:1098200059FC30462146143008F0C0FF304621462E
:10983000303018F0D9FE3046214654300AF0E4FDAD
:109840003046214684301AF0B3FB30462146EC30D6
:1098500009F080F886F83051FFF780F9C6F8340136
:10986000204670BD38B5054C236823B9044D284601
:109870001AF05EF82560206838BD00BF10B80020DF
:1098800018B80020FDF7E4B910B500F50043012237
:10989000044683F8302160301CF034F904F5AD4003
:1098A0002830BDE8104010F031BD000010B5074C65
:1098B00094F830313BB9A4F50040FFF7F9FEA4F568
:1098C0000040FFF7E1FF024810BD00BFD8B60020FE
:1098D000D836002038B500F50043044693F830210F
:1098E000E2B1002583F830512946FDF7CCFF294627
:1098F0002046FDF775FC29462046FDF771FD04F171
:1099000060001CF005F904F5A9400C3002F084FA5F
:1099100004F11100BDE83840FFF7D4B838BD10B5E8
:10992000044660301CF0F6F82046BDE81040FDF714
:109930008FB973B50C4605464822002105F174061F
:1099400020465FF03DF83046FEF7B4FB20803046FD
:10995000FEF7A9FB05F5A043608005F5AB46B3F81B
:109960007E30A380303604F108013046FFF724F83A
:1099700004F1100106F11000FEF7B6FE05F5A14056
:1099800004F118010C30FFF717F805F5A24004F1B7
:1099900020014830FEF7A8FE05F5AE4004F128018D
:1099A0001830FEF7A1FE05F5A44004F13001243083
:1099B0000191FEF799FE05F5A4400199483002B0E7
:1099C000BDE87040FEF790BE00F5A040B0F87C30D6
:1099D000A0F87E307047807F00F00F00012804D08F
:1099E000063801288CBF0020012070470022C0E902
:1099F000002282600246044942F80C1F4261028B39
:109A000002F0800202837047999C0000064B93F895
:109A1000422703F2247002F00F0203F5DC63072AE9
:109A200018BF1846704700BFD886002010B50446FE
:109A30000C30FFF765FAE37A6FF38703E372238B49
:109A400003F08003238310BD38B5FFF7DFFF0C461A
:109A50000546FFF7C0FFB0B10C4BB3F892144FF6B8
:109A6000FE72914203D003F224739D4207D12B680A
:109A700023606B68636002232372002038BDAB8BC8
:109A800023800123F8E70B20F8E700BFD8860020E9
:109A9000074BD3F8C406074B984228BF18464FF42B
:109AA0007A735843B0F57A6F88BFA0F57A60704733
:109AB000D88600209BC4200038B5436900F10C050E
:109AC0009D4204460ED0FFF7E3FF6368834209D14D
:109AD000FCF709F96268206001462846BDE8384075
:109AE000FFF752BA38BD024608B5FFF7D1FF9368B9
:109AF00033F07C4204D0C3F31903984228BF1846C0
:109B000008BD024608B5FFF7C3FF137E990702D5CB
:109B1000642828BF64205B0704D5B0F57A7F28BF8E
:109B20004FF47A70537E13F0F00F02D0BC2828BF98
:109B3000BC20936833F07C4204D0C3F319039842ED
:109B400028BF1846002808BF0A2008BD012938B5DB
:109B50004568044602D1FFF7D4FF6060FCF7C3F804
:109B60006369014604F10C0098420DD06268AA4274
:109B70000DD0246813195B1A0A2B4CBF0A22214608
:109B8000BDE83840FFF700BA62682160F8E738BDE9
:109B9000027ED1070BD4064991F8AA16090700D511
:109BA000FEE742F0010202760121FFF7CFBF7047C6
:109BB000D886002038B5037EDA0705461CD5114C3F
:109BC00094F860345B0717D4FFF720FFFFF703FF1B
:109BD00090B105F10C00FFF793F904F58C6000F0EB
:109BE000BDFB044618B10D2806D0012100E0014656
:109BF0002846FFF7ABFF03E02846FFF717FF0D24C9
:109C0000204638BDD8860020017ECA070FD5C1F393
:109C1000C302013202F00F0262F3C601042A017688
:109C200001D8FFF7C7BF027E6FF3C6020276704706
:109C3000037E13F0010F08D06FF3C60303760B68A1
:109C40001B78DB0601D5FFF7B5BF7047F0B4047E83
:109C5000E6071CD50F4E96F8FE763F0717D0B6F8EC
:109C60000067022E13D90968097809070FD573B95F
:109C70006AB1214663F3C601136801761B78DB06DF
:109C800002D5F0BCFFF796BFF0BCFFF715BFF0BCE4
:109C9000704700BFD88600200148FFF78BBF00BF88
:109CA000608D0020037EDB0702D50121FFF74EBF48
:109CB0007047037E10B4C3F340048C4209D061F3B3
:109CC00041030376DB0704D55DF8044B0121FFF760
:109CD0003DBF5DF8044B7047C37A13F0FC010DD013
:109CE000FC290BD0FC33C37213F0FC0306D1417E78
:109CF00063F3071141760121FFF728BF704708B5CC
:109D000031B1092915D96FF07C43994228BF194612
:109D10008368C3F319028A4201D1002008BD61F3B0
:109D200019038360037EDB07F7D50121FFF70EFFE0
:109D3000F3E70720F2E70000F0B5067E87B00023C6
:109D400016F0010604460F4615468DF8143019D05A
:109D50008B885BB103A9384601F000FB0123009317
:109D6000244803AB2A4639460CF082FD2046FFF713
:109D70004DFE837F180707D12046FFF757FE1E4888
:109D800010F018F807B0F0BD05F0FB030B2B1DD049
:109D9000637E05BB13F0F00F0ED10026237E59071A
:109DA00025D5238B23F4706323F00403238301213F
:109DB0002046FFF7CBFEE5E7F03313F0F00F6376B4
:109DC000EBD1E37A65F38703E372E7E7237E43F0A1
:109DD00004032376EBE75A1C02F00F0262F303033D
:109DE000032A6376DDD8237E5A07CBD4EFE7002E13
:109DF000C8D0DCE7888C0020808D0020C37A427EAA
:109E000010B403F0FC04FC2C1CBF0433C372002903
:109E100008BF08210F2928BF0F211309C9B2994291
:109E200038BF1946134661F307134376037EDB07F9
:109E300007D512F0F00F04D15DF8044B0121FFF7B4
:109E400085BE5DF8044B7047F0B58DB005AE0024BB
:109E50000F460DF1260105948DF824408DF82E4013
:109E6000B48007ADFFF7F0FD48BB9DF82E30154AD2
:109E70003C68022B07BFD2F89814D2F89404B2F8C9
:109E80009234ADF81C300CBFC5E900010123B2F8D3
:109E900068148DF82430304601F0FCFE08230022BF
:109EA000CDE902320523CDE90063074821462B4660
:109EB00003220DF0F9F90421204601F048FD204667
:109EC0000DB0F0BDD8860020888C0020012905D176
:109ED0004FF6FF73C31A584258417047002070472D
:109EE000037861F3000300F82C3B09B101F07EBF59
:109EF00001F092BFF0B5154687B00C463C22002118
:109F000028468DF814105EF05BFD6CB323681B7857
:109F10005B0703D00626304607B0F0BD03AF3946D5
:109F2000204601F0A2FA06460028F4D19DF814302C
:109F3000022BEFD197E8030085E8030005F1320119
:109F40002046019101F064FA019910B1204601F018
:109F5000EFF9A37985F8363094F9153085F8373064
:109F6000A37D85F83830D6E70726D4E70378DB07EA
:109F700004D500F1100114301CF0CABB0B2070474F
:109F800010B5026A90B004460B4672B129B9416A15
:109F9000184610B0BDE81040104701AAFFF7AAFF0D
:109FA00018B9D4E9083101A8984710B010BD036A68
:109FB00007B54BB17F2907D0027C8DF805108DF8CD
:109FC0000420416A01A8984703B05DF804FB000033
:109FD00003898B4210B5044606D1BDE810400948FC
:109FE0004FF40041FEF719BD018106484FF40041CE
:109FF000FEF70AFD218904F12C00BDE8104001F0B4
:10A00000C7BE00BF00370020F0B5036885B003F07D
:10A01000C003036004460191FEF7A0FD2071FEF726
:10A020009DFD00252B4B6071A360A5712A4807F0A8
:10A030001BFD0B2323740F2323834FF0FF33C4E94D
:10A0400007350199E06065826561656204F1280069
:10A0500001F0CDFD214B224AC4E92735234604F502
:10A06000A07743F8A42F2946C4F8AC301022C4F8D6
:10A070003851A4F83E5138465EF0A2FC02A801F027
:10A08000E2FD88222946A4F83C5104F1B0005EF0BC
:10A0900097FC2378264643F0010306F82C3B304614
:10A0A00001F0A4FE0F480AF0B1FF21892046FFF716
:10A0B0008FFF02A9304601F077FE618E304601F035
:10A0C0006DFE384608492A4601F0F2FD204605B0EB
:10A0D000F0BD00BFFFFF0B0BD836002035AF0000EE
:10A0E00029AF0000B08A0020EB62070038B5037882
:10A0F000590758BFC3F3C004C3F38002437858BF65
:10A1000084F00104054654BFE4B200249BB932B187
:10A110004388DB0503D5C169A430FEF72BFF05F1A9
:10A120002C001CB1BDE8384001F0D4BFE97ABDE88D
:10A13000384001F085BE38BD1F2908B50CD8C2686B
:10A14000CA40D20708D50278C17242F020020270DC
:10A15000FFF7CCFF002008BD0720FCE7027891063E
:10A1600006D56FF345120270827AC272FFF7BEBF46
:10A17000704710B50378C3F380028A4204462CD09E
:10A1800061F38203037059B92178C1F3C00104F16E
:10A190002C0001F01DFE2046BDE81040FFF7A6BFD1
:10A1A00043885A0606D5A430FEF7AAFE638823F03A
:10A1B000400363806378062B09D104F1A400FEF705
:10A1C0009FFE0023637004F19C00FEF72FFE2378AE
:10A1D000C3F380015B07D7D5D9E710BD1F2938B578
:10A1E00004461FD8C368CB40DA071BD5837A8B425D
:10A1F00006D10D484FF48041FEF70FFC002038BD1A
:10A20000817209484FF48041FEF7FEFB237800205D
:10A210009B06A4F83C01F2D4A37AE3722046FFF730
:10A2200065FFEBE70720EAE70037002043788B4221
:10A230001DBF438823FA01F000F0010001207047A0
:10A2400029B1012303FA01F143881943418043787E
:10A2500013B99C30FEF7EABD704730B4C56843823D
:10A26000FF230374002A14BF13462B462B4043617F
:10A2700030BCFFF7E5BFF8B51F460378DB0705469E
:10A280000E4619D50121FFF7D1FFB8B902212846A2
:10A29000FFF7CCFF044688B9069B6B62002A18BF03
:10A2A000134628462F6208BF4FF4967332460121A9
:10A2B000FFF7D3FF2046F8BD0D20FCE70520FAE7A5
:10A2C000F8B51F460378DB0705460E4613D5012176
:10A2D000FFF7ACFF88B902212846FFF7A7FF044625
:10A2E00058B9069B6B62284613462F623246FFF729
:10A2F000B4FF2046F8BD0D20FCE70520FAE708B5BD
:10A300000378DB07024608D50421FFF78FFF20B949
:10A31000BDE808401046FFF793BF08BD08B50378B5
:10A32000DB07024608D50721FFF780FF20B9BDE80B
:10A3300008401046FFF784BF08BD38B50378DB0737
:10A3400004460D4609D5FBF7CEFC2844E061082100
:10A350002046BDE83840FFF773BF38BD38B50578F3
:10A36000EB07024610D50521FFF760FF50B953886F
:10A37000C3F3001383F0010363F341051570104626
:10A38000FFF75EFF002000E00D2038BD70B58CB0F7
:10A39000D0F8985005AE00244FF6FF7101233046E7
:10A3A000ADF826108DF82E308DF824400594ADF8C8
:10A3B000184001F06BFC07AB22462846CDE901446A
:10A3C0000096032101F0A6F80721284601F0BFFA04
:10A3D00028460CB070BD70B503468CB0D0F89850CC
:10A3E000996B406B05AE07AA002403C219898DF84A
:10A3F0002E40022230468DF824200594ADF81840F6
:10A4000001F040FC07AB224621462846CDE9014435
:10A4100000968DF82E4001F07DF8284601F0AAFA4A
:10A420004FF0FF3303700F2343708470C4702846CD
:10A430000CB070BD73B50B681B781A0705460C4647
:10A440001DD50DF10301204601F064F99DF803309C
:10A45000082B14D0102B14D05BBBE37E154EA660E6
:10A46000DB0705F1340506D43169204601F072F9A5
:10A470003369013333612946204601F0ECFA02B01A
:10A4800070BD4FF0FF33019305F5A073A360D5F8BD
:10A4900038110131C5F83811204601F05BF901A9E6
:10A4A000204601F070F9FF21204601F099F9024D94
:10A4B000E1E7FEE7188B0020E362070021B9D0F83E
:10A4C000E8300133C0F8E830837A93420DD1B0F818
:10A4D0003E31B3F5007F3CBF0133A0F83E31B0F808
:10A4E0003E2100F59E700AF0C7BE70472DE9FF417E
:10A4F0000B689DF828801F788B8800260446154637
:10A5000008468DF80C60E3B101A900F027FF2C4844
:10A51000012201A907F0200714F02CFE40B13FB141
:10A5200095B10E2D05D13146802226300AF0A4FEC9
:10A5300065B1B8F1000F09D0D4F8DC300133C4F8AC
:10A54000DC3004B0BDE8F0810121EDE7D4F8B03093
:10A550000B2D03F10103C4F8B0301DD1D4F8EC3059
:10A560000133C4F8EC30FFB1D4F8BC300133C4F887
:10A57000BC3025B9D4F8C0300133C4F8C0309DF8E0
:10A580000C10BDF80400FFF7A1FC98B1D4F8B83066
:10A590000133C4F8B830D4E70F2D02BFD4F8F0303F
:10A5A0000133C4F8F030DEE7D4F8C4300133C4F826
:10A5B000C430E4E7D4F8B4300133C4F8B430C0E7B1
:10A5C000EC8D00202DE9F74398460B681B781B079C
:10A5D00005460E46174604D40025284603B0BDE8BC
:10A5E000F0830DF10101304601F084F89DF801304F
:10A5F000052B01D00825F0E701A9304601F09AF8B3
:10A600000DF10201304601F085F89DF80240082C5A
:10A610003AD0102C00F08280002CEBD14348394610
:10A620000246304601F079FA05460028E2D19DF84D
:10A630000230082BD0D198F81E3003F00F03072BFF
:10A64000CAD1D8F818309C4208D0C8F8100001468A
:10A65000C8F8184008F10C0001F024FB019BD8F861
:10A66000142033480133934288BFC8F81430C8F827
:10A670000C30D0F8E8339C42AED90022214600F5D8
:10A6800076700AF005FDA8E7B8F1000FB2D00DF121
:10A690000301304601F08EF89DF80330244A013B57
:10A6A000DBB28DF80330D2F8E84304F07F02934226
:10A6B00019D1314605F1280001F0A6FA98F81E30AC
:10A6C00003F00F03072B0CD1D8F818309C4291D31C
:10A6D00007D1019AD8F80C30511C994223D09A42E4
:10A6E00088D339469CE704F1FF3909F07F02934291
:10A6F00007D14A46314605F1280001F089FA4C4657
:10A70000DCE7013404F07F0293427FF473AF22460A
:10A71000314605F1280001F07BFACFE7054905F540
:10A72000A07000247CE71D2557E700BF188B002090
:10A73000D8860020E362070070B588B000238DF84A
:10A7400010308DF81C3013681B781B0706460C462A
:10A75000154602D4002008B070BD104600F08CFDF4
:10A7600000F44050B0F5005F01D00820F3E7284620
:10A7700001F0AFF80028F8D16946284600F0BAFF8A
:10A780009DF80030052BF0D10DF10301284600F0B3
:10A79000C1FF9DF80330082BE7D10DF101012046E0
:10A7A00001F008F80DF10201284601F003F89DF8C8
:10A7B00001209DF802309A42D7D101A9284600F025
:10A7C000B9FF02A9284600F050FE9DF81030002B7A
:10A7D00039D0012202A92B4814F0CCFC04469DF884
:10A7E0001030022B4BD0002CBFD02068616802AB28
:10A7F00003C302238DF810309DF80230224A013B3A
:10A80000DBB28DF80230D2F8E82302F07F018B42F0
:10A8100024D106F16402A37F03F00F03072B03D1B9
:10A82000636901999942A0D302A9284601F075F9FC
:10A83000002890D1A37F03F00F03072B8AD1019B3F
:10A840000133636187E7204605A900F087FD9DF885
:10A850001C40002CC3D0012205A9BCE7511E01F009
:10A860007F018B4202D106F15402D4E7013202F09B
:10A870007F0293427FF479AF06F17402CBE7002C9C
:10A88000BAD172E7EC8D0020D886002038B50C468E
:10A8900091F8245092F9151004F122000AF091FD6C
:10A8A0000A4B93F8A926022A0ED103F5DC629442E2
:10A8B0000AD193F80437AB4206D0BDE838400448CB
:10A8C0004FF00041FEF7A0B838BD00BFD886002089
:10A8D0000037002037B50D4604460DF10701284624
:10A8E00001F00AF89DF80730042B15D0072B1ED174
:10A8F000D4F80C310133C4F80C31237813F0010083
:10A9000013D0C3F30015DB0604D520460321FFF75F
:10A9100097FC284603B030BDD4F804310748013312
:10A92000C4F8043129461BF081FF0120F2E7D4F876
:10A9300010310133C4F810310020EBE7488D0020BE
:10A9400010B50378044661F3C30303700948FBF7AD
:10A9500045FC23785A0704F12C00C3F3800158BF4B
:10A96000C3F3C00101F034FA2046BDE81040FFF700
:10A97000BDBB00BFD836002070B5C66805460A4882
:10A98000FBF780FF044650B9074807F06DF8B04266
:10A99000E8604FF48001054803D1FEF73EF82046F9
:10A9A00070BDFEF731F8FAE7D836002000370020F6
:10A9B0000148FBF75BBF00BFD836002007B52C303D
:10A9C000019101F0B3FA019903B05DF804EB0AF0CC
:10A9D000B3BC000070B508460D46144600F04CFCB0
:10A9E00000F44050B0F5005F2ED12B681B781B0798
:10A9F0002AD51A21284601F00CF8064620B3214634
:10AA00001248052208F04FFC0446E8B1B3889AB218
:10AA1000092A19D9F278A0F84830B37843EA02231A
:10AA2000A0F84A3090F8403043F0800380F840307E
:10AA3000FBF759F9D5E90223E064C4E9142304487B
:10AA4000BDE8704008F03ABE70BD00BFA08F002086
:10AA5000508D00202DE9F0431D460B6893F80080CF
:10AA60008B8885B004460E46174608F02008002B58
:10AA70003CD001A94FF0000930468DF80C9000F051
:10AA80006DFC9DF80C10BDF80400FFF71FFA70B1C3
:10AA9000A3790133DBB2A3713BB904F12C0001F0BF
:10AAA000AAFB002800F0A480FEE784F80690B8F125
:10AAB000000F1BD0D7B15048012201A914F05AFB56
:10AAC00081469DB93A4631462046FFF735FE054698
:10AAD000B0B9B9F1000F09D03A4649462046FFF710
:10AAE000D5FE01AA39462046FFF774FF6378013B83
:10AAF000072B07D8DFE803F0070614432106695C3B
:10AB00000E25F3E7FEE7D4F8D430618A013304F16F
:10AB1000A400C4F8D43005B0BDE8F043FEF73ABA5B
:10AB2000D4F8D0300133C4F8D0300023637020460D
:10AB300005B0BDE8F04300F0FFB8B38813B1B8F139
:10AB4000000F0DD06DB1D4F8CC302C480133C4F8CF
:10AB5000CC30002363702A463146FFF7EDF8E6E774
:10AB6000FEE7002FEFD02378DA07ECD53B681B789F
:10AB7000DB06E8D506212046FFF762FBE3E7D4F8C1
:10AB8000C8300133C4F8C83025B1D4F8E0300133FF
:10AB9000C4F8E030002363702A46314618480BF0B1
:10ABA0004BFF16482B463A463146FFF74FF8BEE7B3
:10ABB000D4F8C83013480133C4F8C8300023637098
:10ABC0002A46314608F050FEB1E7D4F8C8300133C8
:10ABD000C4F8C83025B1D4F8E4300133C4F8E43007
:10ABE0000023094863702A4631461BF045FF9EE763
:10ABF00005B0BDE8F08300BFEC8D0020608D002023
:10AC0000888C0020508D0020488D0020D0F898308E
:10AC100010B5DA7E0021C3E9041122F0170242F0D8
:10AC200004029980DA760278D107044670D542781A
:10AC3000013A00F19801072A05D8DFE802F005047F
:10AC40002A4938045463FEE704F12C004FF6FF71E3
:10AC500001F09EF82046FFF799FB002858D0237C8E
:10AC600083718376036800229A7004230376237E1F
:10AC70004376C37EDB0603D401462046FFF7DAFBAA
:10AC80000023A37104F12C0001F0B5FA002849D08B
:10AC9000FEE72046FFF79FFB002839D0E37A837157
:10ACA000837623795A1C227102689370DDE7E27A79
:10ACB0009A719A7604221A76227E1B485A76FFF7FA
:10ACC000C3F828B363795A1C627102689370D0E7A5
:10ACD000E27A9A719A7604221A76227E5A7613487C
:10ACE0000CF0A8FCEDE7E27A9A719A7604221A76C3
:10ACF000627E0F485A761BF0E1FD48B1C37E9A0789
:10AD0000B7D4DFE700221A830A4808F0EBFCF4E727
:10AD1000D4F89810002220468A80BDE810400B230A
:10AD2000FFF798BE10BD00BF608D0020888C00200A
:10AD3000488D0020508D002038B543780446002B04
:10AD400079D1037813F0010305D14380BDE8384081
:10AD5000A430FEF7D5B843885A061AD50623637087
:10AD60006278002A48D0012303FA02F2638804F1D2
:10AD7000A40523EA020363802846FEF7C1F863783E
:10AD8000082B58D8DFE803F0383D424747474C4787
:10AD90004700DD0507D5FAF7A6FFE369C01A0028CA
:10ADA00001DB0823DBE76388980701D50123D6E799
:10ADB000590701D50223D2E71A0701D50323CEE7AD
:10ADC0001D0601D50723CAE79806C3F34011C3F354
:10ADD00000120CD572B123789B070BD40423637047
:10ADE0000029BDD0237843F002032370B8E7002A7E
:10ADF000B6D0F3E70523B2E72046BDE83840FFF7B9
:10AE000075B92046BDE8384000F016B82046BDE8C8
:10AE1000384000F02AB82046BDE83840FFF7F6BEBB
:10AE2000E17A04F12C0001F00BF828466421BDE81A
:10AE30003840FEF7AFB838BD10B50446FFF796F8B6
:10AE400020B92046BDE81040FFF7E0BE218904F19B
:10AE50002C0000F09DFF002120466170FFF790F864
:10AE60002046BDE81040FFF767BF38B50446FFF73E
:10AE70007DF840B1236A0020607043BB2046BDE8E6
:10AE80003840FFF759BF638A04F12C0583B9217C50
:10AE9000284600F0D5FF284601F042F8014620463A
:10AEA000FFF785F82046FFF761F80028EFD0E1E7CB
:10AEB00023785B0703D4217C284600F0C1FF628A17
:10AEC000217C284601F084F80028D3D138BD616A7E
:10AED0009847D3E710B50446FFF769F82046BDE868
:10AEE0001040FFF7C2BF00004378012B10B50446A5
:10AEF00003D0062B05D073B1FEE7BDE81040FFF785
:10AF00009BBF002343700748FEF77EFE2046BDE846
:10AF10001040FFF711BF03785A0702D54388DB05BD
:10AF2000F5D410BD608D00200148FFF7DDBF00BFE4
:10AF3000388B00200148FFF7FFBE00BF388B002090
:10AF4000F0B589B000238DF810308DF81C30D0F8A2
:10AF5000F430013304460E46C0F8F4301746002A98
:10AF600040F0B180002900F05D810378DD0740F1F9
:10AF70007981084600F0ADFC0746002840F0A38028
:10AF800002A9304600F071FA05A9304600F0E6F952
:10AF90009DF810502DB1AC48012202A914F0EAF836
:10AFA00005469DF81C10012900F09F80022900F041
:10AFB000C2800DF10601304600F0BAF948B9BDF87B
:10AFC00006304FF6FF72934203D022899A4240F036
:10AFD000BB809DF81030012B00F0BC80022B00F0EC
:10AFE000C2809DF81C10BDF81400FEF76FFF00280A
:10AFF00000F0C980D4F8FC300133C4F8FC302B4693
:10B0000002AA31462046FFF7DDFA074628B11D287F
:10B0100059D16378062B40F01F813146204602AAA1
:10B02000FFF7D8FC89483146FEF702FE95B3294662
:10B0300032462046FFF72AFC33681B78190729D5CA
:10B040000DF10501304600F065FB9DF80530082B39
:10B0500020D1AB7F03F00F03062B04D0072B08D0C1
:10B06000012B40F0E580304600F05AFC002800F04B
:10B07000F98033681B7803F00703012B0AD1AB7FFB
:10B08000DA0907D11A0705D02B8C022B02D9FAF75F
:10B090002AFEA8606378022B7BD0062B00F0838009
:10B0A000012B40F08E8033681B785B0771D1D4F898
:10B0B00008310133C4F8083131462046FEF760FFFD
:10B0C000002F00F09B80A7F10800152800F2CA802D
:10B0D000DFE800F09CC8C8C8C8C8C8C8C8A2A8AEE5
:10B0E00053B43AC8C8C8C8C8C8C22378BDF8142029
:10B0F000580705D51046FEF7E9FE002840F0B88055
:10B10000638E934220D1002D7FF453AF012110466E
:10B11000FEF7DCFE00283FF44CAF4D4890F8AA56ED
:10B1200015F002053FF445AF02A900F2147014F0C7
:10B1300087F805463DE7082204F1340105A85DF0D3
:10B14000F7FA00283FF435AFD4F818310133C4F8CA
:10B15000183153E0002D6BD02868696802AB03C337
:10B1600002238DF81030082204F134010DEB0200A7
:10B170005DF0DEFA00287FF434AFD4F828310133D3
:10B18000C4F828313AE0D4F8F8300133C4F8F83084
:10B1900035E7227CA37A9A4213D0D4F810310133D8
:10B1A000C4F810318CE79DF81C3043B104F1A400C1
:10B1B000FDF7A6FE002363702046FFF7BDFD002FBC
:10B1C00081D133681B7803F00703012B18D0032BC0
:10B1D0000ED0002BE1D1D4F808310133C4F8083186
:10B1E0001C4831460BF0E4FF2046FEF77FFF67E77F
:10B1F00031462046FFF76EFB0028F1D009B0F0BDC4
:10B20000D4F800310133C4F80031E9E7D4F82C3127
:10B210000133C4F82C31F1E7D4F830310133C4F8EC
:10B220003031EBE7D4F820310133C4F82031E5E7C1
:10B23000D4F824310133C4F82431DFE7D4F81431D1
:10B240000133C4F81431D9E7EC8D0020608D002063
:10B25000D8860020888C0020D4F81C310133C4F833
:10B260001C31CBE7D4F834310133C4F83431C5E7AD
:10B27000002D7FF49EAE50E703681888704708B52C
:10B28000FFF7FAFF00F44050A0F500535842584130
:10B2900008BD0268137819B143F02003137070479A
:10B2A00023F02003FAE70268137819B143F0100382
:10B2B0001370704723F01003FAE700F44053B3F51E
:10B2C000005F1ED120F44E5323F03F0348F24002AA
:10B2D00093421CD00CD8B3F5446F18D005D8B3B145
:10B2E000B3F5046018BF01207047B3F50040F9E7DB
:10B2F0004CF6404293420AD000F44C40B0F5404036
:10B30000F0E710F4406F14BF0120002070470020C8
:10B31000704708B5FFF7B0FFBDE80840FFF7CDBFA5
:10B3200008B5FFF7F6FF002814BF0320FF2008BD73
:10B3300038B505460C46FFF7F3FFFF281FBF2B6803
:10B340001B5A2380002008BF062038BD08B5FFF730
:10B35000E0FF002814BF0520032008BD38B50C46C7
:10B360000546FFF7F3FFFF2801461CD02846FFF7EC
:10B3700083FF00F44060B0F5006F05D0B0F5406F7A
:10B3800009D00020207205E02B685B5A238001233E
:10B390002372002038BD2B6801221944204600F09A
:10B3A0005EFC0223F4E70620F4E710F4404218BFE5
:10B3B00080F0400200F4405318BFC2F38012B3F58E
:10B3C000005F05D100F44C43B3F54C4F08BF002299
:10B3D0001046704708B5FFF74FFF0146FFF7E5FF3E
:10B3E000A0B10846FFF769FF01F4406100280CBFD7
:10B3F00003200520B1F5006F03D0B1F5406F03D0F5
:10B4000008BD0230C0B2FBE70830FBE7FF20F7E7DA
:10B4100038B505460C46FFF7DDFFFF281FBF2B6838
:10B420001B5A2380002008BF062038BD10B5FFF747
:10B4300023FF0446FFF741FF04F4406300280CBFDC
:10B4400003210521B3F5006F0AD0B3F5406F0AD090
:10B450002046FFF7AAFF08B10231C9B2084610BD65
:10B460000231C9B2F4E70831FBE738B505460C46AE
:10B47000FFF7DCFF01462846FFF7FEFEFF2908D054
:10B4800000F44040B0F5004F05D0B0F5404F09D072
:10B4900080B1062005E02B685B5A238001232372CC
:10B4A000002038BD2B6801221944204600F0D7FB4C
:10B4B0000223F4E72072F4E7102804D0182814BF00
:10B4C0000020082070470420704700F00700013872
:10B4D00006280BD8DFE800F00406080A0406080076
:10B4E00004207047082070471020704700207047E4
:10B4F000430708D000F01803083BDBB2102B04D838
:10B50000034AD05C7047FF2070470520704700BF9A
:10B51000FB6207002DE9F7431F461B7ADDF82890F0
:10B520009DF82C60012B0546884641EA020424D090
:10B53000022B25D0B97C012925D002292ED0B8F1C3
:10B54000020F04BF24F02004A4B2002E14BF082070
:10B5500000200443B2F5805FA4B203D0B2F5005FCF
:10B5600020D03ABB33B329B3B9F80020B9F8023080
:10B570009A421FD144F040041CE044F40044D9E74F
:10B5800044F44044D6E778894FF6FF7C604514BF09
:10B5900020200020044344F40064D0E744F44264D3
:10B5A000A4B2CCE7002956D199F80520002B4BD145
:10B5B000002ADFD17F22296868461AF0BFF92146A8
:10B5C00068461AF0EAF9002168461AF0CFF92046D9
:10B5D000FFF773FE20B1B9F8021068461AF0DDF9E2
:10B5E00007F10A0168461AF0E3F92046FFF7DDFE8D
:10B5F00020B1B9F8001068461AF0CFF9394668460C
:10B600001AF0D6F9BDF80430AB808EB19DF8301039
:10B610000E43314668461AF0A9F93046FFF768FF35
:10B6200002463046FFF751FF1044AA881044A88014
:10B63000B8F1030F02BFAB880133AB80AB88023394
:10B64000AB8003B0BDE8F083002AB3D199F8043091
:10B65000002BAFD18EE713B999F80530F8E7022B2C
:10B6600082D1022980D1F7E710B50446FFF725FE05
:10B6700004F4406300280CBF03210521B3F5006FDB
:10B6800006D0B3F5406F17D023B1FF21084610BD97
:10B690000231C9B22046FFF788FE08B10231C9B2B3
:10B6A00004F44044B4F5004F08D0B4F5404F08D03E
:10B6B000002C18BFFF21E9E70831EAE70231C9B2DF
:10B6C000E4E70831FBE708B58388042B05D9FFF7C9
:10B6D000D3FDBDE80840FFF7C7BFFF2008BD828843
:10B6E000022A05D903681B781B0701D5FFF7EBBFBA
:10B6F000FF20704738B505460C46FFF7F0FFFF28DE
:10B700001FBF2B681B5C03F00703237014BF0020CE
:10B71000062038BD38B505460C46FFF7E0FFFF2888
:10B720001FBF2B681B5C03F01803237014BF00209D
:10B73000062038BD38B505460C46FFF7D0FFFF2878
:10B740001FBF431C2A68DBB200201ABFD3582360F6
:10B75000062038BD38B505460C46FFF7C0FFFF2868
:10B7600000D1FEE72A68431CD9B252FA83F354543D
:10B77000220A5A70220C240E9A70DC70EB7E43F081
:10B780000103EB7638BD38B505460C46FFF7A7FF39
:10B79000FF28034600D1FEE72D68285C00F0180062
:10B7A000FFF78AFE053302462146E818BDE8384017
:10B7B0005CF0F0BF38B505460C46FFF790FFFF2858
:10B7C00002460BD02B68185C00F01800FFF774FEDF
:10B7D0001344034400205B79237038BD0620FCE746
:10B7E00038B505460C46FFF77AFFFF28024600D120
:10B7F000FEE72B68185C00F01800FFF75DFE1344AD
:10B8000003445C7138BD10B50446FFF768FFFF289C
:10B8100006D02368185CFFF758FE0230C0B210BD96
:10B820000220FCE710B50446FFF74DFFFF28014654
:10B8300010D023681A7812070CD5A488A0420BDA1E
:10B84000185CFFF755FEFF2808D00144C9B28C42AE
:10B85000B8BFFF21084610BDFF21FBE70146F9E70D
:10B86000F8B50546FFF7DEFF84B2FF2C2DD0284641
:10B87000FFF702FD830506461DD52846FFF7C3FFE7
:10B880002F68A988A21C93B210FA82F28A4207EBB1
:10B89000040C1CDC3A5D02F07F0213449CB210FAE7
:10B8A00083F3994213DBBCF80020C2F3C7127F2A4E
:10B8B00001D09942E6D12846FFF7E1FC28B906F00D
:10B8C0000706032E01D10134A4B2E0B2F8BDFF2473
:10B8D000FBE738B50546FFF7C3FFFF28044609D04C
:10B8E0002846FFF790FF0444A8888442CCBF062076
:10B8F000002038BD0620FCE7F8B505460E46FFF7E8
:10B90000AFFFFF28044609D028462F68FFF7B7FC91
:10B9100000B9013C3B5D33700020F8BD0620FCE718
:10B9200007B503681B7803F00703032B03D000203F
:10B9300003B05DF804FB0DF10701FFF7DDFF002800
:10B94000F5D19DF80700031F58425841F0E7F8B5BC
:10B9500005460E46FFF784FFFF28044608D0284618
:10B960002F68FFF78CFC00B9013C3E550020F8BD64
:10B970000620FCE710B50446FFF772FFFF2816BF4C
:10B9800023680020C01810BD10B50446FFF7F2FF71
:10B990002368C01AC0B210BD38B50546FFF7F4FFE2
:10B9A00004462846FFF72FFF2044C0F17F0080B2F5
:10B9B00038BD38B50546FFF7E7FF04462846FFF7D0
:10B9C00022FF0444A888001B80B238BD70B506462B
:10B9D0000C46FFF7D9FF05463046FFF714FF054434
:10B9E0002C44B48070BD10B50446FFF70CFFA3884B
:10B9F000181A2368184410BD08B50246FFF73CFC2E
:10BA0000830504D5BDE808401046FFF70BBFFF20B3
:10BA100008BD70B506460D46FFF7EEFF04463046FA
:10BA2000FFF71EFFFF2C024613D0FF2811D0ADB246
:10BA300094420ED83368195BC1F3C7118D4203EBF2
:10BA4000040007D01B5D03F07F0302331C44E4B203
:10BA5000EEE7002070BDF0B50446E5B000230AA86B
:10BA600005930D461AF00AFE23681B781B074FD575
:10BA70000DF113012046FFF73DFE002848D105A92E
:10BA80002046FFF757FE0646002841D106AF9DF835
:10BA9000132005993B4628461AF0E2FDA1680AA842
:10BAA0001AF01CFC2046FFF7AEFE05462046FFF7C5
:10BAB0006BFF03902046FFF77CFF023D0D230246FB
:10BAC0000399CDE900730AA8EBB21AF013FC2046E3
:10BAD000FFF75AFF216802460AA81AF0AFFC204679
:10BAE000FFF748FF03902046FFF763FF039A009695
:10BAF000034611460AA81AF0E5FC2046FFF773FF3B
:10BB000001460AA81AF08FFDE37E43F01003E376A6
:10BB10000AA81AF0CDFD65B0F0BDF0B50446E9B055
:10BB200000230EA805930E4615461AF0A7FD2368BC
:10BB30001B781B0706D400240EA81AF0B9FD204676
:10BB400069B0F0BD0DF113012046FFF7D3FD0028C9
:10BB50004BD105A92046FFF7EDFD002845D106AFE2
:10BB60009DF8132005993B4630461AF079FD294689
:10BB70000EA81AF0B3FB2046FFF745FE0238C5B207
:10BB80002046FFF701FF03902046FFF712FF0D2329
:10BB900002460399CDE900730EA82B461AF0AAFBC2
:10BBA0002046FFF7F1FE216802460EA81AF046FC77
:10BBB0002046FFF7DFFE03902046FFF7FAFE039AC8
:10BBC0000121034600910EA811461AF07BFC0AA938
:10BBD0000EA81AF028FD2046FFF705FF2A46014669
:10BBE0000AA85CF0A5FD0028A5D00824A4E738B574
:10BBF0000D4605F5A0450446043000F095F8D5F84B
:10BC0000A4342367204638BD004870479C8B002031
:10BC10000748D0F8E833591E914203D001339342CC
:10BC200003D0FEE700F2B440704700F2D440704702
:10BC3000D886002010B54FF6FF74FCF78FFF80B256
:10BC4000A042FAD010BD10B504460821FDF784FBD0
:10BC5000237823F0010343F00203237010BD12B1D7
:10BC6000012A05D070470B6803604B68436070473A
:10BC700001F10803013813F8012D00F8012F8B4260
:10BC8000F9D170470123018003717047012341807E
:10BC90004371704740F201130180418083807047F7
:10BCA0000068704701607047102200215CF088BE78
:10BCB00030B50B46024601F1100518685968144664
:10BCC00003C40833AB422246F7D130BD10230860CD
:10BCD0008B80704738B54FF6FE73C380038A03F03C
:10BCE000FE0343F4FE43002543F0010304460382B0
:10BCF000458005718560C560456180F85D502830DC
:10BD0000FFF7D2FF04F13800FFF7CEFF04F148003F
:10BD1000FFF7CAFFA56584F85C5004F16000BDE838
:10BD20003840FDF797B9000037B5174D019104462B
:10BD30002846FAF74FFA20802846FAF737FA019991
:10BD4000A06104F11C0000F079FB0021C4E9081196
:10BD5000102204F128005CF033FE1022002104F1CF
:10BD600038005CF02DFE0021102204F148005CF048
:10BD700027FE2346054A43F8602F2046A366FFF7B7
:10BD8000A9FF204603B030BDD8360020C1C3000053
:10BD90000148FAF7F9B800BFD8360020C180014841
:10BDA00005F02CBEEA36002013B500F108030C465E
:10BDB00008684968012203C321466846FFF74FFF20
:10BDC0000248694605F014FE02B010BDEA360020B4
:10BDD000037C61F3000303740388DB0502D502488A
:10BDE00005F052BE704700BFD8360020837810B5EA
:10BDF000044663B90748FAF74FF950B90548FAF70E
:10BE00006BF930B9A378012B01D00123A370002076
:10BE100010BDFEE7D836002010B504466030FDF7AF
:10BE200019F90648FAF758F930B90448FAF73EF913
:10BE300010B9A37803B1A07010BD00BFD8360020A0
:10BE400010B504460448FAF7E5FC20B9A378022BA4
:10BE50001CBF0223A37010BDD836002038B50123C3
:10BE6000044603FA01F10020FCF7A6FE237C4FF400
:10BE7000A075DB0700FB05F50BD5A3690748997989
:10BE8000FAF7C8FC294604F16000BDE83840FDF728
:10BE9000D3B80248FAF720F9F4E700BFD8360020FB
:10BEA000837803F0FB03032B10B5044625D10388E8
:10BEB000DB0606D4836911489979FAF7ABFC00B127
:10BEC000FEE7A378042B1CBF0423A370236A1BB1D5
:10BED000626AA06901219847A169094805F094FDAB
:10BEE0000D2808D1A1694B6933B10023C1E904339E
:10BEF000034805F089FD00B1FEE710BDD8360020EB
:10BF0000EA3600200388DA0708D40B681B789B0602
:10BF100004D54FF47A516030FDF78EB870470000B9
:10BF20000148FAF747B900BFD83600200148FAF7B0
:10BF3000E5BB00BFD83600208378022B1CBF02234C
:10BF400083701C3000F096BA03889B0710B5044636
:10BF500000D5FEE71048FAF72DF97F2806D094F9AE
:10BF600011307F2B01D0984200DD6074F9F7BBFEE1
:10BF70006369C01A002808DA616E04F160004FF4AA
:10BF8000FA32BDE81040FDF751B894F9111020467F
:10BF9000BDE81040FFF7D0BFD8360020008880F001
:10BFA0002000C0F340107047008800F00C00B0FA89
:10BFB00080F040097047008880F00400C0F38000E2
:10BFC0007047008880F00200C0F340007047000016
:10BFD000837870B50446164653B3033B042B27D928
:10BFE00003889B0709D51448FAF73AF9A378052B7B
:10BFF00001D00523A370002518E0FFF7E2FFC8B1C8
:10C000000D48FAF707FC054600B1FEE7A378052BBB
:10C010001CBF0523A3707F236374F9F764FE3044CB
:10C020006061002104F16000FDF706F8284670BD4C
:10C030000D25FBE70C25F9E7D8360020008880F0B5
:10C040004000C0F38010704782698378526910B550
:10C050000446F2B1072B1CBF07238370FFF7EEFFE6
:10C0600090B11548FAF76EFBA369D3E904128B1857
:10C07000C3F5A473C34207D504F16000A1F5A47110
:10C08000BDE81040FCF7D2BF2046BDE81040FFF7E6
:10C0900007BF032B1CBF03238370C178FFF784FF06
:10C0A0000028F1D00331C9B20529204628BF052157
:10C0B000BDE81040FFF7D2BED8360020037C024610
:10C0C00013F0010002BF108880F48070C0F30020DC
:10C0D0007047000010B50446FFF7F0FF20B9A378C1
:10C0E000012B07D1002004E00448F9F7F5FF0028F0
:10C0F000F5D010BD0123A370F4E700BFD8360020AF
:10C100002DE9FF470829DDE90C8905460F469246CF
:10C110001C4603D011F0EF0F13D0FEE780F85C202F
:10C1200000F128060FCB86E80F0098E80F0005F114
:10C13000380686E80F0099E80F0005F1480686E802
:10C140000F002846FFF72AFF48B9CDE90190CDF846
:10C1500000800448234652463946FAF7F5FA04B0FF
:10C16000BDE8F087D836002038B590F85C309342AF
:10C1700004460D4607D11C3000F082F9A36D9D42A4
:10C1800024BF0135A56538BD1FB504468069036825
:10C190001B781B072DD5C37ED9062AD40DF10F01BC
:10C1A000FFF7B8FA28BBA069C37EDA0703D494F876
:10C1B0005C10FFF715FB2046FFF7F0FEC8B19DF8B5
:10C1C0000F30082B15D1A06904F138038360C37EBA
:10C1D000DB0709D4A16D0191FFF7BCFA94F85C204C
:10C1E00001992046FFF7C0FFA06904F10801FFF79D
:10C1F00032FC04B010BD38B58378052B05460BD052
:10C200000024FFF7C1FF2846EC702C7185F85D40D3
:10C21000FFF71AFF204638BD0D20FCE737B505466D
:10C220000C46FFF7BBFE20BB0B681B781A0720D516
:10C23000CB7EDB071DD50DF102012046FFF76AFA20
:10C2400000B1FEE79DF80230082B12D101A920466B
:10C25000FFF770FA00B1FEE70DF103012046FFF78A
:10C26000A9FA00B1FEE79DF8032001992846FFF7DF
:10C270007BFF03B030BD2DE9FF411E460446603010
:10C280000D469046FCF7E6FE0E2E25D003D81EB3D1
:10C290000B2E23D0FEE70F2EFCD10027EB7E5B0791
:10C2A00005D5AA79394604F11C0000F0CFF82946DB
:10C2B0002046FFF7B3FF9FB92046FFF775FE78B120
:10C2C000E3782A7E9A420BD90133E370204604B00A
:10C2D000BDE8F041FFF7B8BE0127DFE70127E6E739
:10C2E0000023E3702379002E32D02046FFF763FE4F
:10C2F000074620B16F7E9F4294BF0027012704F1BB
:10C300001C00009732462946039000F0A5F80398D8
:10C3100007B3237901332371EB7E0E2E43F0020322
:10C32000EB76D3D1A37894F85D10062B1CBF0623BF
:10C33000A3702046FFF792FD94F85D300133DBB225
:10C34000052B28BF052384F85D3004B0BDE8F081DB
:10C350003746D4E7A378022B1CBF0223A3704246C2
:10C360003346294604B0BDE8F04100F07DB8000036
:10C370008378033B10B50446042B1DD8DFE803F097
:10C38000030718140300BDE81040FFF789BD836957
:10C390000A489979FAF73EFAA16920460E23BDE8CA
:10C3A00010400022FFF767BFBDE81040FFF74CBE0A
:10C3B000BDE81040FFF7C8BD10BD00BFD836002053
:10C3C0000148FFF7D5BF00BF648B0020036A70B53A
:10C3D00005460C4616462BB121B11AB9426A3146C0
:10C3E000204698472846FFF7D9FD40B93CB1E37D88
:10C3F0009B0704D5227D21692846FFF7B5FE32460A
:10C40000214605F11C00BDE8704000F019B800009D
:10C4100008B512B1836D8B4200D28165FFF7BEFD76
:10C4200048B905481AB1BDE80840FAF7C1B9BDE8F6
:10C430000840FAF7AFB908BDD836002070470000B1
:10C440000148FEF77DBD00BF388B00200148FEF794
:10C4500035B800BF388B00209DF8000000900148DF
:10C46000FEF744B8388B00200148FEF7F3BA00BF4E
:10C47000388B00200148FEF72DBD00BF388B00200F
:10C48000014808F06DBD00BFB08A002030B501F54D
:10C49000A04185B004462B48D1F86C5405F0E8FA69
:10C4A000284008BF284600210390782204F10800A4
:10C4B0005CF086FA01220023C4E9002303A81AF0E5
:10C4C0004CF92567A4F85A00FFF7B4FBA4F858000C
:10C4D00004F16C0008F0DBFB102104F12000FCF7F4
:10C4E0003BFF054658BB102104F15C00FCF734FF0C
:10C4F000054620BB082104F14100FCF72DFF05464D
:10C50000E8B904F1490002F0C1FE0546B8B9B4F833
:10C5100058300D4A009311210C4B04F130005CF0AF
:10C520000BFF012340F2011284F8743084F87B3051
:10C530004FF00133A4F87620A4F87820E36728466A
:10C5400005B030BDD8360020176307000C63070024
:10C5500010B500210446C0F80011A0F80411FE2215
:10C560005CF02EFA204610BD38B5B0F804510446F0
:10C570000544AC4217D26378FF2B01D1002038BDAF
:10C58000A31C9D42FAD3204619F002FC20448542A8
:10C59000F4D3204601F03CFE0028EFD0204619F0ED
:10C5A000F7FB0444E5E70120E9E70A46B0F8041187
:10C5B00019F0AEBD2DE9F3410C460746802200215B
:10C5C00020465CF0FDF93D46012604F11008B7F85D
:10C5D00004313B449D4280F093802B780E2B0BD886
:10C5E0000E2B0FD8DFE803F01A66345A744A0E3F58
:10C5F0000E0E0E0E840E1300342B22D0352B15D0C8
:10C60000332B5ED0284619F0C3FB0544DFE72146F3
:10C61000A81C01F003FF84F87460F3E7B5F8033059
:10C6200084F87C605BBAA4F85A30EBE76946284688
:10C6300001F0D4FD0028E5D1009B236784F87F60DA
:10C64000E0E7D5F8023084F87A601BBA6365D9E771
:10C65000D5F80230C4F84130D5F80630C4F845307A
:10C6600084F87860CEE7D5F80230C4F84930D5F8C0
:10C670000630C4F84D3084F87960C3E7AB1C04F190
:10C68000200C05F1120E18685968624603C208337F
:10C6900073459446F7D184F87660B3E72946684637
:10C6A00001F0F9FC694604F1300001F038FE84F82D
:10C6B0007760A7E76B8884F87B605BBAA4F8583092
:10C6C000A0E74146A81C01F0A9FE84F8756099E72F
:10C6D000AB1C04F15C0C05F1120E18685968624637
:10C6E00003C2083373459446F7D184F87D6089E727
:10C6F000284601F001FD84F87E600090E06681E745
:10C7000002B0BDE8F0810B46B0F8042110B5014637
:10C71000044618465CF03EF8B4F8042180F8FE2088
:10C7200010BD91F8FE20A0F804215CF033B838B5B4
:10C7300015460C4669B90E21FFF737FF10B91724CB
:10C74000204638BDD0F802302B60D0F806306B6040
:10C75000F6E73321FFF729FF0028F0D0D0F80230A8
:10C760002B60D0F806306B600024E9E7FE2B70B533
:10C7700004461E460846114602D90625284670BDC5
:10C780002246FBF782FD05460028F6D1A4F8046195
:10C790002046FFF7E9FE0028EFD0F9F7A4FAC4F825
:10C7A0000001EBE7B0F80431F7B505460F46164631
:10C7B000002B3DD000290CBF182219228DF804202F
:10C7C0000A3B022201A930468DF80530FBF7AFFD88
:10C7D00038BB2C46B5F804312B449C4228D2237830
:10C7E00037B90E2B08D1204619F0D2FA0444F1E7EC
:10C7F000012F01D1332BF5E7342B14D1F9F773FA5C
:10C80000D5F80031D4F80220C11A12BA91423ABFC9
:10C810009B181A1A00223421304619F06AFC0028AD
:10C82000E1D003B0F0BD3146204619F0C4FAF6E776
:10C830000020F6E738B50446084679B14D78B4F8DB
:10C84000042102350B1B55FA83F3D21A29445CF0FC
:10C850003BF8B4F804315D1BA4F8045138BD2DE950
:10C86000F843B0F804518846044617461E46FFF7C1
:10C870009CFEC5F1FE05ADB2014618B14378023306
:10C880001D44ADB206F10209A94518D82046FFF7AC
:10C89000D1FFB4F80431E0189944A4F8049104F8E5
:10C8A0000380467019F07EFA324639465BF072FF1B
:10C8B000F9F719FAC4F800010020BDE8F883032055
:10C8C000FBE737B50C46054609780191204619F07B
:10C8D00070FA637801990246284603B0BDE83040FB
:10C8E000FFF7BDBF91F8743037B505460C4643B12C
:10C8F000684601F0A3FD08236A460E212846FFF78B
:10C90000AEFF94F8753053B104F11001684601F0A0
:10C9100095FD08236A4633212846FFF7A0FF94F8C7
:10C920007A3043B1636D1BBA00936A460423342105
:10C930002846FFF794FF94F87C3053B1B4F85A10AE
:10C94000684611F0DEFE03236A4600212846FFF701
:10C9500086FF94F87F3053B1216F684601F098FC50
:10C960009DF806306A4635212846FFF778FF94F88F
:10C97000783033B1082304F1410202212846FFF741
:10C980006EFF94F8793033B1082304F1490207218E
:10C990002846FFF764FF94F8763033B1102304F192
:10C9A000200205212846FFF75AFF94F877305BB143
:10C9B00004F13001684601F0A7FC9DF80430009AAC
:10C9C00003212846FFF74BFF94F87B3053B1B4F8AE
:10C9D00058305BBAADF800306A4602230121284680
:10C9E000FFF73DFF94F87D3033B1102304F15C0272
:10C9F00004212846FFF733FF94F87E3073B10C23EF
:10CA00008DF8003004F16C01042368468DF8013084
:10CA100001F08FFB69462846FFF753FFF9F763F9EA
:10CA2000C5F80001002003B030BD082311B90E2164
:10CA3000FFF715BF3321FBE710B50446FFF7B5FD3F
:10CA400001462046BDE81040FFF7F4BE2DE9F04F47
:10CA500001F5A84985B001F5A74680460D46174661
:10CA600009F160095836FFF77FFD002867D00FB144
:10CA700000233B7005F5AD4A44460AF1280AB8F890
:10CA8000043143449C425CD223780C2B19D8DFE854
:10CA900003F007121D24432F1848181818184D00CA
:10CAA000B4F8031049BAC9B24846FDF797FB40B144
:10CAB00005B0BDE8F08F618849BA89B24846FDF7F4
:10CAC00087FA204619F064F90444D8E705F5A74031
:10CAD000A11C283000F0C8FDF3E72146684601F0AC
:10CAE000DAFA05F5A7406946303001F069FCE8E75D
:10CAF0006946304608F067FA04F1020B3FB1102294
:10CB0000694658465BF014FE08B101233B70594654
:10CB1000304608F047FBD4E7A11C304608F064F922
:10CB2000CFE7A11C50460DF009FDCAE7204601F0F1
:10CB3000E3FA69460090304608F000FBC1E70620A2
:10CB4000B6E70020B4E710B533210446FFF774FFC1
:10CB500020463421BDE81040FFF76EBF0273427BD0
:10CB6000002122F00302816042730160416070473E
:10CB700010B5017B0446054818F0FCFF0023236034
:10CB80006360637B23F00303637310BD38370020B9
:10CB9000F8B50A4604460D46017B1A4818F0CCFF4A
:10CBA000074620B10023A5F804313846F8BD237BA1
:10CBB00063B933212846FFF73FFF34212846FFF7AA
:10CBC0003BFFF9F790F8C5F80001EEE7342128465D
:10CBD000FFF7EBFC06460028E7D0F9F784F8A468D5
:10CBE000D6F80230021B1BBA9A423ABFE418231A45
:10CBF0003B461A0EB2701A0CF2701A0A3271737137
:10CC0000DFE700BF38370020437B6FF3000370B5C8
:10CC1000437304460E46FFF7BBFF054678B9637BB6
:10CC2000217B43F00203637322463046FFF77FFD0A
:10CC3000627BB0FA80F35B0963F3000262732846FB
:10CC400070BD30B5C3B004460D466846FFF780FCA2
:10CC5000FF22002128465BF0B3FE20466946FFF71D
:10CC600097FF044618B929466846FFF74CFD204651
:10CC700043B030BD70B50D460446B5F80461017B84
:10CC8000BEB9114818F076FF637B66F34103217B40
:10CC9000637322462846FFF74AFD637BB0FA80F0B3
:10CCA000400960F300036373F9F71DF8A0600020EA
:10CCB00070BD05482A4618F033FF0028F8D1637B81
:10CCC00043F00203E3E700BF3837002010B5C4B0DB
:10CCD000044602A80191FFF73BFC019902A8FFF767
:10CCE00020FD02A92046FFF7C5FF44B010BD38B5AE
:10CCF000044604301D46FFF731FF237F224623F010
:10CD00000303237742F8205F0023C4E90B33A262B8
:10CD10006361A361204638BD037F13F0010314BF94
:10CD2000143018467047000010B5C2B0044668467B
:10CD3000FFF70EFC6946201DFFF72AFF20B90246C7
:10CD400002496846FFF782FE42B010BDD836002087
:10CD5000037C0448002B0CBF4FF080514FF0005172
:10CD6000FBF752BE0037002030B5C3B0044668461A
:10CD7000FFF7EEFB04F12000FCF7C2F8237F6FF30E
:10CD8000000323776946201DFFF73EFF0546B0B933
:10CD9000217C04F114026846FFF7C9FC237FB0FA36
:10CDA00080F0400960F300032377237C23B9054911
:10CDB0002A466846FFF74AFE2046FFF7C9FF284685
:10CDC00043B030BDD8360020FFF7CEBF73B50D4657
:10CDD00000F11406017C04460023324628468DF8F3
:10CDE0000730FFF7A4FCF8B1237F13F0010F08BF51
:10CDF0000026637C13F001030CBF1946211D304649
:10CE000001F060FB9DF807300BB900281DDD2946B5
:10CE1000201DFFF72FFFB0B9104813F019FA204674
:10CE2000FFF796FF00200EE0237F43F001032377F6
:10CE3000237C002BDDD10A490DF107022846FFF7BC
:10CE400005FE0028D0D002B070BDE8D041F2883194
:10CE500004F12000FCF79EF8E1E700BF5CB400207D
:10CE6000D836002010B5027F002363F30002044689
:10CE70004361836102770430FFF77AFE04F12000FA
:10CE8000FCF73EF82046BDE81040FFF761BF000008
:10CE900030B5C5B0044602A80D46FFF759FB201D6A
:10CEA00002A9FFF775FE044680B9352102A8FFF7F5
:10CEB0007CFB50B101A901F091F938B9054A019BF9
:10CEC000D2F86C2413402B6003B91724204645B0D8
:10CED00030BD00BFD886002030B5ADF5137D0446C7
:10CEE0002622002104A85BF06BFD4FF2BF030EA8C1
:10CEF000ADF83230FFF72CFB207F83074FD4314B46
:10CF000093F8A936023B012B49D8617C10F001004F
:10CF100018BF04F1140011F0010118BF211D01F028
:10CF2000D1FA00283BDA257C75B950A8FFF710FB31
:10CF300050A92548FFF72CFE02AA294650A8FFF762
:10CF4000F6FB10B3237C6BB31B21204817F026FCA3
:10CF5000054658B30EA9201DFFF71AFEBDF83C2167
:10CF60000EA92846FBF7E3F9F0B904A816F054FB24
:10CF7000174B1648009404AA294618F087F898B968
:10CF8000237F43F00203237709E0617C11F0010164
:10CF900018BF211D02A801F095FA0028D2D10DF585
:10CFA000137D30BD0C21D0E7032807D141F2883131
:10CFB00004F12000FBF7EEFF002DF0D02846FBF730
:10CFC000A6F8ECE7D8860020448A0020FC880020E0
:10CFD0009BD000000E4B93F8A936032B10B50446E6
:10CFE00007D8012B10D863B12046BDE81040FFF7E9
:10CFF000AFBE042BF8D1FFF7B7FE064813F028F9AF
:10D00000F2E7FFF7B1FEEFE7FFF766FFECE700BFDF
:10D01000D88600205CB4002038B505460430FFF700
:10D0200055FE044610B92846FFF7D4FF204638BD08
:10D030000148FFF751BF00BF0C8A00200148FFF7ED
:10D040004BBF00BF408A002013B5002204468DF874
:10D050000720084663B90DF10702102118F0B8FF48
:10D060000346C0B99DF80720AAB1FF2A08BF2523AF
:10D07000227F6FF341022277E26A22B10021E1624E
:10D080001846216B904741F2883104F12000FBF7EC
:10D0900081FF02B010BD0623EAE7FFF7D5BF00000D
:10D0A0002DE9F041C2B0804668460C4617461D4641
:10D0B0009DF82061FFF74CFA694608F10400FFF77C
:10D0C00067FD2146234817F0A6FB0446A0B3E6B946
:10D0D000214E6D46BDF804316B449D4225D22B781C
:10D0E000052B08D196F85634DA0704D4284618F0F0
:10D0F0004FFE0544EEE72146284618F05CFE002866
:10D10000F4D02046FBF703F816E0013E05F1FF38A6
:10D1100055FA86F5104E18F8011F05290FD196F81B
:10D120005634DB070BD4A845F5D10A483A462146C8
:10D1300017F0B8FF0028E4D142B0BDE8F08168469E
:10D14000FFF733FA0028EED0214618F034FE00280D
:10D15000E9D0D6E7FC880020D88600202DE9F047EA
:10D160000F8C94B080460E469146F38BBB420AD892
:10D170000024009404AB4A4631464046FFF790FF36
:10D1800014B0BDE8F087022303AA39463046FBF706
:10D190007CF805460028EBD19DF80C309DF80DA0D9
:10D1A0000D2B24D154463F2C28BF3F24B91C2346C5
:10D1B00004AA89B23046FBF748F8BAF1000FD7D07D
:10D1C00098F81030012BD4D104AB13F8012B342A7A
:10D1D000CFD00135EDB2AC42F7D804F15002631C58
:10D1E0000DEB0204342204F8402CDCB2C1E70AF152
:10D1F000020139448FB2B8E710B5C4B002A801915A
:10D200001446FFF7A5F9019902A8FFF76BFB28B9AF
:10D21000BDF80C2102A92046FBF789F844B010BDE7
:10D220002DE9F0418CB005460C469046002126229F
:10D2300002A81F465BF0C4FB4FF2BF03ADF82A30D3
:10D240002B7F9B0736D42B7C1C48002B0CBF0C215A
:10D250001B2117F0A3FA064670B302462146284662
:10D26000FFF7CAFF044660B97FB902A816F0D4F9E7
:10D27000134B1248009502AA314617F007FF0446E7
:10D2800060B13046FAF743FF10E03A464146304677
:10D29000FBF74DF804460028E7D0F2E7129BEB625B
:10D2A000139B2B632B7F43F002032B7720460CB09C
:10D2B000BDE8F0810524F9E70324F7E7FC880020A6
:10D2C0009BD000002DE9F0430D4691B007469146F2
:10D2D0000021262206A89846189E5BF071FB2C7848
:10D2E0004FF2BF03ADF83A301CB10E238DF8083071
:10D2F00001246B7843B104F14002631C0DEB02047E
:10D30000332204F8382CDCB2AB7843B104F140028C
:10D31000631C0DEB0204052204F8382CDCB2EB7818
:10D3200043B104F14002631C0DEB0204032204F834
:10D33000382CDCB22B7943B104F14002631C0DEBB5
:10D340000204022204F8382CDCB26B7943B104F1F8
:10D350004002631C0DEB0204072204F8382CDCB2F7
:10D36000AB7943B104F14002631C0DEB020434229B
:10D3700004F8382CDCB2EB7943B104F14002631CB1
:10D380000DEB0204012204F8382CDCB22B7A43B1F5
:10D3900004F14002631C0DEB0204002204F8382C57
:10D3A000DCB26B7A43B104F14002631C0DEB020462
:10D3B000042204F8382CDCB2AB7A43B104F1400209
:10D3C000631C0DEB02040C2204F8382CDCB2EB7A5F
:10D3D00043B104F14002631C0DEB0204352204F852
:10D3E000382CDCB23B7C2748002B0CBF0B211921C9
:10D3F00017F0D4F90746002841D018EB04030ED1EA
:10D4000006A816F009F976BB1E4806AA394617F099
:10D4100049FE054618BB284611B0BDE8F0830D2231
:10D420008DF8042001A902228DF80530FAF77FFF5C
:10D430000546A0B95CB9B8F1000FE1D042464946B3
:10D440003846FAF774FF05460028D9D007E022468F
:10D4500002A93846FAF76BFF05460028EBD038469C
:10D46000FAF755FED7E70AAA06F11004306871688A
:10D47000134603C30836A6421A46F7D1C4E703256C
:10D48000C9E700BFFC88002010B5034B044600220A
:10D49000FFF72DFC204610BD31D00000427C034632
:10D4A000C2F34000920742BF187FC04300F0010062
:10D4B0007047427C0346C2F34000920744BF187F86
:10D4C00000F00100704730B5C5B0044602A80D4613
:10D4D00001920093FFF73CF8DDE90021BDF820310F
:10D4E00002A8FFF743F940B901462A4602A8FFF710
:10D4F0009CFA02A92046FFF769FC45B030BDFFF752
:10D500002DBE000010B5064B04460122FFF7EFFBCD
:10D510002346044A43F8342F2046E36310BD00BF7E
:10D520003DD0000059D6000010B50446FFF79AFC24
:10D5300004F13400BDE81040FBF7E2BC10B504462E
:10D54000C2B06846FFF704F8227F002363F30002AD
:10D550006361A361227769462046FFF737FC42B03A
:10D5600010BD10B5C2B004466846FEF7F1FF69462B
:10D57000201D3434FFF70CFB2046FBF7C1FC34219F
:10D580006846FFF712F858B1D0F8023040991BBA3C
:10D590006FF000429A4228BF1A462046FBF7F4FC7F
:10D5A00042B010BD70B5C4B0054602A80E46019247
:10D5B0000093FEF7CDFFDDE90021BDF8203102A880
:10D5C000FFF7D4F8044668B93246012102A8FFF7F4
:10D5D0002CFA02A92846FFF7F9FB044610B92846A1
:10D5E000FFF7BFFF204644B070BD38B50546FFF7D2
:10D5F00013FD044610B92846FFF7B3FF204638BD97
:10D6000010B5C2B004466846FEF7A2FF6946201D69
:10D61000FFF7BEFA34216846FEF7C7FF78B1D0F8AD
:10D620000230A16B409A1BBA881A984207D2521A4C
:10D630001A4404F13400FBF7A7FC42B010BD684661
:10D64000FFF781FA69460348FFF7C0FB2046FFF762
:10D650006BFFF2E70C8A00200148FFF7D1BF00BF43
:10D66000408A0020FFF77ABD38B5082204460D46EF
:10D670005BF05EF830B9BDE8384008484FF400313F
:10D68000FBF7CBB92B6823606B6863600348BDE888
:10D6900038404FF40031FBF7B7B900BF0037002026
:10D6A00010B500230446036043600249FFF7DCFF26
:10D6B000204610BD1F63070010B50446043003F078
:10D6C0008BFF2346074A43F8382F94F84A202364F7
:10D6D000002363F300026364A4F8483084F84A200E
:10D6E000204610BD99D9000007B590F84A30DB07F5
:10D6F00004D5B0F8480003B05DF804FB06480DF10E
:10D70000060112F03DFC18B14FF47A73ADF8063003
:10D71000BDF80600EFE700BF5CB400202DE9F04142
:10D72000184E96F8AA369B07044629D5164812F0DB
:10D7300090FCC8B12046FFF7D7FFA78A0546FFB97E
:10D7400004F1040822461149404604F02FF9294605
:10D750000122404603F0BAFF2A46394606F2D2308B
:10D76000BDE8F04102F054B9A28A4AB106F2D230C3
:10D77000012102F04DF9201DBDE8F04104F032B95D
:10D78000BDE8F081D88600205CB400201DDB0000DD
:10D790008B0501D5FFF7C2BF704790F84A20A0F86B
:10D7A000481042F0010280F84A20FFF7B7BF00009E
:10D7B00070B5C2B06846FEF7CBFE1748142116F0CC
:10D7C000EDFF044628B390F83030042262F3C6031C
:10D7D00080F8303069461148FFF7DAF9A8B9104EE1
:10D7E000082516F8011B6846FEF7DFFE68B12146E2
:10D7F00018F0E1FA48B9013DF3D10A4B0621D3F8FC
:10D80000E823204618F075FC18B12046FAF77FFC93
:10D810000024204642B070BDFC880020108A002001
:10D8200027630700D886002073B504460E46FFF72D
:10D83000BFFF054680B122460A490B4817F0DAF8C7
:10D840000094084B08483246294617F01FFC04464E
:10D8500020B9204602B070BD0324FAE72846FAF743
:10D8600056FCF6E795D90000FC88002002460846E1
:10D87000C98B3B2900D8FEE73C393C2389B2FAF733
:10D8800004BD262200215BF09BB80000F0B50746DE
:10D8900091B024480C4606211546FAF7FBFF0646D0
:10D8A00001A8FFF7EEFFB6B3234601AA04F1200C4E
:10D8B00018685968144603C4083363452246F7D1F3
:10D8C000186820609B88A3804FF2BF03ADF8263014
:10D8D000F8F709FA32302A460B900CAC1035106874
:10D8E0005168234603C30832AA421C46F7D13C22A2
:10D8F00001A93046FAF71BFD78B907F1440001226F
:10D900003146FAF752FE3B6C07F13800984202D1DB
:10D910000B99FBF72FFB11B0F0BD3046FAF7F7FB80
:10D92000F9E700BF4C37002030B5044693B003A898
:10D93000FFF7A7FF636CABB1596899B1236C04F191
:10D9400038059D420ED103A80191FFF78FFFF8F72C
:10D95000CAF90D9B0199C01A002805DA1946284614
:10D96000FBF708FB13B030BD04F14400FAF762FE88
:10D9700007480EA907F00EFB03A92046FFF754FF46
:10D980000028EFD000212846FBF704FBEAE700BFA0
:10D99000B08A0020FFF7C8BF0148FFF7C5BF00BF2E
:10D9A000D8B50020F0B593B00C46032200210646FE
:10D9B0006846FAF781FB08A8FFF763FF204617F0D7
:10D9C000D7FC002842D00DF102021221204618F0A7
:10D9D00011FB00283AD108230DEB03021321204646
:10D9E00018F02CFB90BB11210DF1060301AA204673
:10D9F00018F062FA014648BB371D6A46384603F004
:10DA000097FE054610B3BDF80630BDF80420214648
:10DA1000FAF7A4FCE0B902A90CA801F075FDBDF865
:10DA20000230ADF8423008AA2946384603F014FF08
:10DA300070B910230DEB03021521204618F0FEFAF1
:10DA400020B904AA08A93046FFF720FF13B0F0BDA3
:10DA50002846FAF75CFBF9E770B58CB002A80D46D2
:10DA60001646FFF70EFF4FF2BF032948ADF82A30E4
:10DA70000DF1020112F07CFA002847D125481C2143
:10DA800016F09AFE0446002840D0728C122118F03D
:10DA900024FBC0BB082306F118021321204618F00E
:10DAA000E8FA80BB1C4E1421B6F8B826204618F0C0
:10DAB00014FB40BB11232A8C8DF80430EB8B9B1A8E
:10DAC000FF228DF8052004225BBA0DEB02012046EF
:10DAD000ADF80630FAF72BFCA8B9BDF806302A8C51
:10DAE0005BBA9BB229462046FAF738FC58B9BDF814
:10DAF000021002A815F0B8FD02AA214606F5097029
:10DB000017F0D0FA10B12046FAF701FB0CB070BD47
:10DB10005CB40020FC880020D8860020FFF79CBF62
:10DB200070B5027A531E3F2B0FD80731D0E900455C
:10DB30000E461046072809D9230A083806F8014975
:10DB4000C0B243EA05642D0AF4E7FEE7D308C3EB4D
:10DB50004313A1EBD20102EBC30212F0FF0209D082
:10DB600001239340DBB20A785842013B0240234034
:10DB700013430B7070BD102900D9FEE700F8011B9C
:10DB8000102200215AF01CBF70B503784BB3DA00A5
:10DB9000D5B20A88B2FBF5F4013B05FB1422DCB2D6
:10DBA000C2F3C403E31A50FA83F302F007025B786E
:10DBB000012606FA02F2134013D04A88B2FBF5F3AD
:10DBC00005FB1322C2F3C403E31A50FA83F302F0F5
:10DBD00007025B7806FA02F2134214BF30460020B7
:10DBE00070BD1846FCE77FB504460D4602A841F219
:10DBF000210117F072FE48F2050103A817F06DFE2F
:10DC000004F10806B4420AD014F8011B019102A8DD
:10DC100017F067FE019903A817F063FEF2E7BDF85D
:10DC20000A302B80BDF80E306B8004B070BD13B588
:10DC300000230C466946CDE90033FFF771FF21460A
:10DC40006846FFF7D0FF02B010BD10B510F8014BC9
:10DC50000023DAB2944207D910F8012B8A4203F16B
:10DC60000103F6D0002010BD0120FCE730B5C7B09D
:10DC7000054608A80C4618F023FD08A818F035FD45
:10DC80000822294608A818F036FD694608A818F0A9
:10DC900038FD6B4603CB20602378616043F00203BC
:10DCA000237008A818F019FD47B030BD2DE9F047E2
:10DCB0009946274B8EB004460DF1100A186804905F
:10DCC000904620469A889B79ADF814200F468AF832
:10DCD0000630FBF772F818B907200EB0BDE8F087E0
:10DCE0004FF480712046FAF784FF1121064638462A
:10DCF000FAF77FFFB31F9BB2F92BC5B2ECD8102DFA
:10DD0000EAD81222002109A85AF05AFE9AE8030024
:10DD1000D8F800300690ADF81C10CDF81E302A4619
:10DD2000D8F80430CDF8223039460DF126005AF0EB
:10DD300031FD4FF480431022CDE90032CDF8089038
:10DD400005F10E0306AA31462046FBF711FBC4E796
:10DD5000106307000346074A10B543F8042FC36059
:10DD600047F2305303610446FAF7F8FEA4F8560070
:10DD7000204610BDD5DE0000F8B50546164817460A
:10DD80001E4616F048FD0446B8B13246102118F080
:10DD900099F9E0B9EA682B1D9A420FD1012E06D1FC
:10DDA000B5F856200B21204618F097F978B90A48A3
:10DDB0003A46214617F076F948B9F8BD05F1140343
:10DDC00040220A21204618F06CF90028E6D02046AF
:10DDD000BDE8F840FAF79BB9FC88002037B50D483C
:10DDE0000193154616F017FD044680B1019A1021E3
:10DDF00018F068F928B907482A46214617F052F961
:10DE000028B1204603B0BDE83040FAF780B903B02E
:10DE100030BD00BFFC88002030B58BB026220D46F7
:10DE2000684600215AF0CCFD4FF2BF030B48ADF815
:10DE30002230112116F0B2FC044660B12946684632
:10DE400015F02AFC05486A46214617F02BF910B157
:10DE50002046FAF75CF90BB030BD00BFFC8800200B
:10DE60004A1E47F22E539A429ABF016100200720B2
:10DE70007047000007B50B238DF8043002238DF89E
:10DE80000530B0F85630013304229BB2A0F856306A
:10DE90000DEB02015BBA0448ADF8063012F021FE2A
:10DEA00003B05DF804FB00BF5CB4002010B504466D
:10DEB0000430FBF725F82046BDE81040FFF7DABF35
:10DEC000034B93F8A936042B01D1FFF7EFBF70473E
:10DED000D88600200148FFF7F3BF00BF24B600201A
:10DEE000214B93F8A936042BF7B504460D46174687
:10DEF00038D10DF105021021284618F069F888BBC9
:10DF00000DF106020B21284618F074F850BB174893
:10DF1000092112F00AF860B1B4F85620BDF80630B5
:10DF20009A4206D19DF80560012E04D02046FFF7E5
:10DF3000BDFFFF2610E0F98B43884ABA5BBA92B264
:10DF40009BB29A4203D04180084812F075F94CF216
:10DF50005031201DFBF71EF833463A46294620462D
:10DF6000FFF73CFF03B0F0BDD88600205CB4002072
:10DF7000092310B549BA03700223437041804371ED
:10DF80000B21082352BA04460171C2800372102289
:10DF900000210A305AF014FD012363720023A3729A
:10DFA00010BD08B5083017F0F3FE0830C0B208BD48
:10DFB000F0B50446294890F8A936042B99B00E46CE
:10DFC000154607D0FF232A4631462046FFF7D4FEE8
:10DFD00019B0F0BD02F1100100F5D5600CF0A0FB06
:10DFE0000028EFD0402207AB0A21304617F0DCFFB3
:10DFF00002460028E6D1E368271D9F4209D007A901
:10E0000004F11400FAF759FE0028DBD02046FFF790
:10E010004DFFB4F85630E98B01339AB249BAA4F8EF
:10E02000562089B26846FFF7A3FF6846FFF7B9FF9D
:10E03000694602460A4812F054FD03460028C1D141
:10E0400007AA412104F11400FAF7C1FE4CF2503145
:10E050003846FAF79FFF0123B5E700BFD8860020B6
:10E060005CB4002000BA70474200400800F0553010
:10E0700002F0AA3202439300920802F0333203F016
:10E08000CC33134318011B0903F00F3300F0F030B9
:10E09000184300BA70474A78102A28BF102202316C
:10E0A00001600271704710B5044610220846A11C99
:10E0B00000F018F9607010BD41780230FAF74EBEDA
:10E0C00038B50D4641780446102928BF102128464E
:10E0D000FFF751FD6278102A04F1020105F10100F9
:10E0E00028BF1022BDE838405AF054BB40780228BF
:10E0F00094BF00200120704713B50446684606F01F
:10E10000C6FD62786388023AD2B2022A5BBA28BF9F
:10E1100002226846211DADF8003006F0BDFD009BCF
:10E1200000209AB262F30F001B0C63F31F4002B091
:10E1300010BD0A88034652BA08465A80191D0222A9
:10E1400006F0F9BD00232DE9F3410B604389044635
:10E150000D462BB1DFF88080608910B1022803D80A
:10E16000062002B0BDE8F081606870B32189022307
:10E170006A46FAF76AF86E46737862899F1CBA425B
:10E18000EED33278C2B9042BEAD1606820B121897C
:10E1900006236A46FAF779F8D6F80200FFF762FF1D
:10E1A000FFF762FF3378002B18BF00222B6808BFEF
:10E1B0004246104003432B606389DB1B6381636825
:10E1C0002BB123891F442781C6E72668D4E723683B
:10E1D0003B442360C0E700BF00F8FF071FB50023E2
:10E1E0000293ADF80C30831C01934378ADF80E30E8
:10E1F00001A8FFF7A7FF05B05DF804FB07B501A96B
:10E20000FFF7ECFFB0FA80F0400903B05DF804FBC3
:10E2100002780C2A034611D80C2A11D8DFE802F044
:10E22000120720181E1E1020101010101A000222B3
:10E230005878904234BF002001207047352A0BD017
:10E24000012070474278022A0CD9023010F05FBAE0
:10E25000FFF732BFFFF74ABFFFF7D0BF1022E7E753
:10E260000822E5E7002070471FB50023CDE902032F
:10E270000C46019303AA0DF10E03352117F01CFE85
:10E2800018B9214601A8FFF75DFF04B010BD0000DA
:10E29000002310B583710A4B1B780446002B0948F4
:10E2A00018BF002008400AD0237004236370FFF7D2
:10E2B000DBFEFFF7D7FE0623C4F80200A37110BDF2
:10E2C0000364070000F8FF0713B504466846FFF72C
:10E2D000DFFF9DF806306A463521204617F0C9FE5B
:10E2E00002B010BD70B50B46054600211846164613
:10E2F0005AF066FB2C792968B44228BF344622467E
:10E300005AF048FA204670BD38B50D460446112132
:10E310002846FAF76EFC25602071204638BD70B59E
:10E320000E68097905463046FAF763FCC4B2102C32
:10E3300010D82246294630465AF0FAF908B92B5D22
:10E3400053B12246314628465AF024FA00232B5571
:10E35000184670BD0720FCE71820FAE713B5112313
:10E360000446084600918DF80430FAF726FD28B1DE
:10E3700069462046FFF7D3FF02B010BD0720FBE738
:10E3800010B50C4619B1182907D0204610BD064813
:10E390004FF48031FAF738FBF7E703484FF4803148
:10E3A000FAF73BFB0024F0E70037002010B50446E5
:10E3B000FFF7D4FF01462046BDE81040FFF7E0BF5D
:10E3C00010B50446FFF7ABFF01462046BDE81040FC
:10E3D000FFF7D6BF08B51130FFF7C0FF182808BFF8
:10E3E000002008BD10B5002304460370437404499F
:10E3F000FFF7DCFF03492046FFF7ECFF204610BD86
:10E400000C6307002F63070010B50446D0F8020024
:10E41000FFF728FE218849BA89B210BD38B50C46ED
:10E420000546FFF7F1FFC4E90001EB885BBAC3F3CF
:10E430004E0203F001032281A37238BD38B50546B0
:10E44000D1E900030C465BBA2B80FFF70BFE228953
:10E45000A37AC5F8020043EA42035BBAEB8038BDF9
:10E46000F8B50D460746FFF7CFFF064628460C468F
:10E47000FFF7CAFF8C4208BF86421AD1FB885BBAFD
:10E48000C3F34E0299B2EB885BBA98B2C3F34E0362
:10E490009A4202D011D901200AE001F0010300F0F4
:10E4A000010293420CD0002B0CBF4FF0FF30012033
:10E4B000F8BDB04271EB0403EDD34FF0FF30F7E746
:10E4C0000020F5E720B9081E18BF01204042704720
:10E4D00009B1FFF7C5BF0120704773B50646154661
:10E4E00001910024311901A8FAF7B3FB78B9019B17
:10E4F000032C1A7806D02E2A04F1010407D1013327
:10E500000193EFE7954218BF062002B070BD0620C8
:10E51000FBE708B1F9F7FBBD7047837C5A0701D4CC
:10E5200001F0A5B8C3F3C3007047000070B5002622
:10E5300004460D461022C0E90166067031460C30D3
:10E540005AF03EFA0C4B2946C4E9073604F1240080
:10E5500018F07DFD294604F12C0003F045F829460A
:10E5600004F1380001F0F4FA294604F1D80002F071
:10E57000EBF8204670BD00BF71F10000303113464A
:10E5800002488AB20021FAF746B900BF4C37002092
:10E59000014AFFF7F3BF00BFAC620700024B00F077
:10E5A0003800185C704700BF3D63070020B10228A7
:10E5B00014BF0020202070470820704730B587B076
:10E5C00093798DF80430383000230D46144602A9A3
:10E5D00008328DF8053001F0CFFA02A801F073FA85
:10E5E000023081B204A801F0A6FAA8B102A801F095
:10E5F0006AFA02A902462846F9F7E4FEB0B90222F7
:10E6000001A92846F9F7DEFE80B9A388A0715BBA9C
:10E6100008335BBAA38009E004A801F054FA04A906
:10E6200002462846F9F7CEFE0028DFD007B030BDFD
:10E630002DE9F04F0C468FB0282304AA0021204674
:10E64000F9F723FE9DF8166026B1002630460FB07C
:10E65000BDE8F08F02236A4628212046F9F715FE0F
:10E660009DF80180E38B08F101084FEAC80808F122
:10E67000280B5B4501D20626E8E7B246B14637468D
:10E680002A255B462A46214601A801F023FA9DF877
:10E690000430012B11D96D2B3CD1002FEBD19DF80B
:10E6A00005A0BAF1040FE6D82A2D2BD19DF8013030
:10E6B000002B2F4608BF4FF0010901A801F003FA13
:10E6C0000544ADB2AB45DCD8D5D1B9F1000F30D09F
:10E6D000082208F120012046F9F7F4FE2A2F1CD168
:10E6E0009DF800308DF81630BDF814305BBA083B49
:10E6F0005BBAADF8143004AA282300212046F9F7AC
:10E70000F3FDA3E705F108032F465B4508BF4FF073
:10E710000109D2E74FF00009CFE79DF80130013B36
:10E720008DF801306A46022328212046F9F7DCFDE6
:10E73000DAE7002F89D00AF10201C9B202A801F07C
:10E74000EEF902A801F0BFF902AA03463946D5E75F
:10E7500010B504460C30F9F7EDFF04F11C00BDE8DC
:10E760001040FAF763BB2DE9FF470C8C0F4681463A
:10E7700090469A4602AA022321463846F9F785FDBB
:10E780000646002838D19DF80950FB8B013504EB73
:10E79000C505ADB2AB4233D30234A4B208F10808C8
:10E7A00009F13809AC4223D22B462246394603A848
:10E7B00001F090F9A8B99DF80C30012B05D803A8F9
:10E7C00001F081F90444A4B2ECE76D2B0BD1CDF834
:10E7D00000A0434622463946484601F036FB002851
:10E7E000EDD0064608E013F0C00FE8D0022603E0A3
:10E7F00021463846F9F7B6FC304604B0BDE8F0874C
:10E800000626F9E737B50D460823098C6A462846DF
:10E81000F9F73BFD044660B9BDF802305BBA9AB225
:10E82000C3F3CC0343B9D30706D408212846F9F72C
:10E830008DFC204603B030BD0224FAE738B504460B
:10E840003AB1012A0ED02368002B0CBF0320002010
:10E8500038BD0D680A6000688542F4D0FFF759FEA4
:10E860002560F0E70868C18BFAF720F805462068B4
:10E87000A842F2E7F0B585B00F469DF82850114642
:10E88000112D4FF00002064603920AD03A2D08D00F
:10E89000062D06D000240398FFF73BFE204605B066
:10E8A000F0BD9DF82C20019303A8FFF7C7FF044695
:10E8B0000028F0D1112D0399019B0BD03A2D0FD0D8
:10E8C000062DE7D10A4606F1D800394602F05AFC77
:10E8D0000446E0E71A4606F12C0002F0E1FFF7E7F4
:10E8E0001A4606F1240018F0E3FCF1E72DE9F043A5
:10E8F00085B01F46002301930B689DF830809DF87A
:10E900003490164693F83220D20705460C4601D4BF
:10E91000042407E04268002AFAD0DB8BB3F5A06F2D
:10E9200007D902240198FFF7F4FD204605B0BDE8A1
:10E93000F083334806F110010BF0EAFE10B1B9F193
:10E94000000FEED02B786BB1B8F1000F0AD02C4835
:10E9500031460BF0DDFEC0B9112F36D03A2F21D051
:10E96000062FD5D021469DF8382001A8FFF766FF75
:10E9700004460028D6D101992846FFF759FE019890
:10E980000194D5E901319847CCE706F108084046E3
:10E9900000F044FD0028DFD0404600F073FD002861
:10E9A000DAD1B5E7314605F1240018F001FC002862
:10E9B000D8D0206808230DEB0302018CF9F765FC21
:10E9C0009DF80830802BCDD1ABE720680823018C5F
:10E9D0000DEB0302F9F759FCBDF80A10094849BAD2
:10E9E00089B202F09BFF002892D0BDF80A100548BA
:10E9F00049BA89B202F088FF0028B3D088E700BF87
:10EA0000808D0020848700202DE9F04786B0DDE965
:10EA10000E8705460C4691461E464FF0010A38788F
:10EA200010B998F800307BB920680223018C05AA40
:10EA3000F9F72BFC40B998F800302C2B12D006D8EF
:10EA40004BB12B2B08BF022006B0BDE8F0873B2B53
:10EA50001DD03C2BF8D121683B4632462846FFF7B3
:10EA600082FE0DE0CDF808A03A782146CDE90002FB
:10EA70004A462846FFF73AFF21682846FFF7C2FEBC
:10EA80000028E1D19DF8143088F80030C7E7022053
:10EA9000DAE700002DE9F74F08460F4600F0E7FDE2
:10EAA0003946834637480BF03BFE374A00904FF01B
:10EAB000000AD2F87C61544602F5D568002E5CD07D
:10EAC000314640460BF03BFE68BB3146384600F00D
:10EAD0000BFE327C8242054614D830460192FFF785
:10EAE0001CFD019A8146154610223946304659F0E0
:10EAF0001FFE002840D03CB9327CAA4237D9AA4632
:10EB0000344610E0D946EFE73046FFF706FD0190A6
:10EB10002046FFF702FD019A8242304605D2FFF7F8
:10EB2000FCFC4845E8D27669C8E7FFF7F6FC01909F
:10EB30002046FFF7F2FC019A824205D92046FFF7F2
:10EB4000ECFC4845D8D3EEE7B17CA27C4A40D20722
:10EB500002D5CB07E7D5CFE7AA45CDD3E3D13146E0
:10EB600040460BF0DDFD009B9842DCD1C4E7304607
:10EB7000FFF7D3FC8346C2E73446204603B0BDE826
:10EB8000F08F00BF808D0020D8860020F0B50C46A5
:10EB90008DB002F11801054608460191164600F0B5
:10EBA00096FD019960B11F4804F0C6FC40B1E18BAD
:10EBB0002046F9F77BFE014610B12846FFF7C8FD55
:10EBC0006023029340238DF80F30B3885BBA28335B
:10EBD0005BBA08A8ADF80C3000F0DEFC292308A9C8
:10EBE00028468DF80E30FFF755FF0346B8B104AE46
:10EBF00000F1100718685968324603C20833BB4257
:10EC00001646F7D102AA21462846FFF7D7FC20B9BD
:10EC1000282202A92046F9F7D5FB0DB0F0BD14203B
:10EC2000FBE700BFA08F00202DE9F047112BB1F8C2
:10EC30001EA08AB080460D461646994602F110077E
:10EC400075D1538C52483A46314614F0E3FD002802
:10EC50006DD095F83100C0F3410014F01BFE840123
:10EC600004F47C6444F4C044602364BA96F825201C
:10EC70000093ADF80040C4F3072402F0030324F02E
:10EC8000300444EA031496F824308DF801409AFACF
:10EC90009AFAADF804A08DF806901BB912F0080F8F
:10ECA00008BF402330468DF8073000F0F9FB0028FC
:10ECB00044D13378FF2B41D0334602AC18685968F1
:10ECC000224603C20833BB421446F7D106AA3B468C
:10ECD00007F1100C924618685968144603C40833AB
:10ECE00063452246F7D1384600F0E5FCC0BB282238
:10ECF00069462846F9F766FB0446C8BB28464B46DA
:10ED0000524602A918F06FF9384600F0E0FC98BBB3
:10ED100096F8253095F83120C3F3001363F386127B
:10ED200085F8312029464046FFF712FD20E095F88E
:10ED30003100C0F34100FFF739FC90E73946404607
:10ED4000FFF7A8FE08B3034602AC00F1100C1868E8
:10ED50005968224603C2083363451446F7D1B5E724
:10ED60006A4629464046FFF729FC04460028BED0E3
:10ED700020460AB0BDE8F0876A4629464046FFF7BC
:10ED800005FF0028C4D00446F2E71424F0E700BFD2
:10ED9000FC88002070B50B480E4610F083FF044637
:10EDA00060B9094BD3F87C514DB13146284600F08B
:10EDB0009BFC2B7C834201D96D69F5E70124204639
:10EDC00070BD00BF5CB40020D886002007B508489D
:10EDD0000DF1060311F068F838B9064BBDF80620AE
:10EDE000B3F8B8369A4208BF042003B05DF804FBBC
:10EDF0005CB40020D88600202DE9F04F9DB00F466E
:10EE00000DF120090021804692464846262259F0FD
:10EE1000D7FD002339688DF8163012A800F038FEAF
:10EE200006460446002870D10DF1500B10909BE867
:10EE30000F000CAC84E80F0018AC94E80F0089E8D0
:10EE40000F009DF84F308DF844309DF84930C6F3DF
:10EE500007221B0963F301029DF860308DF84520FD
:10EE6000FF2B58D13B6893F8323013F00C0F50D180
:10EE7000204600F02CFC064620B1AA48214604F0AA
:10EE80005BFB06463B6893F8322012F00C0F03D070
:10EE900093F831305A066DD5A348214601F0F3F8B6
:10EEA00001230546002865D08DF8163038682821E2
:10EEB000F9F758F99DF84E308DF817300DF116031B
:10EEC00001930DF1170300934A4612AB39464046B1
:10EED000FFF79AFD0446C0B99DF81630002B6ED09E
:10EEE0009DF81730292B6AD13B6806903246394687
:10EEF00006A893F831B0FFF7A1FC0546CBF3801BC1
:10EF00000698CDB3FFF705FB2C4620461DB0BDE8A3
:10EF1000F08F0126B6E78448214601F0A3FA0546A2
:10EF200028B101238DF8163035462E46BEE73B68E2
:10EF300093F8323013F00C0F11D0204600F0CBFACA
:10EF400098B921464046FFF725FF70B92246594639
:10EF50004046FFF73BFFB0FA80F6760906E0204610
:10EF600000F0B9FA0028E0D1E7E7012686F00105B4
:10EF7000EDB29BE7012599E790F83130018C6BF3F6
:10EF8000861380F83130F9F705F9069A674821466B
:10EF900008F0AFFB069B524607A94046CDE9064361
:10EFA000FFF72AFF0798FFF7B4FA06988DF8164086
:10EFB000FFF7AFFA9DF8163043B3002501E0002DAE
:10EFC000F8D0BAF1000F13D19DF8163085F0010585
:10EFD000002B14BF1A463246EDB2CDE9013200953E
:10EFE0009DF817304A4639464046FFF77FFC0446F5
:10EFF0009DF8163053B19DF81730009301964B469B
:10F000003A4612A94046FFF735FC0446002E3FF46D
:10F010007CAF3B6893F8323013F00C0F0AD14448B0
:10F0200009F001FA00283FF470AF9DF84F30013B22
:10F030008DF84F309DF84F30FBB18DF81C3038689B
:10F04000012307AA0721F9F74FF99DF817303A2B4A
:10F0500015D138680123018C07AAF9F716F904467F
:10F0600000287FF452AF9DF81C10324A062312F894
:10F07000010B814203D0013BF9D1022445E73868F6
:10F0800090F83250C5F38105022D17D19DF8173045
:10F09000112B13D1018C02312B4607AA89B2F9F743
:10F0A000F4F8044600287FF430AFBDF81C305BBA9A
:10F0B0009BB24FF2BF0293423FF426AF386890F8FC
:10F0C0003230C3F38102012A1FD1DB071DD49DF822
:10F0D0001730112B19D1018C0231022307AA89B2F2
:10F0E000F9F7D3F8044600287FF40FAFBDF81C30C1
:10F0F0005BBA99B2ADF81C309DF81730112B04D1D2
:10F100000D4802F00BFC0028B7D03B6807930023A2
:10F1100006483B6007A908F0F3FA0798FFF7F9F9EA
:10F12000F3E600BFA08F002054880020888C0020C8
:10F13000808D0020766307008487002073B5054624
:10F1400000F10C063046F9F799FA044668B1014619
:10F150003046F9F70CFB002201A928460194FFF77D
:10F160004BFE0198FFF7D5F9ECE702B070BD000047
:10F170000148FFF7E3BF00BF5887002070B53C226D
:10F1800004460E46002159F01BFC3146204600F093
:10F190007FFC054680B9A379112B05D03A2B03D00B
:10F1A000062B0AD1142300E0082304F128022821A9
:10F1B0003046F9F76AF800B10625284670BDF0B56B
:10F1C000044603C989B006AD85E80300294604A8B2
:10F1D00017461E4607F032F910B9BDF814308BBB44
:10F1E000BDF81C3073B3069B1B7803F0E003602B63
:10F1F00028D106F5A8465C3600953B460DF10F0276
:10F200002146304606F0E2FC98B9A379112B07D0CD
:10F210003A2B15D0062B0CD1142204F128010BE057
:10F220009DF80F3004F128012BB12A46304606F034
:10F23000E4FE09B0F0BD0822284616F01FFCF8E7EE
:10F240000822EAE71720F4E78379062B01D0112B77
:10F2500003D1408D40BA80B270470020704770B52E
:10F26000013905460024E6B2F300B242D8B20CD907
:10F270002B5D01340E5DB342F5D073401A0604D401
:10F2800001305B00C0B2DBB2F8E770BDFD2300F8CF
:10F29000013B0721FAF760B838B505461446073236
:10F2A000D20859F077FA2C7438BD10B4027CD31D03
:10F2B000DB1008D0591EC2EBC3044FF0FF32A2404E
:10F2C000445C22404254C3F11002102B92B25DF80C
:10F2D000044B88BF00220021184459F071BB102A4A
:10F2E00000D9FEE7FFF7BBBF10B5037C0C7C9C4246
:10F2F00008D1E21DD208FFF7F2FF84428CBF002044
:10F30000012010BD0020FCE72DE9F0410F7C047CBA
:10F31000BC42A04628BFB84608F10702D2080646FC
:10F320000D46FFF7DCFF804505D8BC422CBF00200E
:10F330000120BDE8F081C0F3C703F05CEC5CA042A3
:10F34000F4E700F0E703202B06D000F0DF00A0F187
:10F35000400358425841704701207047036823B961
:10F360004068B0FA80F04009704700207047036899
:10F3700003330AD182884FF6FF739A4205D183790D
:10F38000FF2B02D1C079C00970470020704708B533
:10F390000821F9F7E1FF00B1FEE708BD0B68036043
:10F3A0004B684360704713B50446086849686B466C
:10F3B00003C39DF80030002283F002036946204613
:10F3C0008DF80030FCF74BFC02B010BD10B50C46B8
:10F3D000002201462046FCF742FC237883F002031A
:10F3E000237010BD10B50C46002201462046FCF7E4
:10F3F00036FC02232372237883F00203237010BDAE
:10F400004FF0FF320023C27049BA6FF0010203705F
:10F410004370837002714371C18070470368B3F118
:10F420007F4F05D18088A0F1FE03584258417047B4
:10F430000020704708B50246FFF7F0FF38B1907919
:10F44000FB289ABF80F00200C0F34000002008BDF6
:10F4500008B50246FFF7E2FF20B19079A0F1FC0366
:10F460005842584108BD08B50146FFF777FF40B93B
:10F470000846FFF77CFF20B9BDE808400846FFF7C3
:10F48000E7BF08BD08B5C288FFF7C8FF38B150BA5A
:10F4900000F57C7080B21F288CBF0020012008BDC1
:10F4A000026842B9436833B9826822B9C068B0FAC9
:10F4B00080F0400970470020704702684AB94368ED
:10F4C0003BB982682AB9C06800F17F43584258416D
:10F4D000704700207047038848F2FE0023F47C53F5
:10F4E0001B1A5842584170476FF001020023027006
:10F4F0006FF07F0242708370C37003714371837138
:10F50000C3710830FFF74FBF6FF001020023027094
:10F510006FF07F0242708370C37003714371837117
:10F52000C3710B6883604B68C360704730B5074C8C
:10F53000034604F11005224603CAAA421860596026
:10F54000144603F10803F6D130BD00BF8463070001
:10F5500030B5074C034604F11005224603CAAA42FF
:10F5600018605960144603F10803F6D130BD00BF9E
:10F57000AC63070030B5074C034604F11005224682
:10F5800003CAAA4218605960144603F10803F6D171
:10F5900030BD00BFC063070030B5074C034604F11F
:10F5A0001005224603CAAA4218605960144603F1A6
:10F5B0000803F6D130BD00BFD463070010B50C7C42
:10F5C000E21DD208FFF78BFEA04234BF00200120CD
:10F5D00010BD10B514460732D208FFF780FEA042D6
:10F5E00034BF0020012010BD0B6803604B684360EE
:10F5F0007047F8B5D40802F00707224605460E46C4
:10F6000059F0C8F867B1013F80233B412A5DDBB266
:10F61000591E0A402A55315D5B420B401A432A5558
:10F62000F8BD0A7C402A04D9403AD2B20831FFF72B
:10F63000E0BF70470A7CFFF7DCBF38B504461546CB
:10F640000430FFF7D6FFE57038BD0B6803604B68E8
:10F6500043604FF0FF310023C17252BA6FF00101D5
:10F6600003724372837201734373C281704708B59A
:10F670000278FF2A03D1407800F00F0008BD03880C
:10F6800048F2FE0223F47C53934206D0FFF715FFA5
:10F69000002814BF00200E20F0E70220EEE708B596
:10F6A0000378FF2B05D1FFF7E2FF831E5842584134
:10F6B00008BD0020FCE708B50378FF2B05D1FFF754
:10F6C000D6FFC31E5842584108BD0020FCE708B5CC
:10F6D0000378FF2B06D1FFF7CAFF032894BF002051
:10F6E000012008BD0020FCE71022FFF7B8BD022969
:10F6F00010B504460BD003290FD0012911D1FFF713
:10F70000CFFE80B92078FF3818BF012010BD0078E7
:10F71000A0F1FF0358425841F8E7BDE81040FFF759
:10F72000D6BF0120F2E70020F0E770B50546087C5F
:10F730000E461446FFF705FE00B9FEE71022002131
:10F74000284659F03DF931462846FFF773FF337CD0
:10F75000621EDB080334082B12F8010F14BF194690
:10F7600009214B1C94426854DBB2F4D170BD2DE9E1
:10F77000F3470B783A2B07460D4690461FD14B783E
:10F780003A2B03D0062002B0BDE8F08702350021F5
:10F7900000262A784245F3B266D0AE464FF0000C00
:10F7A00070461EF8014BA4F14102052A09D8373CE6
:10F7B000E2B202EB0C1CBCF5803FF1D3E2E7FF2183
:10F7C000E6E7A4F16102052A01D8573CF0E7A4F16D
:10F7D0003002D2B2092AECD98542D3D02E2C0CD1DA
:10F7E000062BCFD824D14246294601A8FEF775FE44
:10F7F0000028C8D1019BFB60C5E73A2C01D0A04589
:10F80000C0D1082EBED09CFA9CFC27F816C0027806
:10F8100001333A2ADBB203D142783A2A03D00130CD
:10F8200001360546B5E7FF29ACD102301946F7E7A6
:10F830004FF001090624FF29A4D05B1AD8B2034671
:10F8400007EB410A201A5A00514607EB400059F0D5
:10F850003BF8A21B52000021504659F0B1F8B9F113
:10F86000000FC0D100208EE7082BFBD04FF000091D
:10F870000824E0E70022FFF77ABF00002DE9F843F3
:10F88000DFF83490DFF8348006460D461746002432
:10F89000A7420FD0E3B21BB149462846F9F73CFA1C
:10F8A00036F814305BBA9AB241462846F9F734FA72
:10F8B0000134EDE7BDE8F883887507000D390700CE
:10F8C0002DE9F041027C073288B0D210013203AE3C
:10F8D00004460D465208034600F1100CB046186865
:10F8E0005968374603C7083363453E46F7D101924E
:10F8F0001B783B704046FFF7D8FC019A29464046EA
:10F90000FFF7BCFF237C0733772B03D80549284634
:10F91000F9F702FA227C04492846F9F7FDF908B004
:10F92000BDE8F0817C6307007F63070013B50446E0
:10F930006846F9F7C9F969462046FFF7C1FF02B0EA
:10F9400010BD0822FFF79ABF38B5282204460D469D
:10F9500000F10801F9F7B8F928462146FFF7F1FF51
:10F96000204638BD13B504466846F9F7ADF9694637
:10F970002046FFF7E6FF02B010BD08B5102258F090
:10F98000D7FEB0FA80F0400908BD000030B591F80C
:10F99000314014F0010491B0054603D00124204603
:10F9A00011B030BD01A8FFF7E9FB0028F7D107A887
:10F9B000FFF791FD08B3154B93F8A936002BEDD056
:10F9C00001A8FFF741FC9DF80A20062A05D0112A5C
:10F9D000E5D144F64C539842E0D02A792B4605EB0A
:10F9E00042029A421C460ED02188814203F1020352
:10F9F000F7D1003C18BF0124D1E707A8FFF74FFE5D
:10FA00000028D8D1CBE70024F3E700BFD886002038
:10FA1000F0B512B30379044600EB4306A64225462F
:10FA20001FD02F88974204F10204F7D159B1E3B1F6
:10FA3000013BDBB203711AB200EB43039D421CBFD2
:10FA400030F812302B80002105E0022B07D05C1C1F
:10FA5000047120F813200846F0BD0721FBE70321BD
:10FA6000F9E70029F1D01721F5E71B88FFDE0378BD
:10FA700003F0F003602B09D1808840BA80B22830AF
:10FA8000B0F5A06F8CBF00200120704700207047A8
:10FA900070B50E4602460546282300213046F8F789
:10FAA000F4FB044668B92846FFF7E1FF48B1AB888C
:10FAB000F28B5BBA9BB22833934218BF06242046D0
:10FAC00070BD0624FBE7037813B14078023070471D
:10FAD000012070472DE9F0410F46154606460246C3
:10FAE0009846294601233846F8F7CFFB044610B95B
:10FAF00034781CB974702046BDE8F0810223324688
:10FB000029463846F8F7C1FB04460028F3D13046B1
:10FB1000FFF7D9FF28444045C8BF0624EBE7002380
:10FB20000129036018BF0239C0F803301EBF01234A
:10FB300003704170704711F0070108B506D0C1F19C
:10FB40000801C9B2FFF7EBFF002008BD1820FCE751
:10FB500010B503460021074A80F88C10C0F89010B9
:10FB600043F8942F0446C0F89C308C2258F028FFAC
:10FB7000204610BDF9FF000038B50C4605460E4979
:10FB80001046102258F0D4FD6D23237048B902238B
:10FB90006370A07095F88C305A1C85F88C20E37047
:10FBA00038BD042363704023A370044BB3F8B83608
:10FBB0005BBAA380EEE700BF388F0020D886002014
:10FBC0002DE9F84300250F46904606460446844634
:10FBD0002A462B46294696F803E0BEF1000F09D1CC
:10FBE00000EB8504002908BF2146E578002D46D0AA
:10FBF0007BBBFEE7B6F800E0BCF80090CE450BD02A
:10FC0000B94503D111B90133DBB23146934284BF08
:10FC10001A4664460023B446BE4512D196F802E067
:10FC2000C64505D100EB85000523C37002203BE0EB
:10FC300039B9A8EB0E0E1EF0800F1EBF0133DBB2E8
:10FC4000314601350133232DDBB206F10406C2D162
:10FC5000CBE7BCF80050BD4204D119B9013300F123
:10FC60008C01DBB29A423CBF1A466446012ADDD9B8
:10FC700081B18142DAD931F8043CBB42D6D1234666
:10FC800099420C4612D2814200D2FEE75A1A081D50
:10FC900058F01AFE05230A48278084F80280E37092
:10FCA000082116F003F80020BDE8F883F2D983425A
:10FCB00000D2FEE70C1FE21A191D1846E8E700BF44
:10FCC00028370020002330B4014600F18C051C4683
:10FCD000CA785AB900EB83000022222B13DCC178CA
:10FCE000043081B100F8012C0133F6E7013AD2B2B9
:10FCF000CA7022B10A6840F823200124013304317C
:10FD0000A942E5D1E6E724B930BC0348082115F043
:10FD1000E5BF30BC704700BF28370020044B93F884
:10FD2000A936033B012B94BF02200020704700BF7F
:10FD3000D886002002460846C98B0B2900D8FEE76A
:10FD40000C390C2389B2F8F7A0BA0846C98B0C39D4
:10FD500008B589B2F8F7DFF900B1FEE708BD024641
:10FD60000846C98B0C390C2389B2F8F7BDBA70B5B7
:10FD700005460E46144652B111460020F8F7FAFE29
:10FD80002B7A03443344241A2B602C7270BD104626
:10FD9000F6E72DE9FF411F46002306460D46904633
:10FDA0008DF80330FFF7BAFF002847D0C98B2846EB
:10FDB000F8F77CFD0446002840D095F8323013F067
:10FDC0000C0F14D101230DF1030207212846F8F787
:10FDD0005CFA9DF803305A1E012B8DF8032030D9B0
:10FDE00001230DF1030207212046F8F77DFA95F86B
:10FDF0003230ADF8088013F00C0318BF01238DF8E2
:10FE00000B3000238DF80C308DF80A70F5F76BFF7E
:10FE10004022014601A8FFF7AAFF0C2201A92046B3
:10FE2000F8F785FA68B9214606F190000122F8F743
:10FE3000BCFB019906F19400F9F7B9F804B0BDE8EC
:10FE4000F0812046F8F763F9F8E7F0B50D4685B084
:10FE5000114607461E4602AA042328460191F8F7D8
:10FE600014FA0446B0BB9DF80A30019903F0C002B1
:10FE7000402A27D016D8CAB1BDF80C109DF80B2027
:10FE800049BA89B23846FFF79BFE044628BBBDF845
:10FE90000C209DF80B3052BA92B229463846FFF733
:10FEA00078FF17E01B06E7D5062413E006F10800EB
:10FEB000FFF7B4FAD0B1B37BF27B43EA0223ADF88B
:10FEC0000C30D9E7062302AA2846F8F7DEF90446E3
:10FED0000028D1D0204605B0F0BD95F8323013F09F
:10FEE0000C0FF7D00A9B00241C70F3E70224F1E703
:10FEF0002DE9F04F87B00746F5F7F5FE07F19009B9
:10FF000000F100468046494601A8F8F704FC013E8E
:10FF1000DFF8E0A03546019C002C5CD0214603A808
:10FF2000FFF708FF039BA8EB0302002A08DAEA1A8E
:10FF300015EA220538BF1D4601A8F8F7CCFBEAE711
:10FF40009DF813200132D2B238468DF81320FFF706
:10FF5000E5FE824204D921464846F8F76BFBEBE701
:10FF600033D24022414603A8FFF701FF214603A8F0
:10FF7000FFF7F5FEDDF80CB0E18BA5EB0B02204698
:10FF80003BEA220B28BFAB46F8F790FC0446D0B101
:10FF90009DF81320012A81BF94F83020052363F3D4
:10FFA000C60284F83020214603A8FFF7CEFE94F85D
:10FFB000322022F00D0242F0050284F83220214660
:10FFC0005046FEF7C5FB5D46B6E721464846F8F7C2
:10FFD0000CFBAB46DCE7AE1B002E07DA294607F127
:10FFE000940007B0BDE8F04FF8F7C4BF07B0BDE814
:10FFF000F08F00BF588700200148FFF779BF00BF8E
:020000021000EC
:1000000090870020002370B50E4615461360044605
:1000100044B110223146204658F08AFB10B12C60C2
:100020002469F5E7204670BD002370B50E461546DD
:100030001360044644B110223146204658F078FB44
:1000400010B12C606469F5E7204670BD0023C0E95B
:100050000033C0E903330372436100F1780100F11A
:100060001803994204D042695A6143611833F8E792
:100070000023C0F88C3000F17C03C0F8A03000F100
:1000800090038367704707B5406801AAFFF7BAFF7E
:10009000003818BF012003B05DF804FB0129F7B553
:1000A0000D4604461F460CBF4FF480514FF40051DB
:1000B0000E481646F8F7A8FCB7B9E368A3B1802349
:1000C00030468DF804300096FFF7D1FA9DF80530E0
:1000D00000F00F0023F03F0303438DF8053029465D
:1000E000D4E903326846984703B0F0BD00370020DA
:1000F000F8B506460F4614461D46AC4207D02246C8
:10010000002339463046FFF7C9FF2469F5E7F8BDFB
:10011000F7B50B78FF2B05460C4629D1406801AA9C
:10012000FFF770FF30BB164E10222146304658F0C4
:10013000FFFA08B33669002EF6D1AA6FF2B113693F
:10014000AB671646234604F1100718685968344611
:1001500003C40833BB422646F7D16B6809481361D4
:100160004FF480516A60F8F74FFC002003B0F0BDF7
:100170000720FBE71820F9E72520F7E70320F5E73C
:10018000AC6307000037002037B5044601AA406879
:10019000FFF738FF0546F0B104F17C0398421CD309
:1001A00004F1A403984218D2019B73B963680BB1A0
:1001B0001B6963600A484FF40051F8F725FCA36FF0
:1001C0002B610020A56703B030BD1A69002AF1D069
:1001D00012691A61EEE71720F5E72520F3E700BF63
:1001E000003700204168F8B5044600F17C0600F1B4
:1001F000A40749B1B1420D6904D3B94202D22046E5
:10020000FFF7C2FF2946F4E7F8BD000073B5937C01
:10021000DB0904460D46164633D001290CBF2021C8
:1002200040211C48F8F7F0FB04F118039E4203D369
:1002300004F178039E4222D3E36803B3337C8DF844
:100240000430B37C00965A0720D5C3F3C300B37CB7
:10025000C3F3000200F00F03F07C43EA0213C0F383
:10026000000043EA40139DF8050020F03F000343DF
:100270008DF805302946D4E903326846984702B024
:1002800070BD01290CBF01210221CAE73046FFF7EA
:10029000EEF9DCE70037002038B5CB7CDB070546FC
:1002A0000C4603D50A492046FFF79EF92A681346F3
:1002B0001BB19C420AD05B69FAE7626128462C6058
:1002C00022460121BDE83840FFF7A0BF38BD00BF7E
:1002D000008F002010B4046800222346C3B1994265
:1002E00007D01A465B69F9E753693BB15B69536113
:1002F00004E0002AF8D10CB163690360CB7C6FF392
:100300004103CB740A465DF8044B0021FFF77EBF22
:100310005DF8044B7047036837B50C461546CBB102
:100320009C4212D05B69FAE7224600210190FFF758
:100330006DFFA37C019865F3000322460121A3749D
:1003400003B0BDE83040FFF761BFA37C03F00103B9
:10035000AB42E9D103B030BD2DE9F3410B78FF2B5F
:1003600005460C4603D1072002B0BDE8F0810068C5
:1003700001AAFFF759FEC0B105F118039842F2D364
:100380007835A842EFD2237C0374637C4374A27C4B
:10039000837C62F300038374A37C827CC3F34003F9
:1003A00063F3410282740020DEE72046FFF793F8F2
:1003B0000028D8D16E69AEB173696B610FCC374636
:1003C0000FC794E8030087E80300738A23F460737F
:1003D00073822B68736132462E6001212846FFF735
:1003E00015FFE0E70320BFE737B5044601AA006820
:1003F000FFF71AFE0546F0B104F1180398421CD32A
:1004000004F17803984218D2019B73B923680BB1A9
:100410005B69236020462A460021FFF7F7FE6369E7
:100420006B610020656103B030BD5A69002AF1D0CC
:1004300052695A61EEE71720F5E72520F3E7F8B592
:100440000546044655F8181B00F1780749B1A94242
:100450004E6904D3B94202D22046FFF7C5FF3146A8
:10046000F4E7F8BD07B5006801AAFFF7DDFD003825
:1004700018BF012003B05DF804FB00002DE9F04136
:1004800004681D4E0546B4B1E37CDB0711D5224656
:1004900000212846FFF7BAFEE37C6FF341033146A3
:1004A0002046E374FFF7A0F8224601212846FFF713
:1004B000ADFE6469E7E7114E6C68A6F1500706F1DE
:1004C0001408B4B1B44201D0444510D100231946F8
:1004D00022462846FFF7E2FD402239462046FFF734
:1004E000ACF80023224601212846FFF7D7FD2469F6
:1004F000E7E7BDE8F08100BF008F0020508F0020AB
:1005000010B518220446002158F05AFA40232374EB
:100510000323A37410BD10B50446FFF7F1FF638AEF
:1005200023F4BE7343F48E73638210BD70B514461A
:1005300005460E461822002144F0020458F040FA05
:1005400004F0030401232E746B74AC7470BD38B5D1
:1005500005460C467CB16B6803F17C02944201D2E3
:100560002469F7E7A4339C42FAD2297A2046FFF7A0
:10057000BEF80028F4D02C6038BD10B50023C0E9C7
:100580000031044602724968FFF7E1FF204610BDC2
:1005900000231360036823B18B4204D013601B69EE
:1005A000F9E7172070470020704737B5044601AAC5
:1005B00004300D46FFF7ECFF58B163682B612A4603
:1005C000002301212046656003B0BDE83040FFF7FD
:1005D00065BD03B030BD000013B504460B4901AA48
:1005E0000430FFF7D5FF60B9019B094A934200D15F
:1005F000FEE743B963600023044A19462046FFF72B
:1006000077FD02B010BD1861F5E700BF84630700F5
:10061000C063070013B5002304460C49019301AAE7
:100620000430FFF7B5FF00B1FEE7019B084A934293
:1006300008D0084A43B96260044B064A01212046AB
:10064000FFF756FD02B010BD1A61F5E7846307009D
:10065000C0630700AC63070013B50446094901AA4B
:100660000430FFF795FF48B9019B074A43B9626020
:10067000054B044A00212046FFF73AFD02B010BDA9
:100680001A61F5E7AC6307008463070037B50446D9
:1006900001AA04300D46FFF77BFFA0B9019B63B9A7
:1006A00063680BB11B69636000232A461946204624
:1006B00003B0BDE83040FFF7F1BC1A69002AF3D05F
:1006C00012691A61F0E703B030BD000037B50E4D76
:1006D000044601AA29460430FFF75AFF88B163682F
:1006E0006BB11A461B69002BFBD11561064A00232A
:1006F0000121204603B0BDE83040FFF7F9BC65603A
:10070000F4E703B030BD00BF8463070030B5044692
:100710008DB00D4601466846FFF716F9238A034956
:1007200002AA2846F8F7F8FA0DB030BDE8630700D2
:1007300013B504466846F8F7C7FA69462046FFF73E
:10074000E5FF02B010BD00000246074942F8041F51
:10075000C260064A02610022C0E90522C2614FF46C
:1007600040420284704700BF010E0100310E0100BB
:10077000F0B5034690F855008BB00C4698BB12F0CC
:10078000010FD3F8C81004F110071AD021F000416E
:10079000C3F8C810224605AE10685168354603C537
:1007A0000832BA422E46F7D1228A01A952BA184617
:1007B000ADF80C201AF0B0FD003818BF01200BB0C6
:1007C000F0BD41F00041C3F8C810224603F14001DA
:1007D00052F8045B41F8045BBA42F9D1228A52BA5A
:1007E000A3F85220EBE70D20E9E738B500F51175C5
:1007F0000C4600F51472294618301AF086FF256061
:10080000002038BD70B500F11806054630460C468C
:100810001AF02DFFA0420BD364B1214630461AF0E6
:1008200062FF28461AF002FE003818BF012070BD92
:100830000120FCE72046FAE708B51AF009FE003867
:1008400018BF012008BD08B51AF04EFE002008BDF3
:10085000026802F5A04210B5D2F87041002123468B
:100860006BB198420DD01946D3F81832F8E7D1F899
:1008700018326BB1D3F81832C1F8183208E01720DB
:1008800010BD0029F3D11CB1D4F81832C2F8703170
:100890000024C0F818421AF027FE2046F0E70000B6
:1008A0000238C0B20E289ABF014B185C0020704776
:1008B000F0630700032938B505460C4600D9FEE76A
:1008C000022911D0032911D0012906D001211AF0E3
:1008D0002BFB003818BF012038BD02211AF024FB81
:1008E00030B904212846F2E70821F0E71021EEE7AD
:1008F0002046F1E770B505460E461446F5F7F3F9C4
:1009000021183046FFF7CCFF05EB8000C0F8341209
:10091000286800F5A240BDE870405C30F8F747BB9E
:100920002DE9F74F0446884691461F46002500F5FD
:100930000D7A4FF0010BE9B220460191FFF7BAFFA3
:10094000064690B35AF82530A8EB0302002A23DBB1
:10095000022D19D0019903291AD0012907D0204668
:100960001AF028F908B3304603B0BDE8F08F022131
:1009700020461AF0D9FA18B120461AF01FFAF1E70A
:1009800020461AF087F9EDE720461AF02FF9E9E73B
:1009900020461AF0DDF9E5E73A6889F800B0D11A87
:1009A00033EA210328BF13463B600135042DC2D131
:1009B0000026D8E710B5044608301AF0FBFFD4E94A
:1009C00033329B1A184410BD37B590F86E4214F0BC
:1009D000040405460ED0D0F828425CB108301AF065
:1009E000E9FF01902846FFF7E5FF019902462846F6
:1009F000A04701240023204685F86E3203B030BDA5
:100A000070B50E4615460446FFF7D4FF35448542BF
:100A100010D9D4F828326BB194F86E32206843F0C4
:100A2000040300F5A24084F86E326830BDE87040DF
:100A3000F8F7FCB970BD2DE9F04304468DB00D46C2
:100A40009146FFF7B7FFD4F8C830D5F80880002BDF
:100A5000074624DA04F1400307AA04F1500C186891
:100A60005968164603C6083363453246F7D1B4F8D1
:100A70005230ADF8143003AB00932A46002309F03E
:100A8000010120461AF07AFC054650B920463A4644
:100A90004146FFF7B5FF28460DB0BDE8F0830023BF
:100AA000EAE70120F8E72DE9F04104468CB00E4654
:100AB00002F00108FFF77EFFA36807464BB3D4F8A6
:100AC000C830002B23DA04F1400507AA04F1500CCA
:100AD00028686968134603C3083565451A46F7D187
:100AE000B4F85230ADF8143003AB00930022334613
:100AF000414620461AF042FC054660B920463A4677
:100B00003146FFF77DFF28460CB0BDE8F081002399
:100B1000EBE70D20F8E70120F6E770B590F85530C7
:100B200004460D460BB9002070BD0B8CB0F8502068
:100B30005BBA9BB29A42F6D14B8CB0F852205BBAAA
:100B40009BB29A42EFD100F130063046FEF7A8FC86
:100B500030B910222946304657F0EAFD0028E2D18C
:100B60001022A91804F1400057F0E2FDB0FA80F01D
:100B70004009D9E738B50D4601F5A0410346D1F843
:100B8000740104462CB1A34201D0E469FAE71820AD
:100B900038BDD861C1F87431116819625168926822
:100BA00059629A6221461C22184657F009FF456097
:100BB0002046EDE710B5102204460021083057F01A
:100BC000FFFE00202083206010BD426802F5A04295
:100BD00010B5D2F87441002123464BB1984209D098
:100BE0001946DB69F9E7CB6953B1DB69CB6107E0F3
:100BF000172010BD0029F6D114B1E369C2F8743191
:100C00000023C3611846F4E738B50368012B0D468D
:100C100014D10B8C028B5BBA9BB29A420ED100F1BD
:100C200008042046FEF73CFC38B91022294620462D
:100C300057F07EFDB0FA80F0400938BD0020FCE797
:100C40002DE9F0410D8A86696DBA07460C46ADB2B2
:100C5000D6B1B6F85030AB4202D0D6F81862F7E7FA
:100C60002046FEF71DFC60B906F130084046FEF74D
:100C700017FC30B910222146404657F059FD002894
:100C8000EBD10020BDE8F081FE69C6B1338BAB42E9
:100C900001D0F669F9E72046FEF702FC0028F0D102
:100CA00006F108073846FEF7FBFB0028E9D11022C1
:100CB0002146384657F03CFD0028EAD1E1E7012003
:100CC000E0E738B5054608460C46FEF7E9FBC0B933
:100CD000286800F5A24021465830FFF7B1FF90B1D7
:100CE000234605F1300204F1100153F8040B42F8D9
:100CF000040B8B42F9D1238A5BBAA5F8503000204F
:100D000038BD0720FCE70D20FAE770B505464068BE
:100D10000E8A00F5A24058300C46FFF791FF80B1D3
:100D2000214605F1080304F1100251F8040B43F8C1
:100D3000040B9142F9D176BA01232E832B60002057
:100D400070BD0D20FCE70000F8B504469DF8186062
:100D500015467BB11748FDF79DFE034608B90020F4
:100D6000F8BD2A4600F1100153F8040B42F8040BB9
:100D70008B42F9D1BEB14FF480464FF6FF77238CFA
:100D80002B82BB421ABF01339BB24FF440432384F2
:100D900029462046FFF754FF0028E1D1013EB6B2B4
:100DA000002EECD1DBE729462046BDE8F840FFF7EE
:100DB00047BF00BF58870020F7B50446F4F793FFFC
:100DC00000F100470646013F0023A5698DF8033076
:100DD00001975DB101AB0DF1030231462846FFF7E3
:100DE0009FFD0028F0D1D5F81852F2E79DF80330A6
:100DF0001BB10199201DF8F7DAF803B0F0BD00002F
:100E00000148FFF7D9BF00BF3088002038B584699A
:100E1000054664B12046FFF7D7FD28B105F1100063
:100E2000BDE83840F8F702B8D4F81842F1E738BD09
:100E30000148FFF7EBBF00BF3088002008B5002154
:100E400000F5A140FDF7A4FB28B190F8313043F044
:100E5000010380F8313008BD0846F7F758B906237A
:100E600000F5A140FDF7E0BEF4F73DBFFFF7FCBF82
:100E7000FFF740BD7047D0F830325BB16F2905D025
:100E8000742905D0002918BF022118470121FCE769
:100E90000421FAE7704770B504460D4671B900F1B8
:100EA000180630461AF0E3FB014630461AF01BFCE8
:100EB00065602046BDE8704019F03CBD70BD0FB4C0
:100EC00000B5A3B024AB802153F8042B019302A8F2
:100ED0005BF02CFD23B05DF804EB04B0704700001C
:100EE0000FB400B5A3B024AB802153F8042B0193B9
:100EF00002A85BF01BFD0349034802AAF6F7BCFFFA
:100F0000FEE700BF1B3A0700FF63070010B400F5BF
:100F1000A2409DF80440019458305DF8044BFFF75F
:100F200013BF07B504210DEB0100F8F715FA01987E
:100F300003B05DF804FB40BA80B2704708B5FDF716
:100F400091F808BD036823B1994207D0D3F818324D
:100F5000F9E71720B0FA80F0400970470020F9E760
:100F60002DE9F8430F46164600214FF40672044659
:100F700057F026FD07F5A24021467030FFF7E2FF4B
:100F8000054600284ED107F5A0430146D3F870214D
:100F9000C4F81822C3F870413368C4F81C3273686F
:100FA000C4F82032B368C4F82432F368C4F8283295
:100FB0003369C4F82C327369C4F83032102204F556
:100FC0000D7057F0FDFC2946122204F5177057F0FA
:100FD000F7FC84F86E52D6E90696092306F108025A
:100FE00004F10800B2FBF3F2B61A1AF078FC3246AC
:100FF000494604F118001AF034FB16F0070118BF37
:10100000012109EB060801EBD6014046C4F828800F
:101010001AF07DFA2046656019F08CFC276028469E
:10102000BDE8F8831820FBE72DE9F74F00F118051C
:1010300028460C9F0C4616469846FFF783FF68B378
:1010400094F8553053B33B7BCBB9D4F8243243BB2F
:10105000D4F82832002B54D17B7B002B74D1BB7B7E
:10106000002B71D194F855300A2B17D1D4F83032B7
:10107000A3B10321204603B0BDE8F04F1847D4F8D0
:101080002032002BE1D02046984721462846FFF722
:1010900059FF18B194F85530002BD6D103B0BDE8F4
:1010A000F08F7B68FEB14FF0000BDA467B685B4542
:1010B0001CD0D6F80090BBF1000F09D0214628467D
:1010C000FFF740FF0028E9D094F85530002BE5D019
:1010D000C6F800A03146D4F82432204698470BF1D8
:1010E000010B4E46E2E7002BDDD0FEE72146284605
:1010F000FFF728FF0028D1D094F85530002BCDD031
:10110000A6E72046FFF756FCBB6806460BB94045EC
:101110000FD204F10800D4F828821AF04BFC3246B2
:1011200001462046C04794F86E3223F0040384F849
:101130006E3221462846FFF705FF0028AED094F80E
:101140005530002BAAD087E7D4F82C62002E89D026
:1011500004F1180738461AF08AFAE26A019001325F
:1011600018BF0122384600921AF083FADDE9002107
:1011700003462046B04721462846FFF7E3FE0028F5
:101180008CD06FE72DE9F04F2DED028B98468B88C0
:101190005BBA1FFA83FA8946D38B118C5B1A9A4586
:1011A0009BB08346154606D0062420461BB0BDECF6
:1011B000028BBDE8F08FBAF1130FF5D90C31012382
:1011C0000DF11B0289B22846F7F75FF804460028A4
:1011D000EBD19DF81B301B099B00A3F11402D2B286
:1011E000282A8DF81B30DFD89A45DDDB06224146E0
:1011F000284615F0E1FE04460028D6D19DF81B30A4
:10120000298C0BAA2846F7F740F804460028CCD1D1
:101210000C98FCF727FF0C900D98FCF723FFBDF806
:101220003A30DBF818600D905BBAADF83A30BDF893
:101230003E305BBAADF83E30BDF82C305BBAA8F852
:101240002230BDF82E305BBAA8F820303EB14146BE
:101250003046FFF762FC90BBD6F81862F6E7DBF881
:101260001C70F7B141463846FFF7CEFC40B9FF6924
:10127000F7E70799002998D0002300961A4646E020
:1012800007AE10220021304657F09AFBCDE90076D8
:1012900000232A460BA9484617F03AFF0130E8D14F
:1012A000FEE76F2301939DF81B30AAEB0303009325
:1012B0003A46194B0BA9484616F012FD75E7304621
:1012C00007AF50F8083F08EE103A1AF073FBD6F853
:1012D000D030059004931022D6F8CC30039300212F
:1012E000384657F06DFB00230093019733462A469A
:1012F0000BA9484617F00CFF0130B0D0059A039BAC
:1013000000971344049A9B1A18EE102A3146584647
:10131000FFF78AFE49E700BFD83600202DE9F043E9
:10132000D0F8288087B006460D46B8F1000F24D0CB
:1013300001AFD1F80090144602F1100E3A46206831
:101340006168BC46ACE80300083474456746F6D1D2
:101350005BBA29463046ADF81430C04709F5A240C3
:1013600029467030FFF7EEFD20B195F855000038A2
:1013700018BF012007B0BDE8F0830120FAE72DE98E
:10138000F041D0F8248086B00446B8F1000F04D1B3
:101390004FF0FF3006B0BDE8F08101AE45680B4666
:1013A00001F1100EB44618685968374603C7083370
:1013B00073453E46F7D152BAADF8142061466A46ED
:1013C0002046C04705F5A043D3F87431002BDFD089
:1013D0009C4210D0DB69F9E7009C05F5A24021464C
:1013E0007030FFF7AFFD0028D2D094F85530002BB5
:1013F000CED12046CEE72368002BC9D00028EBD001
:10140000012814BF4FF0FF300020C3E70023C0E9DC
:101410000012C0E9023380F828307047C3688B425D
:1014200030B500D2FEE7D0E901425B1AA51AAB4203
:1014300021BF1B1B9B18836090F82830C16035BF0B
:101440009B18C3F10103836080F8283030BD4268E7
:10145000C068101A70470023C0E9023380F82830B2
:101460007047C368002B14BF0520002070474368F5
:101470008B4200D8FEE78818591A914298BFC01ACB
:1014800070472DE9F84FD0F804B09246C268ABEB34
:101490000208434528BF434604460F461D46002B1D
:1014A00068D002B98260A1682046FFF7E0FF0B9B7D
:1014B00013F00109064605D045452CBF4FF0000941
:1014C0004FF001092068ABEB06084545304429D8A8
:1014D0002A46514657F05EF9F6B9E36894F82810A9
:1014E00013B1C1F10101C9B20C2202FB014300207A
:1014F000186120681946C3E905054A461031384687
:10150000FFF799FA002818BF0025E3682B44E36031
:101510000A9B1D60BDE8F88F4A4629463846FFF70A
:10152000C2FAEFE7A5EB0B0B424651465E4457F07B
:1015300031F932460AEB0801206857F02BF90122F5
:1015400041463846FFF7AFFAB0B994F828300C217D
:10155000C3F101034B43E218103310612168384690
:10156000C2E905164A46E118FFF765FA002818BFD8
:101570004546CAE71846C8E70025C6E738B5028AD7
:101580000B8C9A4204460D4601D0002038BD0B78E2
:10159000FF2B03D1638C6BB90120F7E7FDF780FFC8
:1015A0000028F7D110222946204657F0C1F800281C
:1015B000F0D0EAE76A8C9A42E7D112342046FDF770
:1015C0006FFF0028E8D11022A918204657F0B0F884
:1015D000B0FA80F04009D9E710B534220446002162
:1015E00057F0EEF9204610BD4FF440420280002231
:1015F000C0E9012270474FF2BF03984208D000F5BE
:101600003B50213080B213288CBF0020012070474E
:101610000120704710B584680022234683B19942A7
:1016200007D01A461B6BF9E7136B3BB11B6B1363B7
:1016300004E0002AF8D10CB1236B836000230B6314
:1016400010BD028810B501464FF6FF74A2421ABFC2
:10165000013292B24FF440421046FFF7CCFF00280F
:10166000F4D10A80104610BDF8B5064610460D4666
:101670001446FDF715FF88B122462B4604F11007EA
:10168000106851681C4603C40832BA422346F7D199
:10169000128822802C8A4CB10020F8BD06482146D1
:1016A000FEF7E0FE0028E7D10720F6E73046FFF717
:1016B000C8FF28822046F0E75488002013460A46D7
:1016C00001460148FFF7D0BF8487002030B587B0BE
:1016D00004461546ADF814101022002101A857F059
:1016E0006FF92A4601A92046FFF7E8FF07B030BD91
:1016F00030B401F1120302F1100452F8045B43F814
:10170000045BA242F9D112881A800B8A23B930BC3B
:1017100001230A46FFF7A8BF002030BC7047000035
:101720000831024889B2FCF729BF00BF5887002062
:101730000148FFF7F5BF00BF8487002037B5138C41
:101740005BBAADF80030538C5BBAADF80230CB8B8E
:1017500008330C465BBA1546ADF804300822002366
:1017600069462046ADF80630F6F72CFE48B901462A
:101770002046F6F7F7FC044811232A462146FDF7D8
:1017800053FA03B030BD00BF588700202DE9F04167
:1017900016461A8C8AB005460C4632B1098A914227
:1017A00003D007200AB0BDE8F0816A4603F1200E9D
:1017B0001746186859689446ACE803000833734527
:1017C0006246F6D11868CCF800009B88ACF804306B
:1017D00004A8FDF765FE98B104F112084046FDF734
:1017E0005FFE0028DDD1434604AA04F1220E1868EA
:1017F00059689446ACE80300083373456246F6D155
:10180000BDF8223023B9638C002BCAD0ADF822304A
:101810003846FDF745FE58B12346BC4604F1100E8C
:1018200018685968624603C2083373459446F7D175
:10183000238A43B1238AADF820303A463146284600
:10184000FFF77CFFAEE70123224621462846FFF73B
:101850000BFF0028EED0A5E713460A4601460148D3
:10186000FFF794BF8487002070B585680C46164644
:10187000ADB131462846FFF781FE40B92D6BF7E741
:101880006B6AA86A32462146BDE870401847218C31
:101890002046F6F77FFC238C002BF1D0FEE770BDCD
:1018A0002DE9F3410D468046098C164608236A4609
:1018B0002846F6F7EAFC044610BB112231462846BA
:1018C00015F07AFB0446D8B908212846F6F73EFC05
:1018D000BDF80030D8F804705BBA7384BDF80230EC
:1018E0005BBA33843FB17B68B86832462946984773
:1018F00030B93F68F6E7324629464046FFF7B4FF65
:10190000204602B0BDE8F081806828B1038A8B428E
:1019100001D0006BF9E701207047000044F64C53FA
:10192000994210B50C460AD04FF2BF03994206D037
:101930000448FBF7D9FE001B18BF012010BD002092
:10194000FCE700BFD8B5002003681BB1994206D060
:101950001B6BFAE71720B0FA80F0400970470020AF
:10196000F9E71222002157F02BB82DE9F04100F1E0
:101970000808054640460C4617461E46FFF7E4FF9A
:1019800000B1FEE72046FFF7ECFF04F11200FFF77D
:10199000E8FFC4E9097621464046FFF7D5FF10B9B4
:1019A000AB682363AC600020BDE8F08113460A46B3
:1019B00001460148FFF7D9BF8487002038B50546A6
:1019C00008300C46FFF7C0FF50B121462846FFF70C
:1019D00021FE2046FFF7C5FF04F11200FFF7C1FF0B
:1019E000002038BD01460148FFF7E8BF848700208A
:1019F0000148F4F7D5BA00BFD83600200148F4F703
:101A0000E1BA00BFD83600200148F4F775BB00BF2B
:101A1000D836002000F5004393F8303113B113306D
:101A200015F078BC704700F5004393F8303113B1DE
:101A3000133015F075BC704710B400F5004494F8ED
:101A4000304124B15DF8044B133015F06FBC5DF8E4
:101A5000044B704700F5004393F8303113B1133055
:101A600015F06ABC704700000048704700F8FF0797
:101A700008B5FFF7F9FF08BDF5F7AEBB00207047CA
:101A8000FF207047FF207047704700002DE9F041AC
:101A9000D2E9007506460C4600F5816800F20C415B
:101AA00006F2144C00F5826043466DB93FB14745DC
:101AB00008D08F42034602D0874262D163461D6838
:101AC0001F46F1E70B46FAE7698A4FF6FF73994222
:101AD0001DBF47F6681303EB41132B49002318BFC2
:101AE0005B18C2E9007300212C22204656F068FFE3
:101AF0002B46A44605F1100E18685968624603C2C9
:101B0000083373459446F7D12B8A238247451AD16F
:101B1000E37C43F00103E3746B69E27C013318BF9B
:101B2000012363F38202E2746B695A1C09D063617A
:101B3000164904F11800FDF757FDAB692362EB6904
:101B4000636200201EE006F20C439F420BD101238A
:101B5000A3742A7EE37C62F30003E374AB8A2385DB
:101B6000EB8A6385EDE706F58266B74201D1022371
:101B7000EEE70323A3746A7EE37C62F34103E3741C
:101B8000E7E71720BDE8F081D8360020008F00205D
:101B900008B908687047438A4FF6FF7293421FBF27
:101BA00047F6681000EB4310024BC01808BF002036
:101BB000704700BFD83600202DE9F04F87B01E4691
:101BC00000F58163029300F20C430393002500F5B6
:101BD0008263DFF854B0049300F214401746059076
:101BE000A8464FF6FF7947F6681A02AB53F825303E
:101BF0003B601C68C6F8008074B110222046019139
:101C000056F096FD60B13460648A01994C4503D06A
